:1000000080540020B535010045E701006D35010041
:100010006D3501006D3501006D35010000000000F7
:10002000000000000000000000000000F9260100B0
:100030006D35010000000000A12601006D350100B2
:10004000D927010041FE0100D9270100D92701006D
:10005000D9270100D9270100D9270100D92701009C
:1000600009FE0100D9270100D927010027FE010060
:10007000D9270100D9270100D9270100D92701007C
:10008000D9270100D9270100D9270100D92701006C
:10009000D9270100D9270100D9270100D92701005C
:1000A000D9270100D9270100D9270100D92701004C
:1000B000D9270100D9270100D9270100D92701003C
:1000C000D9270100D9270100D9270100D92701002C
:1000D000D9270100D9270100D9270100D92701001C
:1000E000D9270100D9270100D9270100D92701000C
:1000F000D9270100D9270100D9270100D9270100FC
:1001000053B94AB9002908BF00281CBF4FF0FF317E
:100110004FF0FF3000F00CB8ADF1080C6DE904CEE3
:100120000CF000FADDF804E0DDE9022304B07047CA
:10013000704700BF01480078704700002800002089
:1001400070B50CF08DFC134C6FF0270528B90CF03E
:10015000BDFC10B90CF0C4FC20B10F4860606570A4
:10016000082010E00CF051FC40B90CF058FC28B904
:100170000CF06CFC10B90CF07DFC30B1064831304D
:10018000606065700420A07070BDE821742003F0E9
:1001900019FB00002800002036030100074991F9EF
:1001A0000220904203DA91F90120904201DC1046CE
:1001B00070474968801A08567047000028000020E0
:1001C0002DE9F0411C4690460D4606466FF0150796
:1001D000042804D81CB10CF0F8FAA84202D838461A
:1001E000BDE8F0810548424650F8260018B1405756
:1001F000824200DD024622700020F1E7F008002074
:1002000001480078704700003000002005490A7856
:10021000904201D300207047496800EB400001EB99
:1002200000107047300000200E4910B591F82D00E5
:10023000202812D091F82D00A1F58062C0EBC000FB
:1002400002EB800091F82D104068C1EBC10152F81B
:100250002120BDE810400421104740F6870170209E
:1002600003F0B0FA040D002070B50546202A28D00E
:1002700019481A4C00EB831C03EB43030CEB4200C0
:100280002344202922D00CEB410140784C7848705F
:10029000204601460CEB4100914205704078F8D1B0
:1002A00093F82220202A1ABF0CEB4202547083F8E4
:1002B000214020220CEB410C8CF8012083F8221005
:1002C00070BD40F29221702003F07CFA93F8204038
:1002D000407883F82000DBE7840C0020040D002028
:1002E0002DE9FF4F85B015460C4602F0CBF92844A6
:1002F00020F07F4102912068401A0002C11700EBF4
:1003000011600012002800F3F080DDF82080CA4858
:1003100008EB48010844039090F820502020C74E75
:10032000EA460DF104098DF80000202D1CBFC448D9
:1003300000EB881B39D000BFC5EBC50006EB800081
:1003400000F10801C0682768381A0002C21700EBE4
:100350001260001229D4E08900B3C889F0B9086896
:10036000049003F0A3F8B0F5C67F08BF0D200BD0B2
:10037000A0F54070563808BF1C2005D0A0F50070CD
:100380009F3814BF00203220411C0498381A000204
:10039000C21700EB12600012884206DB0BEB45002F
:1003A0008AF800504578202DC6D19AF8000089F8C7
:1003B0000000202D1CBFA24800EB881B00F03881F4
:1003C000C5EBC50006EB80076068D7F8088007F129
:1003D0000801A8EB00000002C21700EB1260001237
:1003E00027D4C889002800F02381E089002840F044
:1003F0001F81D4F800A003F059F8B0F5C67F08BFFC
:100400000D200BD0A0F54070563808BF1C2005D039
:10041000A0F500709F3814BF00203220411CA8EBCB
:100420000A000002C21700EB12600012884280F23C
:10043000FF8089F80050397E207C814206D90BEB81
:1004400045004578202DBBD100F0F2B89DF804009E
:10045000C0EBC00006EB8000C18AC568E1BBE18942
:10046000D1B3876803F022F8B0F5C67F08BF0D202E
:100470000BD0A0F54070563808BF1C2005D0A0F561
:1004800000709F3814BF00203220411CE81B00027E
:10049000C21700EB1260001288421DDA03F006F862
:1004A000B0F5C67F08BF0D200BD0A0F540705638C0
:1004B00008BF1C2005D0A0F500709F3814BF002095
:1004C00032209DF80410401CC1EBC10106EB8101F4
:1004D0008968084420F07F450298281A0002C11755
:1004E00000EB11600012002803DD09B00020BDE818
:1004F000F08FD4E90010401A284425F07F4120F005
:100500007F40C4E90010089804900398EA460DF172
:10051000040890F8205020208DF80000202D3CD0B9
:100520004748049900EB811BC5EBC50006EB800032
:1005300000F10801C0682768381A0002C21700EBF2
:100540001260001229D4E08900B3C889F0B9D1F84B
:10055000009002F0ABFFB0F5C67F08BF0D200BD0B6
:10056000A0F54070563808BF1C2005D0A0F50070DB
:100570009F3814BF00203220411CA7EB0900000265
:10058000C21700EB12600012884206DB0BEB45003D
:100590008AF800504578202DC6D19AF8000088F8D6
:1005A00000000498202D1CBF254901EB801B3FD083
:1005B000C5EBC50006EB80076168D7F8089007F126
:1005C0000800A9EB01010902CA1701EB1261091227
:1005D00022D4C08960B3E08950BBD4F800A002F0F7
:1005E00065FFB0F5C67F08BF0D200BD0A0F54070A9
:1005F000563808BF1C2005D0A0F500709F3814BFE6
:1006000000203220411CA9EB0A000002C21700EBB7
:100610001260001288420BDA88F80050387E217C84
:1006200088427FF613AF0BEB45004578202DBFD1F4
:1006300009B00120BDE8F08F040D0020040900205E
:10064000840C00202DE9F84F0F46064601EB4700C9
:100650004B4999460844924690F82040202010705B
:10066000A1F58068202C1CBF464800EB871B38D0C2
:10067000C4EBC40008EB800000F10801C0683568D5
:10068000281A0002C21700EB1260001229D4F08968
:1006900000B3C889F0B90868009002F007FFB0F510
:1006A000C67F08BF0D200BD0A0F54070563808BF9C
:1006B0001C2005D0A0F500709F3814BF0020322008
:1006C000411C0098281A0002C21700EB12600012A9
:1006D000884206DB0BEB44008AF800404478202C6B
:1006E000C6D19AF8000089F80000202C1CBF2548CC
:1006F00000EB871A40D000BFC4EBC40008EB8007B2
:100700007068BD6807F10801281A0002C21700EBE3
:100710001260001222D4C88970B3F08960BBD6F889
:1007200000B002F0C3FEB0F5C67F08BF0D200BD0AD
:10073000A0F54070563808BF1C2005D0A0F5007009
:100740009F3814BF00203220411CA5EB0B00000293
:10075000C21700EB1260001288420DDA89F80040DF
:10076000387E317C884202D80020BDE8F88F0AEB41
:1007700044004478202CBFD10120BDE8F88F000050
:10078000040D0020840C00202DE9F04182B00546C4
:1007900014468846D08901AA694601F08FFF02F00D
:1007A000B7FC01F06FFF0746204890F82D10202974
:1007B00004D0C068401D20F07F4124E0E08905F1AD
:1007C0000906B0B102F086FF98B902F06FFEB0F5ED
:1007D000C67F08BF0D200BD0A0F54070563808BF6B
:1007E0001C2005D0A0F500709F3814BF00203220D7
:1007F0000644B8F1000F04D10098874284BF381A2C
:10080000064426F07F41D4E90020801A084420F0F5
:100810007F40C4E90010A94224BF02B0BDE8F081C6
:10082000A068401CA06002B0BDE8F081040D00206B
:100830002DE9F04F97B017468B46054602F0D0F9E8
:10084000044602F065FC0646BBF1010F18BFBBF180
:10085000020F05D040F65D114FF0700002F0B2FFBC
:10086000F84901200860F8498968086000208DF87F
:100870004E000C90401E0D90F449C7EBC70001EBF1
:10088000800000F108010DF1380891E80E1088E8A9
:100890000E10806912900EA800F0C4FB0790EC487F
:1008A000BDF84680808BADF84C00B8F1000F04BF56
:1008B000002006900BD001200690E54890F82A0011
:1008C00028B902F007FF002808BF012700D0002741
:1008D00002F0ECFDB0F5C67F08BF0D200BD0A0F5EF
:1008E0004070563808BF1C2005D0A0F500709F3816
:1008F00014BF002032204FF00009CA460B90464535
:1009000038D90799DFF84C936FEA060C6B4616AAA4
:1009100001EB0C00494504D940F26F51702002F000
:1009200051FFCD498C4504DD4FF4AE61702002F0DB
:1009300049FFCA498C4504DA40F27151702002F037
:1009400041FFC7498142DCBF00F5F700A0F1F85034
:1009500005DD0028BCBFA0F5F70000F1F8501946EE
:1009600001F0ACFE00980E9920F07F400090081A2C
:1009700020F07F49002F18BFDDF82CA005D19DF88D
:100980004C00002818BF4FF0020AB4F1807F08D055
:100990000E98001B0002C11700EB11600012012825
:1009A00001DA03200DE057B1A94890F82B0030B1CF
:1009B0009DF84C0010F1000A18BF4FF0020A2546BE
:1009C000002082440E98A0EB090020F07F42501EC8
:1009D00020F07F40411B0902CB1701EB1361091284
:1009E000514504DBB9F1000F18BF0E922DE0B9F1AB
:1009F000000F05D09DF84D0020B902F07FFB08B133
:100A0000AFB90CE02FB99DF84C00002818BFAAF12F
:100A1000020A4FF000098DF84C904E4607E09DF811
:100A20004C0020B100208DF84C00AAF1020A0E986B
:100A3000A0EB0900401E20F07F40411B0902CA17AD
:100A400001EB1261091251457EDB149705464FF008
:100A50000009069F01F09CFF281A0002C11700EB55
:100A600011604FEA202A02F021FDB0F5C67F08BFD1
:100A70000D200BD0A0F54070563808BF1C2005D0C3
:100A8000A0F500709F3814BF002032200B30824543
:100A900020DABBF1010F02D0149840B112E0B4F19A
:100AA000807F1CD140F6DE01702002F08BFEB4F195
:100AB000807F07D0601B0002C11700EB116000129D
:100AC000042804DD2C46204601F088FF07E00028BA
:100AD00063DC04E02C46204601F080FFB946B4F107
:100AE000807F55D00E980F9A001B121B20F07F407C
:100AF00022F07F42012850D3B0F5000F98BFB2F525
:100B0000000F4AD820460BF099FE0799524A0D1A59
:100B10004FF0000AAA1A7AF1000218D34E4B421A7B
:100B2000D31A7AF1000312D34A4BAB423EBFC0F551
:100B3000902000F1F450451809D3934231D2C1F509
:100B4000902101F1F45100E027E008444542404F74
:100B5000B87F58B3BBF1010F05D0022002F07AF93B
:100B6000012002F077F9B0452CD2A5EB06014FF039
:100B7000020002F0B9F890B3B8F1000F1CBFA5EB6A
:100B80000801012034D000BF02F0AEF838B32FE0E6
:100B900040F6F111702002F015FE17B00020BDE8FC
:100BA000F08F40F6C221702002F00CFEB04534BF39
:100BB000304640461E30A842CCDB40F6052170206E
:100BC00002F000FE0CD9A5EB0801012002F08CF820
:100BD00028B1002E1CBFA91B022009D0D4E730E0A9
:100BE00056EA080004D040F64111702002F0EAFDF8
:100BF0002946002002F078F818B30698012600284C
:100C000004BF97F82B00002802D0B9F1000F33D0B1
:100C100097F82A0018B102F04FFC87F82AA0B9F122
:100C2000000F2CD00B98201A20F07F41052002F0F5
:100C30005BF8E0B397F82B00002808BF87F82B601B
:100C400025E00FE0080500403800002004090020DE
:100C5000040D0020FF7F841E0040420F00C0BDF045
:100C60000080841E022002F0F5F8012002F0F2F864
:100C700017B00020BDE8F08F97F82A0090B197F8E0
:100C80002B0020B1052002F0E5F887F82BA0A5EB9A
:100C90000800A0F1190100290FDC40F62E21702078
:100CA00002F090FD02F024FC87F82A60B7E7FFE726
:100CB00040F2F221702002F085FD032002F014F8CA
:100CC000C0B10F488068C0F800A00E48C0F800A06E
:100CD0000CAC94E80F0038607960BA60FB6010AC2F
:100CE00094E80F0038617961BA61FB6117B00120A7
:100CF000BDE8F08F40F63621702002F063FD000061
:100D000038000020080500402DE9F05F064608780D
:100D10009074C87A5074887A10740889D081DFF88A
:100D2000988170689A46A0FB087914460D46306891
:100D30000BF084FDC11928784FEA680C49F10002D4
:100D4000A8F1010ECCF1000B68B1E089677CC043CB
:100D5000D5F8049004F10C0260455FDD4FF4AE61FC
:100D6000702002F02FFDDFF85491D5E9040311EB58
:100D7000090A42F10009B0EB0A0A73EB090945D2EE
:100D8000411A73EB020141D3C71B7068A06047454D
:100D900005D3401CA7F1F457A7F59027A060E08980
:100DA0006D68C143667C781804F10C02774504D95C
:100DB00040F26F51702002F005FD6145CEDC5945CF
:100DC0002FDB8045DCBF00F5F700A0F1F85005DD12
:100DD0000028BCBFA0F5F70000F1F850214601F053
:100DE0006DFC206820F07F417819401C2160002EA6
:100DF00008BF7A3003D0012E08BF483034D101F04B
:100E000041FC20F07F406060BDE8F09F3068401EEC
:100E100020F07F40206000F57A70F4E701465845E5
:100E200004DA40F27151702002F0CCFC8045DCBF46
:100E3000A1F1F450A0F5902005DD0028BCBF01F120
:100E4000F45000F59020214601F038FC2068002F76
:100E500020F07F4109F10100216008BF7A3008D0FD
:100E6000012F08BF483004D040F22461702002F006
:100E7000A9FC01F007FC20F07F4161607068A06070
:100E8000002122463068FFF77FFC32685346214636
:100E90002869FFF725FA002818BFBDE8F09FD4E9BC
:100EA00000213068891A20F07F42084420F07F40FA
:100EB000C4E90020BDE8F09F0080841E0040420F7E
:100EC00070B51E4D95F82D00202818BF70BD95F8FF
:100ED0002C2002EB4200284490F82040202C27D000
:100EE000174B03EB821101EB4401497880F8201085
:100EF000FF2085F8290085F82D402146022000F0CA
:100F0000CBF8002085F82800A8770E49C4EBC40070
:100F100001EB8000007E002808BF02F05FFE002089
:100F200009494968002908BF70BDBDE870400847FD
:100F30004FF44B71702002F045FC0000040D0020BE
:100F4000840C002004090020380000202DE9F05F07
:100F5000DFF8C08098F82C5005EB4500404490F82D
:100F60002140202C08BFBDE8F09FDFF8ACB0DFF8CF
:100F7000ACA0AAF560790AEB8517072617F81400CC
:100F800001280ED0042808BF02260AD005280CBF6D
:100F90000326062805D040F6A8014FF0700002F0A5
:100FA00011FCBBF1000F18BFAFF30080EFF310800E
:100FB00072B607EB44014A7805EB4501414481F8DC
:100FC000212091F82220A24204BF202281F8222071
:100FD000C0B12A462146012000F05EF8C4EBC401EE
:100FE00009EB810059F8212040683146904798F874
:100FF0002C5005EB4500404490F82140202CBAD1FC
:10100000BDE8F09F0648002818BFAFF3008062B625
:10101000DFE70000040D002000000000840C002029
:101020000000000010B5044600680BF007FC024603
:10103000E089217B144B0844411C50189A4204D982
:1010400040F26F51702002F0BDFB104A914204DD66
:101050004FF4AE61702002F0B5FB0D4A914204DA04
:1010600040F27151702002F0ADFB0A498142DEBFAF
:1010700000F5F700A0F1F85010BD0028BCBFA0F5A6
:10108000F70000F1F85010BDFF7F841E0040420FB2
:1010900000C0BDF00080841EDFF858C010B50023EA
:1010A0000CEB821C07281FD2DFE800F005050505C0
:1010B0000404040001230CF81100002B08BF10BD2C
:1010C00002EB42020C48024492F8220020280EBF94
:1010D00082F821100CEB4000417020200CEB410302
:1010E000587082F8221010BD4FF41A71702002F06F
:1010F00069FB0000840C0020040D00202DE9F74F4F
:101100001746DFF858A102EB47005044884690F894
:1011100020400129254618BFB8F1020F05D040F63E
:101120006C214FF0700002F04DFB4FF0000B202DB2
:1011300044D09AF81E000026002808BF022601F0BD
:1011400027FC474BC4EBC40103EB81018A68C968E3
:10115000121A091A22F07F4221F07F41964299BF6C
:10116000B2F5000FB1F5000F3E4A02EB871923D903
:10117000224609EB42014C78202C15D0C4EBC40167
:1011800003EB810CDCF80810DCF80CC0091A21F024
:101190007F41ACEB000C2CF07F4C8E429CBFB1F534
:1011A000000FBCF5000FE3D8202A05D03B462021D4
:1011B0000420FFF759F80446AC420FD19AF82E00EC
:1011C00020280FD00099DAF80800891C081A0002BC
:1011D000C11700EB11600012002803DD03B00020EE
:1011E000BDE8F08F202D16D02A4641460098FFF723
:1011F0001FFB00281FBF8AF82E50022003B0BDE855
:10120000F08F3B462A4620210420FFF72DF803B03B
:101210000020BDE8F08F9AF82A0018B102F04CF9CE
:101220008AF82AB09AF82B0020B1052001F012FEAE
:101230008AF82BB0042001F00DFE01F07BFE202087
:101240008AF82E0008488068C0F800B00748C0F847
:1012500000B003B00120BDE8F08F0000040D0020B5
:1012600004090020840C00203800002008050040FC
:101270002DE9F04F694E07468DB096F82D0088464F
:10128000202855D096F82D0006F10804C0EBC000C8
:10129000A6F5806909EB800A20208DF8200096F8D9
:1012A0002C000AAA00EB4000304409A990F8205015
:1012B000F06802903068384401F000FADAF80C0067
:1012C0000999652F084438D3554A0021D21B71EB88
:1012D000010232D32268821A22F07F42B2F5000F57
:1012E0002BD820F07F406060304684F8108090F862
:1012F0002C000DF1200A202D1CBF4A4901EB801B58
:1013000050D000BFC5EBC50009EB80086168D8F874
:10131000086008F10800711A0902CA1701EB12618E
:1013200009122DD4C08900283CD0E08948B139E0A9
:101330004FF43361702002F045FA0DB00120BDE892
:10134000F08F20680C9002F0B1F8B0F5C67F08BFAE
:101350000D200BD0A0F54070563808BF1C2005D0DA
:10136000A0F500709F3814BF00203220411C0C985B
:10137000301A0002C21700EB12600012884211DA24
:101380008AF8005098F81810207C814205D80298FD
:1013900060600DB00220BDE8F08F0BEB4500457892
:1013A000202DAFD1052001F055FD1C4C4FF0FF3032
:1013B000606094F82C309DF820202021202A03D052
:1013C0000520FEF751FF04E003EB4300204490F8B2
:1013D000200094F82C20134901EB821194F82D2061
:1013E00001EB42014870206838442060FF2084F8F7
:1013F0002900607E012805D1E068401E20F07F4072
:1014000001F08CFB9DF82000202803D0064840788E
:1014100002F0ACFA0DB00020BDE8F08F040D002002
:101420000040420F840C00203800002070B5244A90
:1014300092F82D1020293AD092F82D10A2F5806351
:10144000C1EBC10103EB810C92F82C1092F82C40F7
:1014500001EB4101114491F82010A2F1800505EB48
:101460008414202928D0C1EBC10503EB85052D7E0E
:10147000854284BF04EB41014978F2D8C1EBC10138
:1014800003EB8101DCF80C0089681468081A00027B
:10149000C11700EB1160001207D40BF0CFF904F173
:1014A0006501884224BF001B70BD002070BD40F65E
:1014B0000231702002F086F94FF0FF3070BD00005D
:1014C000040D0020C0EBC00170B50748074A00EBCF
:1014D000810001690830A1FB0245FFF7A3FD001957
:1014E00045F1000170BD0000040900200080841E49
:1014F000F8B56B4D6B4A05F58064012694F82A1007
:1015000008287CD2DFE800F0047097A9C741AEB389
:1015100019B901F0EDFF84F82A60E08A10B102F0F9
:10152000D9F880B1FFF7CCFCFF2084F82700616870
:10153000B1F1FF3F03D0052001F0D6FB40B1607E42
:10154000012810D109E040F63401702002F03AF988
:1015500040F63901702002F035F9E068401E20F0B5
:101560007F4001F0DBFA94F82D0094F82D10C0EBC9
:10157000C00005EB80004068C1EBC10155F8212097
:1015800001B00121BDE8F040104794F82B0040B1B4
:1015900019B901F0ADFF84F82A60002084F82B000F
:1015A000F8BDFFF78DFC4FF0FF30606094F8270026
:1015B0008DF800009DF8000088B194F82D0094F893
:1015C0002D10C0EBC00005EB80004068C1EBC101ED
:1015D00055F8212001B00621BDE8F04010474FF436
:1015E0000561702002F0EEF8FFF76AFC84F82660CF
:1015F00002F070F820B194F82A0030B109E04AE016
:1016000040F65E01702002F0DDF801F071FF84F811
:101610002A6094F82D0094F82D10C0EBC00005EB63
:1016200080004068C1EBC10155F8212001B00021C4
:10163000BDE8F040104701F04DFDE08A10B102F026
:1016400049F828B101F05AFD002818BF6677F8BDA7
:1016500040F66801702002F0B5F813480660906803
:101660000660F8BD1078BDE8F84002F07FB9FFF7DA
:1016700027FC94F82D0094F82D10C0EBC00005EB6A
:1016800080004068C1EBC10155F8212001B005215F
:10169000BDE8F040104740F67B01702002F092F860
:1016A0000409002038000020080500402DE9F34F10
:1016B0008246F04895B00068EF4DC005C00D0ED0D1
:1016C000103840B20028B8BF00F00F0000F1E02051
:1016D000ACBF90F8000490F8140D40090DD0169896
:1016E0004FF0000B0078002818BF012818D040F2F6
:1016F00004714FF0700002F065F895F82D004FF07E
:10170000010B202807D01698007848B14FF4E0610B
:10171000702002F057F840F2FD61702002F052F89C
:10172000D64C24B1002140F20770AFF300800020B6
:10173000CDE91000D249CAEBCA0001EB80004FF09E
:101740000109009024B1002140F21270AFF3008033
:10175000B9F1000F0AD000BF95F82C604FF00008D7
:1017600085F82980BBF1000F07D038E0C548002874
:1017700018BFAFF3008062B6EEE73746012020EADB
:101780000706C148402200EB871100EB86100BF0E2
:10179000B1F924B1002140F22F50AFF3008007EBE4
:1017A000470106EB4600294428440A8C028491F83C
:1017B000221080F8221024B1002140F23350AFF300
:1017C000008024B1002140F21C70AFF3008095F836
:1017D00029008DF808009DF808000028B2D124B136
:1017E000002140F22670AFF3008002A801F0D6F885
:1017F000DDE90201CDE90E01334609AA0EA81699CA
:10180000FFF782FA24B1002140F22D70AFF300807F
:101810009D4A0E9902EB861709A817F81A20012A8B
:1018200018BF022A38D1099A0A9BA2EB010222F0C2
:101830007F42A3EB0101CDF8448021F07F41022AD1
:1018400064D3B2F5000F98BFB1F5000F5ED84FF02A
:10185000010814AB13AA3146FEF7F4FE00285DD050
:101860009DF84C109DF8502033468A425AD00520EE
:10187000FEF7FAFC07EB4A0148709DF84C0020285F
:101880001CBF07EB400080F801A057D032465146FC
:101890005FF00300FFF700FC24B1002140F232703A
:1018A000AFF300807948002818BFAFF30080EFF352
:1018B000108972B624B100214FF4E760AFF30080C5
:1018C00095F829008DF808009DF8080000287FF49D
:1018D00039AF24B100214FF4E860AFF3008009AFC5
:1018E000009897E80E1000F10807B8F1000F87E89C
:1018F0000E100D99816153D024B1002140F24D703A
:10190000AFF30080BBF1000F3AD11FE032465146E1
:101910000420FFF7C1FB4FF00108BDE732465146F6
:101920000420B7E7202919BF07EB4100407806EBF8
:101930004600284408BF90F820009BE706EB4601CC
:10194000294481F820A0CDF844809FE7119810F039
:10195000FF0F15D095F82D00202811D124B10021BA
:1019600040F25270AFF30080324602210E98FFF72A
:10197000C5FB109020B916980078F0B101282BD043
:1019800024B1002140F26F70AFF30080FF20BBF163
:10199000000F18BF85F8290027D000BF4FF00108BD
:1019A00024B100214FF4F060AFF300801098384E5E
:1019B000022823D0012829D02DE024B1002140F2B3
:1019C0005A70AFF3008095F82C2051460420FFF7A1
:1019D00063FB4FF00108E3E7002C3FF4B3AE0021B6
:1019E00040F26570AFF30080ACE695F82C20012141
:1019F000914385F82C1085F82900CFE7A8680E9947
:101A0000401A0AF01BFF716821B904E071684FF0B9
:101A1000FF3001B18847B9F1000F24D024B1002173
:101A20004FF4F260AFF30080B8F1000F11D095F8D9
:101A30002C0000EB4000284490F82100202808D01A
:101A400024B1002140F29770AFF30080707801F06C
:101A50008DFF24B1002140F29C70AFF3008017B0DD
:101A60004046BDE8F08F0748002818BFAFF300805C
:101A700062B6D3E704ED00E0040D00200000000092
:101A80000409002000000000840C00200000000079
:101A9000380000202DE9F14FC9488AB00068C00520
:101AA000C00D11D0103840B20028B8BF00F00F00B0
:101AB00000F1E020ACBF90F8000490F8140D40094C
:101AC00008BF4FF0010B01D04FF0000B0A980078CF
:101AD00000281EBF00200BB0BDE8F08F4FF0000AB9
:101AE000B84DB94CD14625B1002140F2B950AFF301
:101AF000008094F82C6084F829904FF0000825B1FC
:101B0000002140F2BE50AFF30080BBF1000F23D1A3
:101B10003746012020EA0706AC48402200EB871137
:101B200000EB86100AF0E6FF25B1002140F22F50AD
:101B3000AFF3008007EB470106EB46002144204449
:101B40000A8C028491F8221080F8221025B100211D
:101B500040F23350AFF3008025B1002140F2C6506F
:101B6000AFF3008008A800F019FFDDE90801CDE916
:101B7000060133466A4606A80A99FFF7C5F825B15B
:101B8000002140F2CC50AFF3008094F82D002028C3
:101B900019D0E0680099091A0902CA1701EB12610D
:101BA000091210D5DDE90021891A20F07F4308448D
:101BB00020F07F40CDE90030934202D20298401CD1
:101BC00002904FF001084DB1002140F2DF50AFF319
:101BD0000080002140F2E550AFF3008000990698A4
:101BE000019A091A101A21F07F4120F07F40B1F5C7
:101BF000000F98BFB0F5000F03D8BBF1000F0CD158
:101C000003E0BBF1000F39D0C0E0334669467048AD
:101C1000069AFEF765FB48EA0008B8F1000F23D0EA
:101C200000980AF00BFEBDF80E109DF80C20694BD1
:101C30001144491C4218984256D8654881427CDCC0
:101C4000404281427ADB581C9042DCBF02F5F70229
:101C5000A2F1F85205DD002ABCBFA2F5F70202F19D
:101C6000F8520A98C0E904294FF0010A002D7CD0EF
:101C700000214FF4BF60AFF3008087E00798029027
:101C8000BDF80E0008AA05A9DDF8188000F016FDC1
:101C900001F03EFA00F0F6FC074694F82D002028EB
:101CA00027D0E068401D20F07F4000BFDDE9002123
:101CB000891A0090084420F07F4001900098404528
:101CC00002D20298401C02901F208DF80C00009850
:101CD0000AF0B4FDBDF80E109DF80C203D4B1144E8
:101CE000491C421898422AD940F26F51702001F0E5
:101CF00069FDBDF80E0008F10906B0B101F0EAFC7B
:101D000098B901F0D3FBB0F5C67F08BF0D200BD00A
:101D1000A0F54070563808BF1C2005D0A0F5007013
:101D20009F3814BF4846322006440598874284BF36
:101D3000381A064426F07F40B8E703E00AE024485A
:101D4000814204DD4FF4AE61702001F03BFD22487A
:101D5000814204DA40F27151702001F033FD1F48D6
:101D60009042D8BF02F5F70200E00FE0D8BFA2F121
:101D7000F85205DD002ABCBFA2F5F70202F1F852C5
:101D80000A984FF0010AD046C0E904291AEA080F60
:101D900009D00A981149029BD0E90420E3FB0120F5
:101DA0000A99C1E9042094F829008DF814009DF8DF
:101DB000140000287FF497AE0BB05046BDE8F08FBA
:101DC00004ED00E000000000040D0020840C002061
:101DD0000040420FFF7F841E00C0BDF00080841EC3
:101DE0002DE9F14F944D8CB095F82C00002009900E
:101DF00006900120A5F180094FF0000807468F4C9E
:101E0000CDF81C0000F0C4FD089024B100214FF46F
:101E1000F660AFF30080079800283CD085F8298051
:101E200024B1002140F2B570AFF3008095F82CA0EA
:101E3000402227EA0A0609EB861009EB8A1183463D
:101E40000AF058FE24B1002140F22F50AFF3008079
:101E500006EB46000AEB4A012844294400900A8C0C
:101E6000028491F8221080F8221024B1002140F25F
:101E70003350AFF3008095F829008DF808009DF8E5
:101E8000080078B1002C1CBF002140F2BB70B9D013
:101E9000AFF30080B6E76A48002818BFAFF30080B0
:101EA00062B6BBE724B1002140F2BF70AFF30080FF
:101EB0000C981BF8100003287DD1009A0C9992F819
:101EC0002000884214BF4FF0000A4FF0010A02F1CF
:101ED000200C8346202209EB861303E0024603EB25
:101EE00042004078884202D020280AD0F6E7202815
:101EF00007D0834507D103EB4B0040788CF80000F6
:101F000007E040460CE003EB400003EB4201407861
:101F1000487024B1002140F29A40AFF30080384667
:101F2000C34610EA0A0F18BFBB4600284FD024B1A1
:101F3000002140F2C470AFF30080324601200C99BA
:101F4000FFF7AAF824B1002140F2CD70AFF3008072
:101F50003C48002818BFAFF30080EFF3108072B642
:101F6000079024B1002140F2D270AFF3008095F8C1
:101F700029008DF808009DF8080038B1002C1CBF1E
:101F8000002140F2D6703FF43DAF81E7BBF1000F76
:101F90000AD095F82D00202806D132460221089853
:101FA000FFF7ACF80690F8B124B1002140F2EA70D6
:101FB000AFF3008000E00AE095F82C0027EA00006B
:101FC00085F82C00FF2085F829000120099024B114
:101FD000002140F2F370AFF3008006981A4E0228F9
:101FE00009D001280FD013E094B1002140F2E57030
:101FF000AFF30080ECE7A9680898081A0AF01EFC05
:10200000716821B904E071684FF0FF3001B1884771
:10201000079848B124B1002140F60700AFF30080D3
:1020200009980DB0BDE8F08F0548002818BFAFF340
:10203000008062B6EEE70000040D00200000000002
:1020400000000000000000003800002010B520282B
:1020500011D20E4991F82C30A1F1800202EB831CC1
:102060001CF810303BB191F82C3002EB831212F8BF
:102070001020012A01D0002010BD91F82C2001462B
:102080000020FFF709F8012010BD0000040D00201A
:102090002DE9F84F864E804696F82C00A6F1800771
:1020A00007EB801010F81800002871D096F82C90DB
:1020B000804D25B1002140F67630AFF3008007EB6C
:1020C000891414F81800012818D0C0B204281CBFC5
:1020D0000528062861D02DB14FF0000140F682306E
:1020E000AFF3008001F098FC25B1002140F6863066
:1020F000AFF3008014F818000128E6D1012425B1BF
:10210000002140F68D30AFF30080002C4BD0002032
:1021100086F8290025B1002140F69230AFF3008007
:1021200096F82CB0012020EA0B0907EB8B1107EB86
:10213000891040220AF0DEFC25B1002140F22F5028
:10214000AFF3008009EB490000EB060A0BEB4B00F4
:102150003044018CAAF8201090F822008AF822005E
:1021600025B1002140F23350AFF3008096F82900EA
:102170008DF800009DF80000E0B1002D1CBF00218B
:1021800040F69830BBD000BFAFF30080B7E7FFE761
:1021900040F66D31702001F015FB4A4641460120A2
:1021A000FEF77AFFA0E74448002818BFAFF300808D
:1021B00062B6ACE725B1002140F69C30AFF3008059
:1021C0009AF821300AF1210140461C464FF0200BBD
:1021D00007EB89120AF1220A04E0A34602EB4B0C3A
:1021E0009CF80140844202D0202C2BD0F5E7202C13
:1021F00028D0A34204D102EB43004078087005E0E8
:1022000002EB440002EB4B0140784870BAF1000F3A
:1022100011D025B1002140F29240AFF300809AF82E
:102220000000A04207D125B1002140F29540AFF354
:1022300000808AF800B05DB1002140F29A40AFF30F
:10224000008000E025B100214FF43A60AFF3008038
:102250001A48002818BFAFF30080EFF3108472B65D
:1022600096F829008DF800009DF8000038B1002D87
:102270001CBF002140F6A6303FF441AF84E786F84A
:102280002C90FF2086F8290054B1002D08BFBDE82E
:10229000F88F002140F6B330AFF30080BDE8F88F2F
:1022A0000548002818BFAFF3008062B6EDE70000D4
:1022B000040D0020000000000000000000000000ED
:1022C00070B50D46064601F0F3F90F4890F82C2042
:1022D0000024803800EB821010F8141029B1611C22
:1022E000CCB2202CF8D3202070BD0848C4EBC40128
:1022F00040F8216000EB8100214645600120FEF797
:10230000CBFE204670BD0000040D00200409002013
:102310002DE9F84F00F03CFB054600F00BFE604C49
:102320006068B0F1FF3F1CBF4FF0FF306060A07FDE
:102330005C4F90B9D4E90210401A20F07F404FF46E
:102340000C710AF0A8FAE1680844281A0002C117C3
:1023500000EB11600012C00F12D0607E20B394F821
:1023600027008DF800009DF80000E8B100F03EFC69
:1023700094F82800F0B140F2D531702001F022FA33
:1023800094F82D0094F82D10C0EBC00007EB8000EE
:102390004068C1EBC10157F821200821904740F265
:1023A000BD31702001F00EFAE81C20F07F4000F0F3
:1023B00015FBDDE7012084F8280094F82D00202883
:1023C00021D094F82D90202084F82D0084F82E0040
:1023D000002684F8266084F82760266000F09EFEC0
:1023E000207794F82C8008EB480000EB040A9AF858
:1023F0002000202812D0C0EBC00007EB8000817EB7
:10240000012905D00AE04FF47671702001F0DAF965
:1024100000F1080201212846FEF7B6F942460121E3
:102420002846FEF76BFE0700F8D01F4800EB881027
:1024300010F81900022804D1424649460620FEF74A
:102440002BFEFF2084F829009AF82100DFF85C8039
:1024500020281CBF98F8010001F088FA207F18B1ED
:1024600000F038FE26776677022F0FD0012F18BFB5
:10247000BDE8F88F4FF0FF30D8F80410002908BFEE
:10248000BDE8F88F01B0BDE8F04F0847A068401BD9
:102490000AF0D4F9D8F804100029F3D1BDE8F88F78
:1024A000040D002004090020840C002038000020C6
:1024B00030B5364C054683B094F82D00202808D05E
:1024C0006068B0F1FF3F09D040F6A121702001F013
:1024D00079F94FF42A61702001F074F994F82D0015
:1024E0002B49C0EBC00001EB80000830FEF79AFDDD
:1024F0000146284A2844914204D940F26F51702085
:1025000001F060F924498D4204DD4FF4AE61702082
:1025100001F058F921498D4204DA40F271517020DE
:1025200001F050F91E498142DCBF00F5F700A0F12F
:10253000F85005DD0028BCBFA0F5F70000F1F85009
:1025400001AA694600F0BAF89DF804000F288CBF74
:10255000012000200099084420F07F41616094F838
:1025600027008DF800009DF80000002804BF03B08C
:1025700030BD052000F0B8FB00281CBF03B030BD03
:1025800040F6A821702001F01DF90000040D002084
:1025900004090020FF7F841E0040420F00C0BDF0F0
:1025A0000080841E70B51C4C202184F8201084F813
:1025B000211084F82210002084F82C0084F82D10BB
:1025C000421EC4E90002A07784F8260084F82700A0
:1025D0002077607784F82E1084F82A0084F82B0086
:1025E000A4F182011022887001F8040F521EFAD162
:1025F00000F09EFD094D012684F82860FF20287018
:10260000074801F095F9687001F0F0F9A86000F052
:1026100019FD84F82F6070BD040D002038000020E3
:102620004D0F000070B50546012000FA05F40E4676
:10263000002A08BF08480CD0002000F0E9FCE9009F
:1026400001F1804101F5F831C1F81005C1F81465B8
:102650000248046070BD000008F5014004F5014027
:1026600000B583B0684600F099F900980AF0E6F8E2
:10267000019A034B0021E2FB030103B000BD0000FF
:102680000080841E410B48F2376251430A0C094B0B
:10269000510202FB03020848504300F586306E30B9
:1026A000400D5B4210FB03F3B2EB532F88BF491C74
:1026B00008447047F7C2FFFF6F0C0100430B48F25C
:1026C000376C03FB0CF330B41B0CDFF844C05C0226
:1026D00003FB0C030F4858434FEA505C04EB0C001B
:1026E00043F609541CFB04F404F5807C43F60855BA
:1026F000A3EB5C2C2C440CF0FF0CB3EB542F84BFE9
:102700004FF0000C401C086082F800C030BC7047DD
:10271000F7C2FFFF6F0C01002DE9F0413B4DD5F8EA
:102720000403DFF8EC8010F4803F4FF400664FF0B4
:10273000E0274FF0000419D036480068B0B1C5F862
:102740004041C7F88062D5F84005D8F80010401A1B
:1027500020F07F40022802D3B0F5000F06D94FF4D5
:102760008030C5F808030420FEF7C2FED5F8040344
:1027700010F4003F1AD028480068B8B1C5F84441A9
:10278000C7F880622548D0F84005D8F80010401AF4
:1027900020F07F40022802D3B0F5000F06D94FF495
:1027A0000030C5F808030520FEF7A2FED5F80403A3
:1027B00010F4802F1AD01A480068B8B1C5F8484103
:1027C000C7F880621748D0F84005D8F80010401AC2
:1027D00020F07F40022802D3B0F5000F06D94FF455
:1027E0008020C5F808030620FEF782FED5F8040114
:1027F000002808BFBDE8F081C5F80441C7F8806231
:102800000948C168491CC160BDE8F08100B00040C2
:1028100004B5004040B1004044B1004004B0004065
:1028200048B1004008B00040440000202DE9F041CC
:10283000384D2878042868D0A81C0122017859B1A5
:10284000012908BF6A7002D06978002958D0022196
:102850000170407800F0FEFA2F4CD4F804034FF0DA
:10286000000810F4002F4FF480774FF0E0260AD0D4
:102870002A48006838B1032000F0ECFAC6F88072EC
:102880000320FEF735FED4F8040310F4802F0AD09D
:102890002348006838B1022000F0DCFAC6F88072E4
:1028A0000220FEF725FED4F8040310F4003F0AD0FE
:1028B0001C48006838B1012000F0CCFAC6F88072DC
:1028C0000120FEF715FED4F8040310F4803F08BF82
:1028D000BDE8F08114480068002808BFBDE8F08119
:1028E000002000F0B7FAC6F8807204202870C5F8FE
:1028F0000480C4F80082BDE8F0410020FEF7F8BD76
:1029000040F29F416C2000F05DFFBDE8F0410720E0
:10291000FEF7EEBD44000020008000404C810040E6
:102920004881004044810040408100400122110262
:102930004FF0E0230020C3F8801103F5C073BFF30C
:102940004F8FBFF36F8FC3F800110E4941F8042F6A
:10295000431EC1F80433C1F83C05C1F83C010A4BE1
:10296000C3F84005C1F840011B1DC3F84005C1F87C
:1029700044011B1DC3F84005C1F84801CA60034962
:1029800048707047008000400480004044000020F0
:10299000014800687047000004B5004030B4EFF310
:1029A000108C72B600250B4B0B4A00BFD3F80415F0
:1029B000D3F804412CB1D168491CD160C3F804514B
:1029C000F4E7D268BCF1000F00D162B6C0E9001292
:1029D00030BC704700B00040440000202DE9F047B3
:1029E000464E0546B71E3378B968012B04BFA9428D
:1029F000BDE8F0874FF04040414A1060424A4148EC
:102A0000C2F8080302F1040C4FF00004002B62D05E
:102A10003E48C2F84803CCF84045C2F8444100BFE4
:102A2000D2F848014FF0E0294FF00108002801BF1B
:102A3000D2F8040100284FF40060C9F880024FF476
:102A40008030C2F80803C2F84803C2F84041304859
:102A5000D0F800C0A5EB0C0C2CF07F4CBCF1020FA1
:102A600044D3BCF5000F41D8C2F840554FF4803C28
:102A7000C2F844C32BB102688A1A22F07F42022AAC
:102A8000F9D3C7F804803C70FFF750FF2148D0F815
:102A9000041564F30101C0F80415D0F808250221DB
:102AA00061F30102C0F808250421C0F81015C0F830
:102AB0000C807968C0F800128015C9F88002C9F846
:102AC00000011549C00508600420BD60707086F8DB
:102AD0000080BDE8F087C2F84803C2F84045C2F85C
:102AE0004041CCF84045C2F8444199E70020C2F883
:102AF000400540F293216C2000F064FE4600002067
:102B000008F50140FDFFFBFF00B00040FDFFFAFFAC
:102B100004B500400080004004F5014070B52A4C27
:102B2000A168814214BF01220022DFF8A0C09CF8F6
:102B30000050022D02D0002A34D002E0002A08BF43
:102B400070BD62789AB3224B4FF080421A60214BDD
:102B50009213C3F80823C3F848230022C3F8402186
:102B60001D4A1668861B26F07F46022E24D3B6F532
:102B7000000F21D8C3F840054FF48036C3F84463F2
:102B80002DB11368CB1A23F07F43022BF9D3134BDB
:102B900002214A071A60A06004208CF801008CF81A
:102BA000001070BD40F2A1216C2000F00BFE40F23D
:102BB000A5216C2000F006FE0020C3F8400540F27D
:102BC000B1216C2000F0FEFD4400002046000020F2
:102BD00008F5014000B0004004B5004004F5014094
:102BE0000148806870470000440000202DE9F04152
:102BF0003648354AC0F80823DFF8D4C0031D002149
:102C00009CF8004084B1334AC0F84823C3F840150B
:102C1000C0F84411D0F848210123002A04BFD0F89D
:102C20000401002811D10AE0C0F84823C0F840157B
:102C3000C0F84011C3F84015C0F84411EAE74FF05E
:102C4000E0224FF40060C2F88002022C04D040F26F
:102C5000BD216C2000F0B6FD1F4E30681F4CC01C1B
:102C600020F07F40A2681E4D90420BD03768D71BE2
:102C700027F07F47042F05D3B7F5000F02D8FFF7E1
:102C8000ADFE1BE03068101A20F07F40022813D3FD
:102C9000B0F5000F10D8134A4FF080401060636009
:102CA00021706B60EB604000111F086004208CF8FD
:102CB00001008CF8003001E0636021706068C5F8A5
:102CC0000002BDE8F0810000FDFFFBFF00B0004006
:102CD00046000020FDFFFAFF04B50040440000203C
:102CE0000080004008F501402DE9F041544A0025DC
:102CF000012492F800C053784FF4A07607287DD2C3
:102D0000DFE800F004040404585858004D4A97685E
:102D1000B7F1807F04BF5278002A03D0BCF1020FC4
:102D200005D026E040F24D316C2000F04BFD1A1F1B
:102D3000D2B206EB820202F1804606F5304600224E
:102D4000BCF1010F03D0BCF1020F08D00EE0042B40
:102D500024BF3768002F08BF4FF0004206E0042B65
:102D600024BF3768002F08BF42F0804212F0804F26
:102D7000E5D1DFF8D4C000F1100204FA02F2CCF879
:102D800008234FF0400303EB8003DBB263441C6075
:102D90000CEB8000D0F84035A1EB030323F07F4318
:102DA000032B26BFC0F84015CCF80423C0F84055CB
:102DB00037D23CE0BCF1000F06D0834204D140F290
:102DC0006D316C2000F0FEFC021FD3B2032B04D344
:102DD0004FF4E4716C2000F0F5FCDFF870C003F1F3
:102DE000100204FA02F2CCF80823CCF8482306EBD0
:102DF00083034CF80350164B1B6800E01AE0001FD9
:102E0000CB1A23F07F43C0B20CEB8000022B0BD314
:102E1000B3F5000F08D8C0F84015CCF80423CCF85F
:102E200044230120BDE8F0810021C0F840150020B6
:102E3000BDE8F08140F271316C2000F0C3FC00006D
:102E400046000020440000200080004000B0004008
:102E500004B500402DE9F843012600274FF4A0787F
:102E6000072851D2DFE800F00404040419191900FE
:102E700000F1100106FA01F22649C1F8082301EB1E
:102E800080030022C3F8402508EB80028F502249BE
:102E900051F820000090BDE8F883204D011FCCB20E
:102EA000297879B16A7882420CD11D4A4FF04040AE
:102EB0001060012908BFFFF739FD2F7019494FF045
:102EC00080708860184904F1100006FA00F0C1F81B
:102ED0000803C1F84803A0000844D0F84005134A8D
:102EE0001268801A20F07F40022807D301EB840289
:102EF0000020C2F8400508EB84000F500C4850F841
:102F000024000090BDE8F88340F2F5316C2000F019
:102F100059FC000000800040408100404600002035
:102F200008F501404400002000B0004004B5004016
:102F300040B100402548244AC0F808232449031D15
:102F400091F800C00021BCF1000F10D0214AC0F858
:102F50004823C3F84015C0F8441100BFD0F84821F9
:102F6000002A04BFD0F80401002811D10AE0C0F8FB
:102F70004823C0F84015C0F84011C3F84015C0F808
:102F80004411EBE74FF0E0224FF40060C2F88002FA
:102F900011484FF0FF32C0F80823C0F84015C0F8C0
:102FA000401100F10402C2F84015C0F8441102F1CA
:102FB0000402C2F84015C0F8481102F10402C2F838
:102FC0004015C0F84C117047FDFFFBFF00B00040FA
:102FD00046000020FDFFFAFF0080004010B50728E2
:102FE0000DD2DFE800F004040404060606000649DA
:102FF00002E0001F0549C0B201EB800010BD40F2A5
:1030000095316C2000F0DEFB4081004040B1004073
:1030100010B507280DD2DFE800F00404040406060A
:103020000600064902E0001F0549C0B201EB80001E
:1030300010BD40F295316C2000F0C4FB408100408F
:1030400040B1004070B51F48002404210470801E68
:1030500001708905C4608160FFF768FC01254FF0AD
:10306000E02CEB02CCF88031BFF34F8FBFF36F8FB2
:10307000CCF8803214484560856014490A68002AFB
:10308000FCD1511EC0F80813C0F84813C0F84045E1
:10309000C0F840410E49C1F84045C0F84441091DFF
:1030A000C1F84045C0F84841C0F80441CCF80031AF
:1030B00005604FF48271C0F844130221C0F8041374
:1030C00070BD00004600002000B0004004B5004084
:1030D00004B00040084890F900000028B8BF7047CD
:1030E00000F01F01012202FA01F14009800000F105
:1030F000E020C0F80012704700020020034800786A
:1031000003280CBF0120002070470000F0010020C0
:103110000148408870470000F00100200348007813
:10312000022816BF0328012000207047F00100206C
:10313000024800210170418070470000F00100202A
:103140002DE9F041164C607A002827D04FF48071A9
:103150008D05284609F0C3FB80464FF4827128464E
:1031600009F0BDFB00260746B8F1000F09D0012089
:10317000C5F80803207920B12671E06908B18047BD
:10318000E66137B1C5F804610220C5F8080300F014
:103190004DFA4046BDE8F04100F058B8BDE8F08176
:1031A0005400002010B509F044FC30B909F062FC6D
:1031B00018B909F095FC002802D0024902200860E5
:1031C00010BD0000340C004070B500F091F900F023
:1031D00081FA094C4FF0804530B1FFF7E3FF012041
:1031E00028610420A07204E00320A0720120C5F829
:1031F00004030020E07170BD5400002070B5124C33
:10320000A079E0B1E179401E814218DA00F062FA5B
:10321000054600F04BFBA179012902D9E179491C4F
:10322000E1710DB1616900E02169411A022902DAF8
:1032300011F1020F07DC0DB1606100E02061BDE813
:103240007040FFF7C1BF70BD540000202DE9F0476A
:1032500006464FF080454FF48671284609F03FFB43
:1032600080464FF48871284609F039FB274C824686
:10327000277804F1080009F0A6FB10B140F2B9115B
:1032800016E04FF0010946B1A07A032805D10420C9
:10329000A072FFF787FFC5F810900026B8F1000F65
:1032A00018D0C5F80C61A07A042804D040F2CB11E4
:1032B0006D2000F087FA09F0BCFB28B909F0DAFBB1
:1032C00010B909F00DFC08B1114806600220A07287
:1032D00000F0F2F8BAF1000F08D0C5F81061A07A3A
:1032E000022801D1FFF78AFFC5F814903FB126707C
:1032F000A07A022801D1FFF767FF00F0DDF8BDE8F2
:10330000F0470248083009F075BB00005400002067
:10331000340C00402DE9F0475F4C00270646A761BA
:10332000427881780078E0726271A171E7714FF0A4
:1033300001084FF08045052825D2DFE800F0100392
:1033400006202200C4F8188009E000F0D1F801211D
:10335000284609F0C9FA0028F9D00220A06109F036
:10336000EFFAB0B100F0D0F9217E01F003018842FC
:103370000FD1B07950B10220C5F8040370E047487E
:10338000ECE74748EAE740F23A314DE000F090F9C7
:1033900066E0C5F80C804FF4827AC5F80471A06924
:1033A000C5F8180509F031FB40B909F038FB28B918
:1033B00009F04CFB10B909F05DFB38B14FF08050BB
:1033C000D0F844023749C0F34230086009F01DFBD1
:1033D00040B909F024FB28B909F038FB10B909F00D
:1033E00049FB18B12F491031C1F80080C5F8088099
:1033F0000220C5F80403B07990BBD5F8040310F09F
:10340000020F0FD0DFF8A090D9F80010C94341F3A4
:10341000001101F10108D9F8001041F01001C9F8BC
:10342000001007E040F2FB216D2000F0CBF900BF57
:1034300000F0F2FA5146284609F051FA0028F7D078
:1034400000F036F9B8F1000F05D1D9F8001021F0DD
:103450001001C9F800100220C5F80803C5F804716E
:10346000A07970B1307860B900F034F9064600F008
:103470001DFA6FF0004116B1C4E9041001E0C4E97F
:1034800004010121284609F02FFA08B100F01CF9C7
:10349000A772BDE8F0870000540000200100020080
:1034A000010003003C05004010ED00E00148C08928
:1034B000704700005400002010B5EFF3108472B67E
:1034C0000A48417829B14178491E4170417829B1B3
:1034D00008E04FF48E716D2000F074F9807808B91F
:1034E00000F006F9002C00D162B610BD5400002097
:1034F00010B5EFF3108472B606484178491C41704C
:103500004078012801D109F006FA002C00D162B6FA
:1035100010BD000054000020054810B5C17821B14D
:1035200000210171C170FFF7C7FF002010BD00002E
:103530005400002070B50C4CE17861B90125E570AC
:10354000E061FFF7D5FF00F0C5F830B1E06910B1D8
:1035500080470020E061002070BD4FF08040257161
:10356000C0F80453F7E70000540000202DE9F041B3
:1035700005006FF015003FD0297804293CD80029B8
:1035800069783BD0002937D1A978002934D10020AF
:1035900009F070F9002009F060F94FF080484FF011
:1035A000FF31C8F808130026C8F80061C8F80461A4
:1035B000C8F80C61C8F81061144C6670A888A08126
:1035C00009F0A0F9012708B1E770677001214046B2
:1035D00009F08AF908B100F077F840F2F550E0817F
:1035E0002846FFF797FE6772002009F036F94FF082
:1035F000E0213046C1F80071BDE8F0810029FBD020
:103600002029F9D8A9782129C1D9F5E7540000204B
:103610000148808970470000540000200248807AE9
:10362000002800D00120704754000020F8B51F4D3D
:10363000E87A00280FD1287E00F0030009F070F925
:10364000002808D0EFF3108172B6FFF7E7FF18B13A
:10365000002900D162B6F8BD0126AE7201B962B68A
:1036600018204FF08044C4F80803A6614FF420707E
:10367000ADF80000BDF80000411EADF80010F9D211
:103680000027C4F80C71C4F810710848083009F01C
:10369000ADF92F70FFF798FD6661687900F07F0043
:1036A000C4F838051820C4F80403F8BD54000020FD
:1036B00010B5044C207E00F0030009F031F9002819
:1036C000F8D010BD54000020014901200870704757
:1036D000010200204FF08040D0F8000118B90348E3
:1036E0000078002800D0012070470000010200206F
:1036F0004FF08040012141600021C0F800110148D5
:1037000001707047010200200248006800F00300C9
:10371000704700001C04004010B531B1012907D0EA
:1037200040F2023105A000F021F8D0F8140401E0C5
:10373000D0F8080400F0010010BD00006E72665F52
:10374000636C6F636B2E6800BFF34F8F0548016891
:10375000054A01F4E06111430160BFF34F8F00BFE0
:10376000FDE700000CED00E00400FA0572B6034A24
:10377000526802B19047FFF7E7FF00007400002095
:10378000064810B50021016001210160084609F0DA
:10379000EEF8BDE81040012009F0DCB8FC1F004045
:1037A000074810B501214160891EC0F808130C209C
:1037B00009F0DDF8BDE810400C2009F0CBB800009E
:1037C00000C000400EB572B60F4A5568D5B1002250
:1037D00003466E460A2403E0B0FBF4F0521CD2B25A
:1037E0000028F9D1B05409E0B3FBF4F004FB103029
:1037F000B3FBF4F3521ED2B23030B054002AF3D1EE
:103800003046A847FFF7A0FF740000202DE9F041E3
:10381000184C0646174660780D4618B14FF0FF3039
:10382000BDE8F081FCF78CFC06B9134E676025708B
:10383000FFF7A6FFFFF7B4FF3046FFF797FE06003D
:10384000EED1FEF7AFFEFFF7F1FE08F0D1FF2846FC
:1038500009F080F80120002D09DB05F01F0100FAB6
:1038600001F16A09920002F1E022C2F800116070D1
:103870003046D5E77400002090C900000148407828
:103880007047000074000020074890F900000028ED
:1038900009DB00F01F02012191404009800000F186
:1038A000E020C0F800127047740000202DE9F041BC
:1038B00001264FF0E02231034FF000084046C2F8E5
:1038C0008011BFF34F8FBFF36F8F164CC4F8000108
:1038D0000C2009F06BF8144D2868C04340F3001722
:1038E000286840F010002860C4F8046326607F1C3C
:1038F00002E000BF00F090F8D4F800010028F9D0F1
:103900001FB9286820F01000286008480568666024
:10391000C4F80863C4F800810C2009F047F8284671
:10392000BDE8F08100C0004010ED00E008C5004097
:1039300010B5024605200C4904E000BF01EBC003AE
:103940001B7933B1401EC0B2F8D248216920FFF77D
:1039500039FF41F8302001EBC00100224A718A7121
:1039600001220A7110BD0000340D002010B5052899
:1039700001D3582106E00A4901EBC0000179012971
:1039800003D059216920FFF71DFF41798279491C35
:10399000C9B28A4200D04171BDE81040FFF774BF40
:1039A000340D002070B505250E4E0F4C16E0217821
:1039B00006EBC1000279012A08D1427983799A4243
:1039C00004D04279827156F8310080472078401C3B
:1039D000C0B22070052801D3002020706D1EEDB20A
:1039E000E5D270BD340D00200202002000B509F0C0
:1039F0000CF840B909F013F828B909F027F810B904
:103A000009F038F808B1024800BD024800BD0000C6
:103A10000C05004000E7014010B509F02BF830B369
:103A2000EFF31080C8B1002172B612480268036833
:103A3000C2F3001243F0100303604FF0E023D3F809
:103A40000042D3F804321C4300D040BF20BF00BF67
:103A500000BF00BF00BF12B105E00121E4E702682A
:103A600022F010020260002900D062B610BD20BF13
:103A700010BD000010ED00E00149096889680847A1
:103A80007C00002001490968096908477C00002082
:103A900001480068406800477C000020014909682F
:103AA000096808477C000020BDCC0000B5CC0000B0
:103AB000A9CC0000B9CC0000B1CC000070B50E4C10
:103AC0006078002817D120780025012806D102202F
:103AD0002070206910B12069804725612078032873
:103AE00009D125702069002805D0606840698047A9
:103AF00020698047256170BD8000002010B5084C0A
:103B00002078022802D02078032802D160688068DB
:103B100080470020A0706070BDE81040FFF7CEBF66
:103B20008000002002480078002800D00120704763
:103B30008000002038B50446052804D340F23D112A
:103B40006820FFF73FFEFFF7B9FF104D01206870B6
:103B50002878022816D16868C168204688470C4931
:103B600001EB4402527882420DD3A87801280AD092
:103B700011F814008DF800008DF8014068680168A4
:103B80006846884738BD0120F4E700008000002027
:103B90009810002005490A78022A04D00A78032ADE
:103BA00001D000207047496809690847800000205B
:103BB00010B558B108490A78022A02D00A78032AB7
:103BC00009D149684968BDE81040084740F25311DF
:103BD0006820FFF7F7FD10BD80000020014901209B
:103BE000887070478000002005480178022904D0C1
:103BF0000178032901D000207047406880690047A0
:103C000080000020E1CC000019CD000003CD0000B1
:103C1000F1CC0000FDCC0000EBCC0000DFCC0000BC
:103C2000DDCC000015CD000009CD0000F7CC000070
:103C3000E5CC0000D7CC0000CFCC0000D3CC0000F6
:103C4000C9CC0000014800680068004794000020CB
:103C5000014800684069004794000020014A12684A
:103C6000D26810479400002001490968C96A0847D2
:103C7000940000200148006800690047940000207B
:103C8000014A1268926810479400002001490968AF
:103C9000496A08479400002001490968896A084771
:103CA00094000020014B1B685B68184794000020BB
:103CB0000148007870470000030200201FB5144C33
:103CC000207A8DF80100E0798DF80000A079ADF838
:103CD00004006079ADF80200684606F0A1FA08B168
:103CE000832110E0E068029002A806F0AFFA08B164
:103CF000872108E007480068039003A80BF02CFD1B
:103D0000002803D08B21032000F058F91FBD0000CC
:103D10005C0D0020684000007CB5044600680D463C
:103D200000F1030020F0030020604FF0000000903D
:103D3000019008788DF8010048788DF802008878A5
:103D40008DF80300C8788DF80400287916008DF8E6
:103D5000050001D0002000E02068694600F012FB59
:103D6000216808442060A97841B16B8AEA7806B1DD
:103D7000002000F0D9FD2168084420601948C1786E
:103D800079B1297C69B1007908B1FF2200E02522D0
:103D90000EB1002000E0206800F05CFE21680844BD
:103DA0002060287968B12068C01C20F003002060E2
:103DB0002A7D297906B1002006F0B4FD2168084467
:103DC0002060687D00280CD02068C01C20F0030013
:103DD0002060697D06B1002000F06CFE2168084477
:103DE00020607CBD9800002010B528B11422044941
:103DF00008F080FE002010BD6FF0150010BD00001F
:103E00008440000070B510B16FF02C0070BD304CD4
:103E1000607810B14FF0FF3070BD21B36FF0150026
:103E2000002AF9D02B4B0C29F6D2DFE801F0060767
:103E30000A0D1D202C3426373A3FEDE71078187014
:103E400038E01078587035E091780029E4D0D178C6
:103E50000029E1D011781B29DED351781B29DBD34F
:103E60001068C3F8050025E01068D86022E01178DA
:103E7000DA789142D0D399701CE011789A78914207
:103E8000CAD8D97016E0E17811B111780229C3D3EC
:103E9000107818740EE0108858820BE010781871B2
:103EA00008E011780229B7D3197503E011780829C1
:103EB000B2D8597501220749002008F047FFB0F534
:103EC000803F02DB6FF00B0070BD0121A17070BD5F
:103ED000980000205C0D002070B50C46050019D03C
:103EE000C4B100F003F9C0B12846FFF721FD0C4D25
:103EF00000220C492870204608F028FF0CF0EEF94B
:103F00000021287806F05EFCFFF7D8FE01206870DB
:103F1000002070BD6FF0150070BD4FF0FF3070BD18
:103F2000980000205C0D002030B587B005000CD053
:103F3000FFF7A4FC4FF0FF3420B1FFF769FBB0F5A9
:103F4000FA7F05D9204607B030BD6FF01500FAE7BB
:103F5000154C1648A56000F0F1F900206070A070C3
:103F6000E070207101461822684608F03DFE1822D4
:103F70000F49684608F0BEFD182269460D4808F052
:103F8000B9FDEFF3108472B66FF00C0000F0D4FDB1
:103F9000094800F09FFE18B19E21032000F00EF8A2
:103FA00004B962B60020CEE798000020BD3C0000B6
:103FB0006C4000005C0D0020194100000EB572B687
:103FC000154A9568DDB1002203466E460A2403E0D7
:103FD000B0FBF4F0521CD2B20028F9D1B0540AE080
:103FE000D8B2B0FBF4F7B3FBF4F304FB1700521E96
:103FF000D2B23030B054002AF2D13046A847BFF3D5
:104000004F8F06480168064A01F4E06111430160E0
:10401000BFF34F8F00BFFDE7980000200CED00E0DC
:104020000400FA05064810B581784078014302D0B3
:104030004FF0FF3010BD06F0F1FB002010BD000076
:1040400098000020074810B581784278114302D0CB
:104050004FF0FF3010BD0121C17006F0F1FB0020D0
:1040600010BD0000980000200100000001010100C7
:10407000001B1B03020000004C1D000003001F007A
:1040800002000000295C92F1368192D1B7A9F0F1CB
:1040900099E94C191F23834A054A10B5526812B199
:1040A000BDE81040104792210420FFF787FF000071
:1040B000740D0020054A10B5126812B1BDE8104019
:1040C00010478C210420FFF779FF0000740D0020B9
:1040D000054A10B5926812B1BDE81040104798210A
:1040E0000420FFF76BFF0000740D002005480168F5
:1040F00029B1416819B1806808B1012070470020DA
:1041000070470000740D002002490DC881E80D00C1
:1041100000207047740D0020F8B5124C0026256869
:1041200011E00098022802D003280CD106E0206894
:1041300010B10020266005E028210CE0206868B15D
:1041400001202660A847684600F096FD0028E8D0C8
:10415000052805D035210420FFF730FF2D21FAE78F
:10416000F8BD0000A40000207CB51F4C0546207857
:1041700040B1A278611C2846921C08F0BBFC0020CC
:10418000207021E0194801F0F5FA00281DD0174CE5
:104190002078142804D10A213E2000F029F818B113
:1041A00020780A2805D009E01049284609F0B8F817
:1041B0000AE005213E2000F01BF838B10B492846E3
:1041C00008F006FE002800D001207CBDA088ADF8D4
:1041D000000001A9684609F0D9F90028F5D09C2112
:1041E0000820FFF7EBFE0000880E0020800D002065
:1041F00070B50C46054600F04BF8002802D03E2D65
:1042000001D0012070BD122C06D106480178022988
:1042100002D040780028F5D02046BDE8704000F07C
:1042200049B80000040200200149487070470000AE
:104230000402002070B50A7882703AB3012A25D8AA
:104240001323037000230AE001EB430400EB430552
:10425000A678EE706488240A5B1C2C71DBB2934252
:10426000F2D300230BE000BF01EB430500EB430456
:104270002E796671AD882D0A5B1CA571DBB2934265
:10428000F2D3012101EB8200C0B270BD002070BDED
:10429000402803D2401EC1B2054805E0FF2805D0E2
:1042A0004038C1B20248083009F064B801207047B4
:1042B000A8000020401EC1B2014809F05BB8000010
:1042C000B8000020024902680A61406848617047EE
:1042D000A8000020054902680A60406842F48C2268
:1042E0000A60034A1043486070470000A80000209D
:1042F000F807400207484FF0FF3100220160C90C67
:10430000416000F108011F200A604A600831C1E9DC
:1043100000027047A800002010B5FFF7EBFF002057
:10432000FFF782FF0BF082FB04460348006800B1F0
:104330008047204610BD0000C000002001490860F1
:1043400070470000C0000020022101804180002150
:1043500001712921417149F25C21C18001498160CB
:1043600000207047F136819210B5052804D34FF430
:10437000D6711720FFF722FE0149085C10BD00002E
:104380008C0F0020F8B504468A7848780244FF2A4A
:1043900002D940F25F111DE00A78824202D940F250
:1043A000631117E00094C4B100264B7891F802C065
:1043B0004A790CEB0300C5B2AA4200D91546C87869
:1043C000A84200D90546E71C27F00307A74206D0FC
:1043D00040F279111720FFF7F1FD0126E5E7154FAF
:1043E0003B7087F801C0B8700879F8703A713146AF
:1043F000684600F00FF900218C460098C01C20F0A0
:10440000030000905EB907EB8103D861002004E04F
:10441000DA6942F820C0401CC0B2A842F8D3009824
:10442000491C00EB8500C9B200900529E5D3001BAB
:10443000F8BD00008C0F002070B5044609F0D0FCD8
:1044400008B1102070BD257800F020F902460C4814
:10445000618800EB85000EE0C36953F8213043B159
:104460004A1C6280A180C06950F82100A060002031
:1044700070BD491C89B29142EED36180052070BDA8
:104480008C0F00202DE9F041074611B1002038B90A
:1044900001E00120FBE7012902D0002038B901E04A
:1044A0000120FBE7022902D0002038B901E00120F9
:1044B000FBE7032902D0002060B901E00120FBE7FF
:1044C000042907D0002000281FD000241248012909
:1044D00002D002E00120F6E7047800234FF6FF76D1
:1044E00000EB810C10F801E008E01819DCF81C5012
:1044F00080B255F8205025B15B1C9BB29E45F4D884
:1045000030463880B04202D10020BDE8F081BDE8DD
:10451000F04100F035B800008C0F00202DE9F0418B
:104520000746A0F57F400C4643F20206FF3820D034
:10453000052C02D30720BDE8F081384600F05AF878
:10454000050016D00C48294650F8242038469047DC
:104550000A48002100EB8406F06940F82710204645
:1045600000F08AF802462946B06809F03BFA0020BC
:10457000E1E73046DFE70000C84600008C0F00206E
:104580002DE9F04190460E46074609F077FA48B10A
:10459000164800EB8604E06950F8270028B14FF474
:1045A0009D7115E040F2391112E0A06800281AD080
:1045B000304600F061F80146A06809F0BBF905003B
:1045C00010D0E069052E40F8275004D340F2451181
:1045D0001720FFF7F3FC06484246294650F82630DC
:1045E000384698472846BDE8F08100008C0F00202F
:1045F000B446000070B50C46054609F03FFA0028A5
:1046000005D0034800EB8400C06950F8250070BD58
:104610008C0F00202DE9F843164F884605460024EC
:104620002868C01C20F003002860204600F024F811
:10463000395D4143B8F1000F01D0002000E0286847
:10464000009018B100261EB1002002E00126FAE712
:10465000684609F0A0F91EB907EB8401009A8A6048
:104660002968641C0844E4B22860052CD8D3BDE84E
:10467000F88300008C0F0020034931F810004FF63A
:10468000FC71C01C08407047DC460000084B1878DD
:1046900059780844C1B29878814200D30846DA7844
:1046A000904200D210461979884200D208467047DD
:1046B0008C0F002091DA000091DA000091DA0000FE
:1046C00091DA000091DA000065F20000A1EE00002E
:1046D000E9E50000C7020100CD020100E80248033D
:1046E00058018000900000002DE9FF4F274C07463D
:1046F00081B020689A46934658B1017AB94203D9ED
:10470000406850F8270040B143F2020005B0BDE810
:10471000F08FA5211820FFF751FC1946029809F0E7
:10472000D1F9804658460E9909F0C2F9064608EBC1
:104730000600001D85B22068A1462946006809F0E0
:10474000F9F804001FD0658026800E98251D009082
:1047500031465A460123284609F049F82088414647
:1047600028440A23029ACDF800A009F040F82088D6
:104770004119284609F06EF8D9F80000406840F861
:1047800027400020C2E70420C0E70000C40000204A
:1047900070B5144C23688BB1197A814212D95A68CA
:1047A00052F8201071B1002542F820504A8818684C
:1047B00009F018F9216800200A7A0CE0C8211820B5
:1047C000FFF7FCFB43F2020070BD4B6853F820304A
:1047D00033B9401CC0B28242F7D8086809F0F7F834
:1047E000002070BDC40000202DE9F0410D460400FA
:1047F00090464FF0000609D00027E01C20F003008F
:10480000A04205D086211820FFF7D8FB0127F4E746
:10481000CDB11146002009F0BEF80C3000EB850642
:104820008FB90A4F04F10C00AA003C602572606049
:1048300000EB850020600021606808F0D5F9414652
:10484000386809F0A8F83046BDE8F081C4000020BF
:10485000094910B502460968002049B10B7A934214
:1048600005D9496851F82210002900D0081D10BD53
:10487000EE211820FFF7A2FBC40000200A4910B562
:1048800002460968002059B10B7A934207D949685A
:1048900051F82210002902D031F8040B084410BD51
:1048A000FC211820FFF78AFBC40000202DE9F0410D
:1048B0001C4E456804460022A1B10120607070883A
:1048C0008308002004EB400104EB80060A830B847C
:1048D00000FB035171602118401C0A750428F1D3B4
:1048E000BDE8F0816270002004EB40010A830A8475
:1048F00004EB80014A602118401C0A750428F3D398
:10490000708809F05EF90746708809F061F9656002
:1049100020842918A1606784E560A0842161E78470
:10492000DEE70000C80000202DE9F04780B1002636
:104930001144CFB2DFF89C80C11C002421F0030198
:1049400088F80070814205D04E210920FFF736FB20
:104950000126EDE71F2B04D84FF6FF7101EA83050E
:1049600009E05900FF2B0CD903F1FF02B2EB430F12
:1049700000D211468DB24FF6FC71ED1C0D4036B1E0
:1049800009E07C22B2EB430FF4D37C21F2E7C8F8B4
:104990000400A8F8025007EB870104EBC1020021D4
:1049A0004FF001090FE05EB9D8F8044001EB810334
:1049B00000EB020C04F8339004EBC303C3F804C00B
:1049C000491C2A44C9B2B942EDD3D21D22F00700D6
:1049D000BDE8F087C800002070B5114800242146CA
:1049E00002780CE0456801EB810315F8333023B100
:1049F00001EB810105EBC10403E0491CC9B29142FE
:104A0000F0D344B10025A57001212046FFF74EFFE9
:104A10002570204670BDA9210920FFF7CFFA0000BC
:104A2000C8000020044810B54088840809F0D0F878
:104A3000844200D3204610BDC800002001484078C1
:104A400070470000D0000020014840687047000017
:104A5000D00000202DE9F8430C46074616462E21CB
:104A600010460D46224608F024FF804657B13846CE
:104A7000414632462B46009408F0B9FE0348476091
:104A8000047046704046BDE8F8830000D000002066
:104A90000248427801784068FFF7DCBFD000002070
:104AA000034B00211878C0EBC002586808F09CB88E
:104AB000D800002010B50C4610B1002212B10FE052
:104AC0000122FBE7C11C21F00301814203D0202118
:104AD0004120FFF773FA044948600C70FFF7E0FFCC
:104AE000C4EBC40010BD0000D800002030B50D4953
:104AF00001204860821EC1F808230B49886000230A
:104B0000C1F80032C1F80823084C2360251D286035
:104B10008860C1F8082323602860064904480860BB
:104B200030BD000000E0004000F0004000F5004013
:104B30000000F63F08F5014010B50446FFF7D6FF28
:104B400009F01BF900F088F8054904480860204680
:104B500000F0B8F8BDE8104000F0D0B80000F63F13
:104B600008F501402DE9F84F8246384807F02BFF41
:104B7000DFF8D8B028B101260BF10100FF21017048
:104B800000E000264FF48075314C4FF000082F1DD7
:104B900001216160C4F80081C4F80481C4F804A54F
:104BA0002160DFF8B0901CE0D9F80000C00618D5ED
:104BB0000E2009F0F1F8EFF31080009072B6032197
:104BC0002046C4F80413294609F0F3F830B93946F1
:104BD000204609F0EEF808B9FEF71EFF009800B96C
:104BE00062B62946204609F0E4F828B9394620463D
:104BF00009F0DFF80028D7D03946204609F0D9F867
:104C00000028C5D106BB9BF801108DF80010009953
:104C100000919DF8001009B1012500E000250BF17D
:104C2000010080F800800320C4F80803C4F8048160
:104C3000C4F800810E2009F0AFF8044807F0DAFE4E
:104C400015B11120BDE8F88F0020FBE70602002017
:104C500000E0004010ED00E010B5064807F0C6FE89
:104C600018B127211D20FFF7A9F902480021417042
:104C700010BD00000602002070B511490A68EAB1B3
:104C800000231D4601244A68521C4A600C2A00D3A6
:104C90004D600E7904FA06F20E6816420BD0EFF35F
:104CA000108372B60C6894430C6003B962B649680D
:104CB0000160002070BD5B1C0C2BE4D3052070BD8F
:104CC000E0000020024800210160416070470000C0
:104CD000E000002010B5084C617809B10F2010BD2C
:104CE000FEF726FE2070FF2801D0002010BD78219D
:104CF0001F20FFF763F90000000000200149002099
:104D0000487070470000002005498A8D824218BF14
:104D10007047002081F82A004FF6FF7088857047A1
:104D2000601000200A4A10B1012807D00EE0507828
:104D300060B1D2F802000860D08804E0107828B191
:104D40009068086090898880012070470020704733
:104D500008020020094A012340B1012818BF70470A
:104D60001370086890608888908170475370086855
:104D7000C2F802008888D080704700000802002036
:104D8000064910B1012803D006E0487810B903E0C5
:104D9000087808B101207047002070470802002001
:104DA0000149087770470000820700200246074843
:104DB00010B5007838B10648817821B1C01C05F0E3
:104DC000F3FD012010BD002010BD0000F401002003
:104DD000A210002000487047751200202DE9F04114
:104DE000124C00263546A07800288CBF104FBDE835
:104DF000F081601990F83B2190F80311012A02D04C
:104E000090F84B0158B104EBC100BD5590F8532107
:104E100000F5AA713046731CDEB207F08DF8681CED
:104E2000C5B2A078A842E4D8BDE8F081A210002065
:104E3000F801002004498A78824286BF084490F82D
:104E40004301002070470000A210002004498A7826
:104E5000824286BF01EB00108330002070470000C3
:104E6000A2100020054A01EB410102EB410102685A
:104E7000C1F80B218088A1F80F017047A210002013
:104E80002DE9F041134C06460025A078002898BF74
:104E9000BDE8F081C0B2A84214D904EB05108330FC
:104EA00010D0611991F8431161B905EB450104EB8C
:104EB000410707F20B11324608F0CFFFB7F80F0198
:104EC000A7F80F01681CC5B2A078A842E2D8BDE8D7
:104ED000F0810000A210002004498A78824286BF37
:104EE00001EB0010C01C002070470000A210002041
:104EF00008498A78824203D90A1892F843210AB1F4
:104F00000020704700EB400001EB400000F20B1066
:104F100070470000A210002010B540F2D31200210B
:104F2000074807F061FE0822FF21064807F05CFEF3
:104F300005480021017041704FF46171418010BD3E
:104F4000A2100020F8010020F401002070B50C46EA
:104F5000054605F04FFE05F03FFD0A482A46007859
:104F600068B1094B997851B1002C0CBF03F1830053
:104F7000D81C05F019FD05F059FD012070BD002079
:104F800070BD0000F4010020A21000200B4B93F82C
:104F900002C084459CBF00207047184490F803016C
:104FA00003EBC00090F853310B70D0F8541111602E
:104FB000B0F858019080012070470000A210002036
:104FC00007498A7882429CBF00207047084490F8C5
:104FD000030101EBC00090F85A0100F00100704796
:104FE000A210002010B500F077F9102814D00B4A59
:104FF0000146002092F802C0BCF1000F0CD9131832
:1050000093F803318B4203D1102818BF10BD03E081
:10501000401CC0B28445F2D8082010BDA210002068
:105020000246064810B500EB01100121833005F05F
:10503000BBFCBDE8104005F0F9BC0000A210002048
:105040000148408870470000F40100202DE9F0413C
:105050001746012500221E462C463A7000F03CF906
:10506000102827D0184901EBC00292F85A2102F00B
:1050700001023A708B780022002B1BD901EB020C45
:105080009CF803C1844519D1102A13D0002E18BFF3
:105090003270887890420DD901EB021010F1030FA5
:1050A00008D0881890F84B4190F83B0101280CBFBC
:1050B0000125002545EA0400BDE8F081521CD2B26A
:1050C0009342DBD8F6E70000A210002006498A7858
:1050D000824206D9084490F83B01002804BF012011
:1050E0007047002070470000A210002070B50D46E8
:1050F000044600F0F1F81A4A102814D002EBC0015F
:1051000091F85A0110F0010F1CBF012070BD5078BA
:1051100008283CBF012081F85A011ED25078401C5B
:105120005070012070BD5078082816D213780120E5
:10513000591C1170102B03D346212820FEF73EFF87
:1051400002EBC3032968C3F85411A988A3F85811C6
:1051500083F8534183F85A01E0E7002070BD000056
:10516000A21000200148407870470000F4010020A0
:105170000149487070470000F401002070B42B48CA
:1051800000250178491E4BB2002B46DB00EBC30122
:1051900091F85A1111F0010F3BD04278D9B2521E4A
:1051A000427000EBC10282F85A5190F802C000220E
:1051B000BCF1000F0BD9841894F803618E4202D120
:1051C000102A26D103E0521CD2B29445F3D80278BB
:1051D000521ED2B202708A421BD000EBC20200EB18
:1051E000C10CD2F85341CCF85341D2F85721CCF836
:1051F0005721847890F800C00022002C09D9861825
:1052000096F8036166450CD1102A1CBF024482F84F
:105210000311591E4BB2002BB8DA0548457070BC1B
:105220007047521CD2B29442E9D8F2E7A210002093
:10523000F40100202DE9F041254D00263446287860
:1052400000288CBF234FBDE8F08100BF05EBC400F0
:1052500090F85A1111F0010F32D0AA78002123469C
:10526000002A09D905EB010C9CF803C19C4504D028
:10527000491CC9B28A42F5D810218A4286BF05EB83
:105280000112D31C0023002210290CD005EB010CC5
:105290009CF83B81B8F1010F04D09CF84BC1BCF1E4
:1052A000000F00D00122521E134209D1B95590F8C7
:1052B000532100F5AA713046731CDEB206F03CFEA5
:1052C000601CC4B22878A042C0D8BDE8F0810000BC
:1052D000A2100020F80100202DE9F00F204B02461B
:1052E000002093F80080B8F1000F34D90F784E7881
:1052F0008D78CC7891F804C091F805A003EBC0013B
:1053000091F8539191F854B182EA090987EA0B0B9D
:10531000D94491F855B186EA0B0BD94491F856B1AE
:1053200085EA0B0BD94491F857B184EA0B0BD944A9
:1053300091F858B191F859118CEA0B0BD9448AEACB
:10534000010111EB090F04BFBDE8F00F7047401CCD
:10535000C0B28045D2D8BDE8F00F102070470000E1
:10536000A2100020254910B44A7801EBC003521E58
:105370004A70002283F85A2191F802C0BCF1000F54
:105380000DD98B1893F80341844204D1102A1CBF15
:1053900010BC704703E0521CD2B29445F1D80A7891
:1053A000521ED2B20A70824204BF10BC704701EB99
:1053B000C00301EBC202D2F853C1C3F853C1D2F803
:1053C0005721C3F857218C7891F800C00022002C97
:1053D0009CBF10BC70478B1893F80331634506D10E
:1053E000102A1CBF114481F8030110BC7047521CE5
:1053F000D2B29442EFD810BC70470000A210002037
:1054000070B58CB000F110041D4616460DF1FF3C3E
:105410005FF0080014F8012C8CF8012014F8022D1C
:105420000CF8022F401EF5D101F1100C6C460DF165
:105430000F0108201CF8012C4A701CF8022D01F8FD
:10544000022F401EF6D1204608F0C0FC7EB16A1E35
:1054500004F130005FF0080110F8013C537010F8BF
:10546000023D02F8023F491EF6D10CB070BD08980B
:105470002860099868600A98A8600B98E8600CB0EA
:1054800070BD000070B50446012669B1012924D021
:1054900002294BD0032918BF70BD04F1A701BDE854
:1054A0007040A63000F0E6B84FF45272002107F0C9
:1054B0009BFB84F8A66005F0F9F944F62B12104026
:1054C000C4F8F20001F00601C4F8F610FE2084F8DA
:1054D0002C017F2084F8990070BD0025A4F8865225
:1054E00084F87B52616916480A460844B0FBF1F023
:1054F000C4F8C80040F6B830A4F8CC00E38B04F13F
:10550000900000F067F804F1A701481E00F0B2F81F
:1055100007F0CCFA38B1A06900F052FC002804BFB3
:1055200084F86C6270BD84F86C5270BDB4F82A3394
:10553000D4F824236169BDE87040903000F04AB887
:105540007FC3C90141F64C5291423DBF0549A1FBC1
:105550000010400940F2E24128BFB0FBF1F080B2F8
:10556000704700001F85EB5141F64C5291423DBF00
:105570000549A1FB0010400940F2E24128BFB0FB01
:10558000F1F0C0B2704700001F85EB5130B400222B
:10559000A1F1010CBCF1000F12DD431E11F0010F4F
:1055A00008BF13F8012F5C785FEA6C0C08D000BFCD
:1055B00013F8025F22435C782A43BCF1010CF7D157
:1055C000491E5CBF405C0243002A0CBF0120002042
:1055D00030BC704710B44FF0000CA0F842C0B0F8D7
:1055E00046C0184C0CFB01FCBCFBF2FCA0F846C00A
:1055F00042F2107C03FB0CF3B3FBF2F35B1C9BB297
:1056000003FB02FCA0F84430A44584BF5B1EA0F855
:1056100044300D4B40F2712CB3FBF2F35B1CA0F84D
:105620004A30838F03FB0CF302EB03135B1EB3FBC7
:10563000F2F38363436B5943B1FBF2F1416310BC56
:10564000704700000048E801005A6202074908B5A7
:1056500009788DF800109DF8001000291CBF00206B
:1056600008BD03490AF05EFE012008BD16020020B5
:105670001702002010B50446401C884218BF0AF0EB
:1056800051FE607900F01F006071002084F80B006B
:1056900004EB000C401C9CF8012002F001015208B0
:1056A00002F001031944520802F0010319445208A0
:1056B00002F001030B44510801F001021A444908A9
:1056C00001F001031A44490801F001031A4402EBF6
:1056D00051018CF80610E27A05281144E172D7DBFB
:1056E00010BD00000449897D01F0040108430CBF8E
:1056F0000120002070470000BC0F00200348807D7F
:1057000010F0020F0CBF012000207047BC0F0020DA
:105710000348807D10F0010F0CBF0120002070476E
:10572000BC0F002008B5D8B1037A8DF800309DF881
:105730000030002B18BF08BD002303604160EFF369
:10574000108372B60A49D1F800C0BCF1000F1ABF2D
:10575000D1F804C0CCF800000860486033B904E018
:1057600040F241411020FEF729FC62B6027208BDEA
:10577000EC0000202DE9F04F87B004000FD0FE4868
:10578000012700250178002908BFDFF8F0B30BD00E
:105790006570032121702771057000F0BAB840F2DE
:1057A0005D311020FEF70AFCDBF80000A846002857
:1057B00008BF464622D0017A8DF800109DF80010EF
:1057C000082909D140680088FFF742F807F03BFF3D
:1057D000002808BF2E4611D0EFF31080DBF80060E0
:1057E00072B63168CBF8001000B962B6307A8DF825
:1057F00000009DF80000002808BFB846B8F1000F6F
:10580000D2D1DEB1307A8DF800009DF80080B8F179
:10581000220F80F08482DFE808F0FEFD8024FCFD8A
:10582000FDFBFDFDFDFDFDFE24FCFDFD24FC5454AF
:1058300054FDFD24FDFDFAF924F815F707B000200A
:10584000BDE8F08F6570142020706560A560E5608C
:1058500025616561A561E5610220256220713572CF
:1058600057E0C7480368002B04BFA946357250D0E3
:10587000706842462146984720787168142802D003
:10588000172803D01BE0207930B918E02079B0B197
:10589000084608F0D8FF90B9E4880121204608F0B6
:1058A000D2F860B10088FFF72FFA01212046FEF7F9
:1058B00035FE20B14FF4AF711020FEF77FFB35723B
:1058C00027E0B0480368002B04BFA946357220D0FA
:1058D000B8F1150F17D077684246214638469847E9
:1058E00020781B2803D019280BD1207948B138899A
:1058F0000421FEF713FE28B14FF46B711020FEF760
:105900005DFB357205E0A04B706800221B682146E4
:10591000984707B00120BDE8F08F9C480368002B32
:1059200004BFA9463572F4D00222214600209847D0
:1059300004F05AFF0028ECD02078052803D0CF21AE
:105940001020FEF73BFBA07B10F0100F22D01C2292
:10595000211D8F4807F0CEF8227B04F120018D48ED
:1059600007F0C8F88A49887A10F0040F02D0C87C82
:10597000FE2815D04FF00402227008686060486865
:10598000A0600889A081887A10F0080F18BFA27360
:1059900033D11DE04FF0D0014FF01000FEF70EFBA9
:1059A000132020700878207167714878A071D1F8B1
:1059B0000200C4F80700C888A4F80B00FE2060733A
:1059C0004869C4F80E00088B6082487A2075A0E709
:1059D00010F0010F1CBF10F0020FA5730DD110F0D5
:1059E000040F18BFA77308D110F0010F16D110F0E3
:1059F000020F18BF022011D0A0730A7A1F2A17D9EC
:105A00004FF48A71102007E051E183E170E178E101
:105A100058E113E03AE082E1FEF7D0FA10F0030F0C
:105A200008BF0320E8D040F211111020FEF7C6FA9B
:105A3000584904F10F0007F05DF86AE7534803681E
:105A4000002B04BFA94635723FF463AF424621469E
:105A5000002098472078182804BF2079012813D106
:105A6000E0884FF0000107F0EEFF04000CD0208822
:105A7000FFF74AF920880021FEF750FD20B14FF4CE
:105A800096711020FEF79AFA357242E74248006894
:105A9000002800F04981706878B100F1900900F5A4
:105AA000B971B0F800A04046B8F1100F63D009DC1E
:105AB00001280CD00B2821D0C0E040F28221102018
:105AC000FEF77CFA1A2878D01B2831D0B6E0B9F15D
:105AD000000F0DD0657027702571A4F805A099F806
:105AE0005D00E071B9F85E002081B9F86000608166
:105AF000B8F10B0F1CBFA94635720AE75046FEF7F6
:105B0000BDFE80B165700F212170A4F806A0278129
:105B100000222771114607F0A0FEB8F10B0F1CBF41
:105B2000A9463572F5E64FF4CE711020FEF746FA1D
:105B3000FFF7EEFD90B335725046ADF800A002A914
:105B400008F00BFA20B14FF4B7711020FEF736FAC7
:105B5000039890F86E108DF8021090F86F108DF881
:105B60000310B0F87000ADF804000221684609F097
:105B700064FFD0B114E051E0C0120020EC0000201E
:105B8000F400002004010020000100200801002092
:105B900085120020A1120020FC0000204DE00CE046
:105BA0004FF4C2711020FEF709FAB8F10B0F1CBFB9
:105BB000A94635727FF4F8ADABE6FFF79FFDE0B381
:105BC000357203A9504609F0A6FD20B140F28B11B1
:105BD0001020FEF7F3F9ADF800A0BDF81200ADF803
:105BE0000200BDF81400ADF80400BDF80E00ADF8D9
:105BF0000600BDF81000ADF80800684609F0BAFDCF
:105C000020B14FF4CA711020FEF7D8F9B8F10B0F8C
:105C10001CBFA94635727FF4C7AD7AE691F82C0017
:105C200000F00100FFF75EFDC0B1B8F10B0F1CBF23
:105C3000A94635727FF4B8AD6BE6FFE7B8F1080FFF
:105C400011D03A4803681BB1706842462146984714
:105C5000B8F10B0F1CBFA94635725AE633480368EA
:105C6000002BF1D1F4E75046FEF7F2FD07F0EBFC14
:105C7000C0B15046FFF748F800215046FEF74EFCF1
:105C800001215046FEF74AFCB9F1000F08D06570BB
:105C90000C2020702571A4F805A099F82E00E07161
:105CA000357236E640F2C3211020FEF787F96570A1
:105CB0001D202070D6F809006060D6F80D00A060A5
:105CC000357226E61948006880B1706865700A214F
:105CD00021700188A180D0F83813D0F83C23C4F893
:105CE0000610C4F80A20B0F84003E081357210E6CF
:105CF0000F4803681BB100222146104698473572B1
:105D000007E60C4803681BB100222146104698475D
:105D10003572FEE56570272020703572F9E540F296
:105D20002D411020FEF74AF93572F2E5FC00002003
:105D30000C010020F800002009490870002048608C
:105D400088600849C1F83B00C1F83F00C1F8430032
:105D5000C1F84700A1F84B0081F84D0070470000E2
:105D6000E800002085120020084900204860886073
:105D70000749C1F83B00C1F83F00C1F84300C1F832
:105D80004700A1F84B0081F84D007047E800002063
:105D90008512002001480078FDF7E8BDE8000020EA
:105DA0000249014808607047A5E60000F4000020A1
:105DB0000249014808607047257A00000801002068
:105DC00070B46FF01F02010C02EA90251F23A1F5A9
:105DD000AA4054381CBFA1F5AA40B0F1550009D023
:105DE000A1F52850AA381EBFA1F52A40B0F1AA009B
:105DF000012000D100204FF0000C62464FEA0C0455
:105E00008CEA0106F6431643B6F1FF3F11D005F0C8
:105E100001064FEA5C0C4CEAC63C03F0010652084E
:105E20006D085B08641C42EAC632162CE8D370BCCD
:105E3000704770BC0020704710B50C4C08212046FC
:105E4000FEF746F92068002804BF60680028F5D0F6
:105E5000074C00BF4FF008012046FEF739F92068D3
:105E6000002804BF60680028F4D010BD1001002095
:105E700018010020094A0A48D2E9001348434B4060
:105E800083EAB11181EA432111604FEAF0604FEAE1
:105E9000F34100EB800051607047000010010020CA
:105EA000BB79379E094A0A48D2E9001348434B4060
:105EB00083EAB11181EA432111604FEAF0604FEAB1
:105EC000F34100EB80005160704700001801002092
:105ED000BB79379E2DE9F0410446807C002816BF2F
:105EE00002280020012084F8600018B3607E68B3A7
:105EF000D4F81300C4F86100B4F81700A4F86500E2
:105F0000A07C022816BF032801210021A1764FF0B2
:105F10000800E07694F860004FF001074FF00008A9
:105F2000012804BF94F8662012F0C00F1BD001288E
:105F300011D016E004F161010020FEF7F3FE002805
:105F4000DED140F28A412D20FEF738F840F28E4132
:105F50002D20FEF733F894F8660000F0C0004028CA
:105F600001D0002000E00120207731B194F86700D3
:105F700004F16801FFF736F8E076FFF761F837497A
:105F8000A0FB0165FCF76CFB80196941C4E91601AF
:105F90000026E07EFEF75AFF0546A07E002818BFC7
:105FA000002D03D0E07EFEF745FF58B194F87A004B
:105FB00000281CBF207F00281DD094F86000012815
:105FC0000ED013E084F86070324604F16101284677
:105FD00007F043FFE17E04F16100FEF743FF0AE0B2
:105FE00094F8660000F0C00040282FD0414604F12C
:105FF000610007F021FF84F86E80A07810F0040F94
:1060000008BFBDE8F0810026E07EFEF765FF0500D1
:1060100008BFBDE8F0811021FFF7B8FA002818BFCB
:10602000BDE8F08184F86E70324604F16F012846B5
:1060300007F013FF04F16F01094CA06808F05BFA48
:10604000A068BDE8F041012108F05CBAFEF7C2FE8D
:10605000324604F1610107F000FFCCE740420F0037
:1060600020010020F8B50446283008F08FFC618834
:10607000C1F3001222B1BDE8F840282201F034BA81
:10608000C1F34002002A14BFB4F854C0B4F84CC0A5
:1060900022791E4B4FF47A75082A33F8123003F236
:1060A000E733B3FBF5F608BF40250AD0042A08BF42
:1060B000102506D0022A07BF04251223082519231C
:1060C00000E0142315FB03F3082A08BF402519D06C
:1060D000042A08BF2E2515D00025022A0CBF18223D
:1060E00028222A441A4412FB00626FF07F0303EB5C
:1060F000C01010440091014662790123604600F00F
:1061000083FEF8BD4FF4A872EBE700009C7400001A
:106110002DE9F04F80468DB00C46C269D8E90501E3
:10612000D8E90076D8E903A90592CDE90301D8F8AA
:106130002000069001A808F0A1FCA07A60F317499E
:10614000207860F30707B4F80100ADF800009DF86F
:10615000000000F00101C0F3400241EA4201C0F337
:10616000800241EA8201C0F3C00241EAC201C0F3E9
:10617000001241EA0211C0F3401241EA4211C0F399
:10618000801041EA801B207D6BF31F47012818BF58
:10619000022803D0032808BF08200ED1617860F3DD
:1061A000070611F0100F0FD1A17D012918BF022998
:1061B00008D0032908BF082104D040F2BB210620E3
:1061C000FDF7FCFE61F30F26CAF30741012908D051
:1061D000617A01A808F02DFC207D012102280FD151
:1061E0000BE00421082808BF61F30706C6F3072067
:1061F000082808BF61F30F26EAE7607D401CC1B2A2
:10620000A07E401CC2B201A808F0A9FB380C10F017
:10621000080F4FF0000524D101A808F0B7FB617802
:1062200011F0100F7BD02822594601F05DF900BF14
:1062300040F2712100F2D920B0FBF1F000FB01F532
:10624000D4F8020040F27122000A4143D4F805005C
:10625000000A50438D4298BF0D4602D9854288BF3F
:106260000546A07C60F30F29207E012818BF00207E
:1062700060F3070AD8F8440007F0B6FC8346D8F864
:10628000440007F059FD834528BF584698B101A93D
:106290000891390CADF824108DF82C60310A8DF876
:1062A0002D100A9508A901F003F8002802BF452027
:1062B0000DB0BDE8F08FC8F80CA0C8F80070C8E9B0
:1062C0000165DDE90301059AC8F81090C8F81C20A3
:1062D000C8E905010698C8F820000198C8F8280008
:1062E000BDF80800A8F82C00E07A002816BF0228A4
:1062F0000020012088F86700E068C8F86800208A5C
:10630000A8F86C00E07D98F83E1060F3071188F85B
:106310003E100DB04FF00000BDE8F08FFFE70346E0
:10632000F0B221494FF47A72082831F8101001F2C6
:10633000E731B1FBF2F208BF4FF0400C0DD004285A
:1063400008BF4FF0100C08D0022807BF4FF0040C14
:1063500012214FF0080C192100E014211CFB01F15F
:10636000082808BF40251BD0042808BF2E2517D0B9
:1063700002280CBF182028202844084410FB0320C2
:106380006FF07F0101EBC3114518FEF74BFB390C91
:106390000091C6F307220123294600F035FD47E7A7
:1063A0004FF4A870E8E700009C740000104A10B594
:1063B000002111700F4CA060107820B140F20A311A
:1063C0002D20FDF7FBFD116051609160D1601161DE
:1063D00051619161D16104F00DFC04F0FDFAE068B7
:1063E000002818BF10BD40F20D312D20FDF7E6FD4D
:1063F000E80F00202001002002490148C8607047D2
:10640000D07400002001002002494860C968096872
:1064100008470000200100200B4910B5087800282B
:1064200018BF0C2401D0204610BD00240C604C6025
:106430008C60CC600C614C618C61CC6104F0DAFB47
:1064400004F0CAFAEFE70000E80F0020054910B594
:10645000097801291CBF002010BD00F0BDFE0020FE
:1064600010BD0000E80F00202DE9F041704E0F0034
:10647000044627D004F1280008F0DDFAC0B9A0785E
:10648000C0F3C000002838D004F1280008F07EFADC
:10649000054604F1280008F0CEFA281AC0B208F028
:1064A000FAFA71680844706004F1280008F0EEFA06
:1064B00004F1280008F07AFA05F062FA2179252023
:1064C00005F02AFA5B4D94F86E800021A8680180DF
:1064D000017801F0DF010170618813292DD011DCF2
:1064E000102908BF02213DD0122908BF062139D04A
:1064F00040F24A612D20FDF761FD2046BDE8F041E4
:1065000000F06ABE152918BF1D29F1D14FF0010115
:1065100007F0CFFFA868B8F1000F017801F0DF01A4
:1065200041F02001017013D004F16F0107F0E3FF87
:106530000121A86807F0E6FF16E0002107F0B9FF87
:10654000A868017801F0DF0141F0200101700BE043
:1065500004F1680107F0CFFF94F86710A86807F00E
:10656000D1FF01E007F0A5FFA04604F16101A86892
:1065700007F0D1FF98F86010A86807F0D3FF608893
:106580001D2818BF152805D094F84C20A16CA868C8
:1065900007F07FFFA86804F09DFF0420307027B348
:1065A0006088102831D004F12800B56808F0EEF9B1
:1065B000074604F1280008F03EFA381A401EC0B21F
:1065C0006188282200F0B6FF0544A078C0F3C0001F
:1065D00030B17068054408F062FA2844C4F8180124
:1065E00022792946002004F0C3FF6088132815D0C3
:1065F00010DC102808BFBDE8F08112280ED000BFC3
:1066000040F648512D20FDF7D9FC2179002004F0F7
:10661000C1FBEAE7152818BF1D28F1D12279BDE892
:10662000F0414FF001014FF0000005F0E9B8000023
:10663000E80F0020200100202DE9F8434A4E814652
:10664000307802281CBF3078032805D040F6B941C5
:106650004FF02D00FDF7B2FC444C6568287B40B13B
:1066600005F13F0005F03AF9002804BF7F2085F8C6
:106670003F00D4F808C061684FF000089CF80000A3
:106680000A6A00F00F07002A18BF92F87780B9F164
:10669000000F4DD001F1610391F86020C0090CF1A9
:1066A000090107F0A2FB002842D06568052F21D11F
:1066B000A06890F8240000F01F0010281AD9E87B89
:1066C000C0B1FF208DF800006A460521284600F081
:1066D00013FB68B3A0682222C11C05F1E10006F09B
:1066E00009FA1E22294605F1D800FFF71BF8FFF72B
:1066F00051FB1DE04146A06807F01DFEC0B1327895
:1067000060683946022A1CBF3278032A05D040F659
:1067100092414FF02D00FDF751FCE2683378526949
:106720006FF0070C0CEB8303D2589047054600E04E
:106730000125B07B18B104F05DFA04F04DF9002D8D
:1067400008BFBDE8F883606808F0BBF938B104F011
:1067500079FAE068806801B0BDE8F04300476068FE
:10676000BDE8F84300F038BDE80F0020200100200C
:1067700030B583B0032902D0052974D06FE00446F8
:10678000FF208DF8080002AA0321204600F0B4FA89
:10679000002864D0207B384D00283ED094F8CE00ED
:1067A0008DF800009DF80000B8BB9DF80800217826
:1067B00084F8CF10FF2811D004F1D102511EFEF74A
:1067C000E5FB30B194F8D00040F0020184F8D0101D
:1067D00012E040F693712D20FDF7F0FBA8680178D8
:1067E000C1F3801284F8D020D0F80320C4F8D1205F
:1067F000B0F80700A4F8D50094F93F007F2829D00D
:1068000084F8D7007F2184F83F101922214604F133
:10681000C600FEF787FFFFF7BDFAA86800210180D8
:10682000042107F046FE04F16101A86807F073FE39
:1068300094F86010A86807F075FE94F85420216D54
:10684000A86807F078FE0D4905200870A86804F0D4
:1068500041FE0EE040F6FB512D20FDF7AFFB03B0EB
:10686000012030BDFFE70649096811B188470028BB
:10687000F5D003B0002030BD20010020E80F00203B
:1068800030010020094A0300506801D000F0A4BC88
:10689000002908BF7047D168054A096912786FF06E
:1068A0000F0303EB820289580847000020010020F3
:1068B000E80F002070B504464088102810D0114D14
:1068C000A87B20B104F0C8F8402004F0A1F90E48DC
:1068D000806804F0FFFDA07810F0040F0BD105E0F4
:1068E0002046BDE870400121FFF7BEBD002122799E
:1068F000084604F085FF002004F07AFC022028708E
:1069000070BD0000E80F00202001002070B51F4C72
:106910006568287B40B105F13F0004F0DFFF0028E7
:1069200004BF7F2085F83F00194DA87B18B104F003
:1069300061F904F051F8606808F0C3F8A8B1606824
:106940004188C1F30012002A04BFC1F3C00100292D
:106950000BD0297802291CBF297803290AD040F6D8
:10696000C6314FF02D00FDF729FB6068BDE870408F
:1069700000F032BCE1682A78C9686FF0070303EBC6
:1069800082028958BDE870400847000020010020BD
:10699000E80F00202DE9F047A34D04468AB028787F
:1069A00000287CD12078FF2879D00026AE816E6047
:1069B0006E70AE7084F879609C4802AFDFF8708228
:1069C0000FC887E80F00D8F80C004068059002A8AF
:1069D00004F0F8FB04F0D6FC05F0E6FA04F00AF93E
:1069E00003F0FAFF934804F083FF934804F08AFF12
:1069F0000020FDF79FF804F1280008F047F804F1A3
:106A0000280007F0D3FF04F0BBFF2179252004F014
:106A100083FF94F9100004F051FD2179002004F067
:106A200083FA0127A860002801BF2F7000200AB058
:106A3000BDE8F087207F002801BFA07E0028A07855
:106A400010F0040F66D0D4E916016FF0004281EA1D
:106A5000020171EA000079D0FBF702FED4E91623A7
:106A6000801A71EB030071D3FEF7EAFA7349A0FBB9
:106A700001A9FBF7F5FD10EB0A0041EB0901C4E9A0
:106A800016014FF0010AE07EFEF7E0F98146A07E94
:106A9000002818BFB9F1000F05D0E07E00E00EE03D
:106AA000FEF7C8F978B194F87A0000281CBF207F5F
:106AB000002821D094F86000012812D017E00AB015
:106AC0000C20BDE8F0873A4684F8607004F161015B
:106AD000484607F0C2F9E17E04F16100FEF7C2F911
:106AE0000AE094F8660000F0C000402813D0514638
:106AF00004F1610007F0A0F9A07810F0040F25D090
:106B0000E07EFEF7E9F95FEA00091FD01021FEF7E9
:106B10003DFD40B11AE0FEF75DF93A4604F161012E
:106B200007F09BF9E8E73A4684F86E7004F16F01CC
:106B3000484607F092F904F16F01D8F8080007F011
:106B4000DAFC0121D8F8080007F0DCFC04F1480168
:106B5000606C07F0BFF8074604F15001606C07F065
:106B6000BCF894F87C1038438DF804109DF804109C
:106B7000002918BF0121084318D0A078C0F30010E5
:106B8000002804BFB4F83D00C0F30B070ED100BFCE
:106B9000FFF770F9C0F30B00B842F9D0B4F83D101C
:106BA00060F30B01A4F83D1084F87C60FEF742FB13
:106BB000D8F80800C01CFEF7F9F8A873A07810F008
:106BC000010F2CD006A9012006F047FF20B140F6A6
:106BD0008C112D20FDF7F2F9FF20287606A8266AF1
:106BE000FDF72AFCD8B9089CB44213D0727A607AB7
:106BF00006F10A0304F10A0107F0F7F850B1A07892
:106C00002876D4F80300C5F81900B4F80700A5F8F1
:106C10001D0004E006A8FDF70FFC0028E3D00AB031
:106C20000020BDE8F0870000E80F0020B0740000ED
:106C300020010020D6BE898E9974000040420F00CA
:106C400010B50446FFF7A6FE002818BF10BD054882
:106C50000078012803D000212046FFF705FC002022
:106C600010BD0000E80F00202DE9F041204E214D1D
:106C700074682878002808BFBDE8F08128780228C9
:106C80001CBF2878032811D1207B48B1274604F186
:106C90003F0004F023FE002804BF7F2087F83F0058
:106CA000A87B18B103F0A6FF03F096FEFCF726FFC1
:106CB0003078C0B1204607F004FFA0B17068817839
:106CC000C1F3C00121B1BDE8F0410121FFF7CCBB08
:106CD0000446283007F0AFFE28B12046BDE8F04159
:106CE0000121FFF7C1BB2046BDE8F04100F074BAB6
:106CF00020010020E80F00202DE9F04790460D46C6
:106D0000044603291BBF94F8780000284FF00009BF
:106D10004FF0010903F088FF0646032D08D0012734
:106D2000052D02BFA07810F00100BDE8F08707E054
:106D3000A0780227C0F34000002808BFBDE8F08714
:106D4000B9F1000F59D12E48807B40B107F0EFF820
:106D500088F80000FF2802D0FEF732F90643294DDB
:106D600094F8672004F16803A96811F8030BC0F3D5
:106D7000801007F03AF898F80010FF2904D0B8B94D
:106D8000E07E884216D113E0A0B1A96811F8030B88
:106D9000C0F38010FEF726F98046FEF797F938B168
:106DA0004046FEF799F818B11021FEF7EFFB08B145
:106DB000012000E00020A17811F0040F01D0E0B123
:106DC00018E0BEB9607C002818BFB84215D1A96888
:106DD00011F8030BC0F38010FEF704F90446FEF728
:106DE00075F938B12046FEF777F818B11021FEF793
:106DF000CDFB10B10120BDE8F0870020BDE8F08791
:106E0000E80F0020200100202DE9F84F44F255251D
:106E1000DDF828C00CF00104CCF3400AA0F1EB0C23
:106E2000009454EA0A0B1FFA8CFC0CF1F60404FBE4
:106E300005F44FEA94590CFB05F44FEA9457FCB261
:106E40006FF0F60514FB05F404EB0C061FFA86FC44
:106E50000CF105084FF0000C4FF4C8744FF4BF75E7
:106E600000F0488101F5A571BAF1000F1BD0082A86
:106E700004BFA3464FF0400A0FD0042A04BFAB461C
:106E80004FF0100A09D0022A07BF0CF1180B4FF07F
:106E9000040A0CF1280B4FF0080A0AEB8A0E0EEBDD
:106EA0008A1ADA441AE0DBB1082A04BFA3464FF07D
:106EB000400A0FD0042A04BFAB464FF0100A09D095
:106EC000022A07BF0CF1180B4FF0040A0CF1280B33
:106ED0004FF0080A0AEB8A1A0BEB8A0A514421E0A8
:106EE000FF2834BF82464FF0FF0A0AF1050B082A3B
:106EF00004BF4FF0400A0BFB0A1127D0042A1FD011
:106F0000022A0CBF4FF0040A4FF0080A0BFB0A11CB
:106F100007BFE2464FF0180B4FF0000A4FF0280B66
:106F2000DA4451449C3102F00C0ABAF1000F18BF48
:106F30004FF0280A514418BF01F5416126D108E0FD
:106F40004FF0100A0BFB0A114FF02E0A4FF4A87BEA
:106F5000E6E7082A04BFA3464FF0400A0FD0042AF0
:106F600004BFAB464FF0100A09D0022A07BF0CF14C
:106F7000180B4FF0040A0CF1280B4FF0080ACAEB6B
:106F8000CA0A0AEB4A0A0BEB4A0A514401F1980A71
:106F90000099C1B1082A08BF40200CD0042A04BFC0
:106FA0002C46102007D0022A07BF0CF11804042039
:106FB0000CF12804082000EB400101EB00102044F4
:106FC00000EB0A0191E0BBB1082A04BFA3464021AF
:106FD0000CD0042A04BFAB46102107D0022A07BFF9
:106FE0000CF1180B04210CF1280B082101EB811185
:106FF0000BEB810151441CE0FF2834BF0146FF2107
:1070000001F1050B082A04BF40210BFB01AA1ED089
:10701000042A18D0022A0CBF042108210BFB01AA64
:1070200007BF61464FF0180B00214FF0280B594461
:107030005144EB2859D913B3082A0ED0042A09D099
:10704000022A0CD00FE010210BFB01AA2E214FF4D5
:10705000A87BECE72C46102008E0402006E00CF16D
:107060001804042002E00CF12804082000EB801032
:1070700004EB800000F5A57009FB001135E0FBB2C0
:10708000082A04BF204640270CD0042A04BF284603
:10709000102707D0022A07BF0CF1180004270CF1B3
:1070A0002800082707EB871700EB870000F5A5707D
:1070B00003FB00113004000C17D0082A07D0042A63
:1070C00002D0022A05D008E02C46102008E040201B
:1070D00006E00CF11804042002E00CF1280408205A
:1070E00008FB0010204400F5A57101F20B10BDE86B
:1070F000F88F00BF01F5A57ABBB1082A04BFA346EB
:1071000040210CD0042A04BFAB46102107D0022A2C
:1071100007BF0CF1180B04210CF1280B082101EB1F
:1071200081110BEB810151441CE0FF2834BF014663
:10713000FF2101F1050B082A04BF40210BFB01AA26
:1071400021D0042A1BD0022A0CBF042108210BFBEA
:1071500001AA07BF61464FF0180B00214FF0280B22
:1071600059445144EB28C0D983B1082A3FF475AF84
:10717000042A3FF46FAF022A7FF475AF6FE7102146
:107180000BFB01AA2E214FF4A87BE9E7FBB2082AEA
:1071900004BF274640200CD0042A04BF2F461020ED
:1071A00007D0022A07BF0CF1180704200CF12807AA
:1071B000082000EB801007EB800000F5A57003FBB2
:1071C00000113004000C90D0082A80D0042A3FF42B
:1071D0007BAF022A81D17CE72DE9F0410446B0F86B
:1071E0004000324E401CA4F84000B07B002520B186
:1071F00003F000FD03F0F0FBB573357094F87900EF
:1072000028B12046BDE8F041012107F06FBC607B4A
:10721000002844D0B4F84010884240D801212046CC
:1072200007F064FCA07810F0010F22D0206A4326FA
:107230000788FEF7AFFD03F0D7FA002818BFBDE8B6
:10724000F081207884F8B300A4F8B47084F8B260B8
:10725000607B10B984F8B65003E094F8400084F8DD
:10726000B600214604F1A800BDE8F0411222FEF765
:1072700059BA4FF6FF774326FEF78CFD03F0B4FAB8
:10728000002818BFBDE8F081207884F8B300A4F886
:10729000B47084F8B260607B0028DED1DAE7204663
:1072A000BDE8F041002107F021BC0000E80F0020FC
:1072B000F8B50A7912F0180F5CD105460C0028D0F9
:1072C000206800282AD007F061FB237B627B042B17
:1072D00008BF0823042A08BF082229494FF47A7CF2
:1072E000082B31F8131001F2E731B1FBFCF708BFAE
:1072F0004FF0400C17D0042B08BF4FF0100C12D0E9
:10730000022B07BF4FF0040C12214FF0080C19217B
:107310000AE040F2E2312D20FCF750FE40F2E3316A
:107320002D20FCF74BFE14211CFB01F10026082B3D
:1073300008BF4FF0400C1FD0042B08BF4FF02E0C9D
:107340001AD0B446022B0CBF1823282363441944D7
:1073500011FB00716FF07F0303EBC0100144A088A4
:10736000009000232846FFF74FFDA16881423CBFF3
:107370003046F8BD0120F8BD4FF4A873E6E70000E1
:107380009C740000F8B5044690F8860016460D4639
:107390008DF800009DF8000020B140F6FA312D2054
:1073A000FCF70CFE84F888302888A4F88A00002BAB
:1073B00018BFF8BD686906F0F4FDA4F8A000A88B1A
:1073C000A4F8A200E88BA4F8A40095F86D0284F854
:1073D000A600A07E002148B194F86000012805D1E4
:1073E00094F8660000F0C00040282ED094F87A008F
:1073F00040B194F86000012804BF94F8660010F0D2
:10740000C00F22D0C4F89410A4F898101C48FF2E86
:1074100080680178C1F3801184F88D10D0F80310D2
:1074200021D0C4F89A10B0F80700A4F89E0004F127
:107430008E02511E3046FDF7A9FD78B194F88D00FB
:1074400040F0020084F88D00F8BDD4F86100C4F863
:107450009400B4F86500A4F89800D7E740F61B4103
:107460002D20FCF7ABFDC4F88E10B0F80700A4F88F
:10747000920004F19A00BDE8F84008F058BF0000FF
:1074800020010020024801214068FEF7EDBF000006
:1074900020010020030000000155555500002CA6D6
:1074A000E0A1000020A800000000000020A80000CB
:1074B0000D690000396600008568000000000000CA
:1074C00071670000B568000053E9000059E9000049
:1074D000416C0000696C000085740000CC740000F1
:1074E000C4740000C074000010B5421E022A03D903
:1074F000CA212F20FCF762FD401E102902BF0A4955
:1075000031F8100010BD122914BF1329074907D004
:10751000152908BF064903D0D8212F20FCF74EFDBE
:1075200031F8100010BD0000B6EA0000B0EA00001B
:10753000BCEA0000421E10B5D2B2012A05D91D29AD
:107540001ED0EE212F20FCF739FD132914D008DCC2
:10755000102902BF0D4830F8120010BD12290BD0BF
:1075600005E0152908BF0A4807D01D2908D04FF4A7
:1075700081712F20FCF722FD064830F8120010BD63
:1075800040F25A3110FB01F010BD0000A4EA0000E7
:10759000ACEA0000A8EA00002DE9F043044690F8A8
:1075A000200183B016460D4640BB21466A48FAF7D3
:1075B00087FE0746202821D05022002104F5847040
:1075C00005F012FB84F808714FF00108C4F80C5163
:1075D00084F8208135B1FEF765FC00F00700401CFF
:1075E00085F89C02204607F032F9002808BF6B2579
:1075F00029D0204607F01DF920B10AE003B00C2085
:10760000BDE8F083204607F026F9002808BF422590
:1076100000D049256846FCF73FFB9DF80000002894
:1076200014BF0127002701A8FCF71EFB9DF80400EA
:10763000002818BF0120384318BF0935FCF772FA3B
:10764000002818BF1835A4F83051022084F8320100
:1076500084F83381002584F8285105F0E4F80746C2
:10766000B4F83091FBF722FF4F4598BF4F4638449E
:10767000CC3087B2204607F0E6F878B308F009FE70
:1076800000F5CD6081B2304605F005F93044C4F80C
:107690002C01FAF7E5FFC0196941C4E94E0184F8ED
:1076A000095184F81081204607F0C7F840B1204600
:1076B000FEF7D8FC00F59670301AA0F57F7005E053
:1076C000012007F0E8F900F59670301AC4F81401AB
:1076D0004FF0FF304108C4E9520126E0FFE72046A1
:1076E000FEF7C0FC00F59670C4F82C0184F80981FF
:1076F000FAF7B6FF81468846FEF7D4FB42F21071D6
:10770000B0FBF1F201FB1200384410EB090045EB2D
:107710000801002EC4E94E0104BF4FF0FF304108BC
:1077200001D080196941C4E9520194F8080104F5B7
:107730009471F9F7BBFF48B1A4F8405100212046ED
:1077400007F0AFF803B00020BDE8F0834FF4F67106
:107750003020FCF733FC000085EC000003480021DA
:10776000017001228270417000F002B834010020E3
:107770002DE9F04186B06946022006F06EF920B18D
:1077800040F237113020FCF719FC6846FCF754FE34
:107790000126002510BB029C94F82001C8B184F892
:1077A00050610121204607F07CF894F8200180B157
:1077B00094F80801FAF714FB94F80801FAF768FC4A
:1077C00094F80801FAF742FC002818BF84F8205109
:1077D00010D06846FCF730FE0028DCD02C4F7E70BD
:1077E00003A9012006F039F9002808BF4FF6FF76FB
:1077F0002DD027E040F209213020FCF7DFFB05986F
:1078000000281CBF90F8AC12002920D00088B0429C
:1078100018BF4FF0200835D0012106F014F90400FC
:107820001BD094F8F402FAF733FC84F8AC5294F8C5
:10783000F402FAF70BFC84F8F48203A9012006F0A5
:107840000CF9D0B140F203113020FCF7B7FB03A8CC
:10785000FCF7F2FD0028D2D014E040F223113020D2
:10786000FCF7ACFB059800281CBF90F8AC1200296F
:1078700003D00088B042CFD104E003A8FCF7DCFDC0
:107880000028EFD07D7006B00020BDE8F081000038
:1078900034010020014908707047000034010020C5
:1078A00008494FF47A72B1FBF2F110B501F2D71129
:1078B00006F051FEB0F5296F28BF4FF4296080B261
:1078C00010BD00007D52010010B5114C626892F8A5
:1078D0007820032A04D040F621413220FCF76EFBC9
:1078E000022818BF032805D040F62F414FF0320080
:1078F000FCF764FB002918BF01F0E6FA002061687C
:10790000A1F8C20081F8C40081F8780010BD000021
:107910004C01002001484068C03070474C010020F5
:107920002DE9F041384C616891F84800002816BFF5
:1079300002280020012081F8490001F14A01FDF7E9
:10794000F1F9606890F84810022916BF0329012157
:10795000002180F8851090F8492000F14A034FF08B
:107960000007012A04BF5B7913F0C00F0AD000F1B1
:107970004A03012A04D15A7902F0C002402A01D0F8
:10798000002200E0012280F85C20002A04BF0029C8
:10799000BDE8F08100F1A808FDF752FB1B49A0FBF0
:1079A0000165FAF75DFE80196941C8E90001606868
:1079B00090F8850000281CBF0020FDF761FA002523
:1079C000606890F85D1000291ABF90F85C100029DB
:1079D000BDE8F08190F8491000F14A02012904D174
:1079E000517901F0C001402905D03946BDE8F04188
:1079F0004A3006F021BAFDF7EDF961682A46BDE884
:107A0000F0414A3106F029BA4C01002040420F00F3
:107A1000034810B540688C3008F02CFC002010BDE5
:107A20004C01002070B50846022A0DD0224E0025D8
:107A3000042A71680CD00F2A10D0132A34D040F2D7
:107A4000F3313220FCF7BAFABDE8704001F03EB9DC
:107A5000457007220270496B416070BD0446486D55
:107A60000A69C0F803208A8AA0F80720C87B00288A
:107A70001ABF0228012000204A6D01F10A0190700E
:107A800065704FF0140020704FF0200204F10400E4
:107A900005F030F825727068406D0088FCF7D8FE5C
:107AA000BDE8704005F09DBE457018220270D1F807
:107AB0004210416070BD00004C0100200B4840683E
:107AC000816E002904BF0C20704700F16D01FF2278
:107AD0000A70002282660A7090F86C00012101FA97
:107AE00000F0034908600020704700004C010020AE
:107AF00008F50140024610B50F480C468260C16887
:107B0000A1B142680020A2F8C20082F8C40082F845
:107B1000780001F0AFF9204600F034F8002808BFE3
:107B200010BD40F674113220FCF748FA40F66E1191
:107B30003220FCF743FA00004C01002002490148C2
:107B4000C8607047A08C00004C01002070B504464E
:107B5000FCF77AFF0546FCF771FF0146284605F061
:107B6000B6FE010006D00648C06802682046BDE89F
:107B70007040104740F67B213220FCF71FFA0000CE
:107B80004C01002070B5224D0646686890F87810C8
:107B900001291FBF90F8780000280C2070BDFCF769
:107BA00077FF01F067F96868002490F8840030B12D
:107BB00003F020F802F010FF686880F88440462245
:107BC0000021686805F010F86968012081F85D40BF
:107BD00081F8510081F8584081F8824081F85E6058
:107BE00081F8B040072081F8500001F16D00FF22BC
:107BF000027081F86C408C66047081F8B34081F8A3
:107C0000B440483004700020C1F8B84070BD000096
:107C10004C0100200548406890F84800002816BF35
:107C2000022800200120FDF7ABB800004C01002025
:107C30000178002211F0010F2349496809D04278E8
:107C40000023032A08BF4B6581F85820012281F8E0
:107C5000C620037813F0020F0ED083784FF0000C8B
:107C6000032B08BFC1F854C081F85830022301EB40
:107C7000020C521C8CF8C630037813F0040F0CD0A1
:107C8000C3784FF0000C032B08BFC1F854C081F833
:107C900058300A44082382F8C630027981F8482017
:107CA0004279002A16BF022A0123002381F85130AD
:107CB00081F85920827981F85020C07981F85B00E1
:107CC0004FF00000704700004C0100200148C068E0
:107CD000406800474C01002038B5134C0022606812
:107CE00090F86D108DF800109DF8001031B9816E7C
:107CF00000291CBF90F86C00FAF794FC606800251E
:107D000090F8840030B102F075FF02F065FE606803
:107D100080F884506068A0F8C25080F8C45080F8A1
:107D20007850002038BD00004C0100200948406810
:107D300090F8581003290CBF0121002180F842104F
:107D400004BF416D0988A0F8441013220021383087
:107D5000FDF7E8BC4C0100200248406890F858004C
:107D6000704700004C0100200C48416891F8580011
:107D7000032804D0012818BF022807D004E091F896
:107D80005A00012808BF70470020704791F8590039
:107D9000012814BF03280120F6D170474C010020B0
:107DA0002DE9F0411D4E05460F4670681C4990F8BC
:107DB00082000C5C204603F0E3FD706880F89A4076
:107DC00090F8A410C6300C5C012C08BF25200ED002
:107DD000022C08BF0D200AD0042C14BF082C0F2041
:107DE00005D040F6E1014FF03200FCF7E7F82146FC
:107DF00003F092FD384603F06DFB21464FF0010081
:107E000035B103F091F8002808BFBDE8F08101E02A
:107E100002F0C0FF0120BDE8F08100004C0100200D
:107E2000970301002DE9F84F734C0F460646406852
:107E3000616890464FF0010A072F04BF0028B8F18F
:107E4000000F0AD04FF000098DF80090EB46002893
:107E50007AD0727C012A11D017E081F88AA0D1F87B
:107E6000B800002808BFBDE8F88F08F030FA0028F5
:107E70001CBF606880F88BA0BDE8F88F427902F0E3
:107E8000C002402A08BF012500D00025072F28D1B5
:107E900091F88420002A18BF002D11D0B8F1000FEE
:107EA00004BF91F8C110012915D000BF06F03FF8BA
:107EB0000146606880F8801080F8811080F888A002
:107EC000606890F88010FF2913D00846FDF778F815
:107ED0008DF8000038E00121FDF738F8616881F87D
:107EE0008400606890F88400002818BF002DE7D057
:107EF000DCE796F811C000F180035A4660467168CD
:107F0000FDF7A4F890F0010F1ED0606880F88A9009
:107F100080F88B904FF00002B068002808BFBDE8E1
:107F2000F88F072F18BFBDE8F88F616891F88010AF
:107F3000FF2914BF002ABDE8F88FFDF771F86068CB
:107F400080F889A0BDE8F88F61689DF80000072FD0
:107F500091F8515009D3082F29D8B8F1000F02D059
:107F600091F88A1019B3716819B1002D08BF054640
:107F70001EE0B8F1000F05D1707810F0100F18BF97
:107F8000554615D106F097FF30B1606890F88A0029
:107F9000002818BF012000D10020284305D1FDF79B
:107FA000E1F8002808BF002502D0012500E04D4679
:107FB000606880F88A50114802682AB1414630460C
:107FC0009047616881F88B00706850B16068717C7F
:107FD00080F89B1071680A68C0F894208988A0F81E
:107FE0009810606890F88B10002906BF90F88A00FE
:107FF0000028012290D18DE74C0100205C01002077
:1080000010B50C4803F06AFC0A4C002804BF7F201E
:108010002070606890F8840038B102F0EBFD02F047
:10802000DBFC6168002081F8840002F00BFE052073
:1080300010BD00004C01002010B5054803F04EFCB7
:1080400010B903497F20087002F0FCFD052010BD27
:108050004C01002070B506468AB0144803F03EFC7F
:10806000124D002804BF7F2028703078694600F048
:108070000F042246304600F097FF00222146684652
:10808000FFF7D0FE2146684600F01EF969680446F5
:1080900091F8841039B102F0ADFD02F09DFC6868E2
:1080A000002180F884100AB0204670BD4C010020E9
:1080B00070B501788AB001F00F06324601A900F0D0
:1080C00073FF0298284C0178606890F894209142E0
:1080D00025D1029990F89520497891421FD10299B3
:1080E00090F896208978914219D1029990F89720BA
:1080F000C978914213D1029990F898200979914258
:108100000DD1029990F899204979914207D19DF8B3
:10811000151090F89B00814208BF012500D0002572
:1081200002F090FD104803F0D9FB7F21002808BF22
:108130002170042E10D17DB194F900007F280ED05B
:1081400021700090606890F89A3090F8B02090F814
:10815000811001A806F065FF0AB0052070BD40F24D
:108160001D413220FBF72AFF4C0100202DE9F04190
:10817000544C074600216068032F00F17806A06880
:10818000018002D0052F04D05AE0032106F091F9B6
:1081900056E0052106F08DF9D4E90105416D8969A4
:1081A000C5F80F10416D0A8CA5F8132091F8221024
:1081B0006975406D4169808CFDF7D6F9A875D4E9E1
:1081C0000105406D4169806AFDF7BCF9E875000A58
:1081D0002876D4E90105406D406905F0E2FE687635
:1081E000000AA876D4E90120516D898BC176090A6D
:1081F0000177516DC98B4177090A8177516D1F3025
:10820000A73108F08FF8D4E90105406D95F82410E6
:1082100090F8B20001F0E00100F01F00084385F87B
:10822000240002F079FB072888BF072095F8241066
:10823000E02201F01F0102EA4010084385F8240003
:1082400006F11C01A06806F056F996F82310A06804
:1082500006F058F9606800F14A0590F8496090F816
:108260008510A1B190F858104FF00108032906D1EC
:1082700090F85110002918BF90F8830001D190F8B0
:108280008000FCF735FE00281CBF464605462946FF
:10829000A06806F040F93146A06806F043F9A068EE
:1082A00003F018F9052F18BFBDE8F08160682A684F
:1082B000416DC1F80A20AA88CA81406D4672BDE8A6
:1082C000F08100004C0100202DE9F04FEE4C7F269C
:1082D0000127002594F90030626883B0002967D037
:1082E00001297CD00527022907D006292AD002F0CF
:1082F000A9FC03B03846BDE8F08F054602F0A2FCA9
:10830000606890F88A10C9B190F85810012918BF18
:10831000022913D194F900107F2900F0B081267052
:1083200090F89A2090F88130CDE90032029100F166
:108330004A02FF230221284606F0CFFD03B038464B
:10834000BDE8F08F92F88A1029B192F858100229EE
:1083500007D001291DD002F075FC03B00520BDE84F
:10836000F08F7F2B00F08B81267092F89A1092F894
:1083700081C0CDF800C0CDE90113FF2306214A32A8
:1083800006F0ABFD61680B2081F8B05003B0BDE88A
:10839000F08F7F2B00F07381267092F89A1092F87C
:1083A00081C0CDF800C0CDE90113FF23062139E0DB
:1083B00092F88A10002900F0418192F858100229A1
:1083C00008D0012920D003292ED040F6EC613220BC
:1083D000FBF7F4FD7F2B00F05281267000E05EE099
:1083E00092F89A1092F881C0CDF800C0CDE901133F
:1083F000FF2300214A3206F070FD606880F8B070FB
:1084000003B00B20BDE8F08F7F2B00F03881267081
:1084100092F89A1092F881C0CDF800C0CDE901130E
:10842000FF2300214A32A6E0416892F861C00B7830
:1084300063451FD14B7892F862C063451AD18B789F
:1084400092F863C0634515D1CB7892F864C0634558
:1084500010D10B7992F865C063450BD1497992F838
:108460006630994206D1407C92F86010884208BF7D
:10847000012000D0002092F85A1001297ED0002857
:108480007CD1824890F88310082978D090F8800039
:10849000884273D0D2E003B00520BDE8F08F0546D6
:1084A00092F8850092F88AA0002814BF4FF00009C6
:1084B0004FF001090027A87CA968012807D1487955
:1084C00000F0C000402808BF4FF0010801D04FF075
:1084D000000892F85800032806D192F851000028AD
:1084E00018BF92F8830001D192F880000090FCF749
:1084F000ADFC5FEA000B43D00098FCF79BFC002822
:1085000018BF4FF00109B8F1000F39D05846A968DB
:1085100005F0DBFC0700606890F849B018BF4BF02D
:10852000020B014690F8580003282DD002F08AFB78
:10853000BAF1000FAFD06068AA7C00F14A0190F850
:1085400049C0AB68604605F050FC002808BF002F0A
:1085500077D094F900007F286FD02670616891F879
:108560009A2091F88130CDE90032029001F14A025F
:108570005B460121284606F0B0FC8CE758E05DE040
:10858000606890F849B0CCE7686891F8613002788B
:108590009A4220D1427891F862309A421BD1827877
:1085A00091F863309A4216D1C27891F864309A42B9
:1085B00011D1027991F865309A420CD1407991F845
:1085C0006620904207D1687C91F86020904208BFF5
:1085D0004FF0010801D04FF000082C4C94F88000B7
:1085E000082805D094F88320904208BF012600D0C7
:1085F000002657B9B9F1000F09D091F84900AA7CBB
:108600004A31AB6805F0F1FB08B1012100E000211F
:10861000BAF1000F09D094F85A00012803D020B90C
:1086200058EA060001D0012000E00020014205D0F8
:1086300003B00C20BDE8F08F03E020E002F002FB65
:1086400029E7606890F85910032918BF02297FF4C0
:1086500022AFB8F1000F3FF41EAF94F900107F294C
:108660000DD0267090F89A2090F88130CDE9003234
:108670000291FE2300F14A02012128467BE740F2E5
:108680001D413220FBF79AFC4C010020A807002076
:108690002DE9F0410746FCF7D7F90446FCF7CEF97F
:1086A0000146204605F013F905000ED0324C6068F3
:1086B00090F8580001281CBF022803280AD041F274
:1086C00019514FF03200FBF779FC41F2135132207F
:1086D000FBF774FC6FF0130627B3284605F04FFD37
:1086E00018B9284605F08AFEE0B16168284691F87D
:1086F0007820052A04D241F29D413220FBF75EFC2E
:1087000091F878200B2A04D341F29E413220FBF7E6
:1087100055FCE26891F87810526906EB81015158D6
:1087200088471AE0606890F87810052904D241F271
:1087300009513220FBF742FC90F878100B2904D342
:1087400041F20A513220FBF739FCE16890F87800D9
:10875000896906EB8000085880470F2804D341F24E
:108760002E513220FBF72AFCE168096951F82000FC
:10877000BDE8F041004700004C01002010B518B1E1
:10878000BDE8104000F042B9002908BF10BD1048F4
:10879000416891F878200B2A04D241F2E35132204B
:1087A000FBF70CFC91F878200F2A04D341F2E45136
:1087B0003220FBF703FCC06891F8781080686FF0F6
:1087C0002B0202EB81014058BDE810400047000039
:1087D0004C01002010B5FCF737F90446FCF72EF9E0
:1087E0000146204605F073F850B102F073FE0020F8
:1087F00002F0FEFC05490620496881F8780010BDAA
:108800004FF4C0613220FBF7D9FB00004C0100207F
:10881000104910B5486890F87820062A04D241F231
:1088200011613220FBF7CAFB90F878200B2A04D3A1
:1088300041F212613220FBF7C1FBC96890F8780061
:10884000C9686FF0130202EB80000858BDE81040C1
:10885000004700004C01002010B5064803F03EF828
:1088600010B904497F20087002F0ECF9BDE810400F
:1088700000F0F4B84C010020F8B54B4D04460E460C
:10888000686890F87810002918BF012903D00329DF
:108890001CBF0C20F8BD217B80F8A410A168C16723
:1088A000227B00F1C601515C80F8C1102168C0F83C
:1088B000A010207902281FD002F064FD02F09AF97E
:1088C00002F08AF803F070FB384802F07BFC38486D
:1088D00003F018F8374803F00BF8686890F8700058
:1088E00000280CBF01200220FBF724F9207903287F
:1088F0001CBF304602F0EEFD607B78B16868012253
:1089000090F86D108DF800109DF8001031B9816E4F
:1089100000291CBF90F86C00F9F784FE2079032829
:1089200001D028B11EE040F611213220FBF746FBB2
:108930006A68DFF884C0002092F8501092F8823004
:108940005B1CACFB03746408A4EB8404234482F82E
:10895000823021FA03F313F0010F03D1401CC0B29F
:108960000328EBD3686890F95E0002F0A7FD31465A
:108970000120FFF715FA002808BFF8BD00F000F944
:10898000686890F8510060B1FCF728FA0B4800685D
:1089900003281CBF0020F8BD40F623213220FBF73E
:1089A0000DFBFCF747FCF1E74C010020BC8C0000FC
:1089B00094030100D6BE898EABAAAAAA5015004026
:1089C00038B5114C0022606890F86D108DF80010D9
:1089D0009DF8001031B9816E00291CBF90F86C0021
:1089E000F9F720FE606890F87800002818BF012889
:1089F00007D002281CBF0C2038BD00F02FF8002043
:108A000038BD00F003F8FAE74C01002070B50C4CBB
:108A10000025606890F8840030B102F0EBF801F0B6
:108A2000DBFF606880F884506068012180F878106E
:108A3000A0F8C25080F8C450BDE8704000F05EBBA2
:108A40004C010020044841680020A1F8C20081F8D0
:108A5000C40081F8780070474C0100202DE9F041F6
:108A6000FBF7F2FF0446FBF7E9FF0146204604F05E
:108A70002EFF050037D000F0D5F9334C606800F1C7
:108A8000C60290F8A4108E5C80F8C160002000F04F
:108A9000DBFA00282DD0606890F87800022803D017
:108AA00029460020FFF77CF9012E07BF012703208C
:108AB000002705202844FCF779F96168002581F832
:108AC000840040B1002F18BF402616D001F0C4FF2B
:108AD000304602F09DF8606890F85810032918BFDE
:108AE00002291CD10FE040F2EE414FF03200FBF7BB
:108AF00065FABDE8F041FFF789BF16F00C0F14BF0F
:108B000055265026E2E790F8A41000F1C600085C54
:108B1000012804D100210122084602F071FE60689C
:108B2000FF2180F8801080F8811080F8895080F84B
:108B3000885080F88A5080F88B5080F8B05005211A
:108B400080F87810BDE8F0814C01002010B50320BA
:108B500000F07AFA68B10320FFF708FB0122114602
:108B6000002002F04DFE05490B20496881F878008D
:108B700010BDBDE81040FFF749BF00004C010020C8
:108B80002DE9F0412E4C0021606880F8B01090F87B
:108B90005C10002904BF90F88510002942D000F134
:108BA000A8056FF00042D5E9000181EA02014FF00B
:108BB000010771EA000035D0F9F752FDD5E900232D
:108BC000801A71EB03002DD3606800F1A808FCF750
:108BD00037FA1C49A0FB0165F9F742FD801969418C
:108BE000C8E90001606890F8850000281CBF0120DA
:108BF000FCF746F90121606890F85D20002A1CBF4F
:108C000090F85C20002A0DD090F8493000F14A021B
:108C1000012B04D1527902F0C002402A08D04A3018
:108C200005F00AF96168022081F87800BDE8F0815A
:108C3000FCF7D0F861683A464A3105F00EF9F1E7E1
:108C40004C01002040420F00458A00000D8A0000C0
:108C5000A9EE0000A9EE0000A9EE00005D8A000068
:108C6000A9EE0000A9EE0000A9EE0000A9EE0000A8
:108C7000A9EE00004D8B0000A9EE0000A9EE000057
:108C8000A9EE0000D5870000000000005988000010
:108C9000018000003980000055800000B180000094
:108CA00079880000C1890000848C0000888C000055
:108CB000488C0000988C0000908C00001188000007
:108CC000918600007D870000B3EE00002DE9F04F93
:108CD0008BB00746FBF7B8FE824604F048FD05005E
:108CE00010D001464FF001086A46504604F072FD6C
:108CF0000446FBF7A3FEA04209D040F255113320F1
:108D0000FBF75CF940F24B113320FBF757F901A94F
:108D1000009806F07FFA3C1D284604F0F4FC8346D8
:108D200000F112011C22204603F0E4FE9BF81C0017
:108D30003B4D10F0100F4FF000060FD010F0040F55
:108D400018BF26723CD19DF8142004F11C00049930
:108D500003F0D0FE9DF81400207231E028784FF027
:108D6000010928B99BF82D00252838BF85F8009007
:108D7000287800281ABF9DF804000228267218D00F
:108D8000AB784FF0E50204F11C01009805F053FAAE
:108D90002072A9780844A870009805F044FAA978D0
:108DA000884206D0A07A4FF0000820F06000203002
:108DB000A072A07AC0F34111012918BF2E7015D0FE
:108DC00005207E703870B8F1000F04BF0BB0BDE80D
:108DD000F08F504604F0B2FCE0B10022114650463C
:108DE00004F03BFDAE700BB0BDE8F08F2A78002A8E
:108DF00008BF85F80090E3D00321012A02D0022A9F
:108E000006D0DDE710F0020F1CBF02202870D7D17A
:108E10002970D5E740F295113320FBF7CFF8000019
:108E20006001002010B582B0FBF70EFE01AA694672
:108E300004F0C2FC009804F066FC04461C220021E9
:108E4000123003F0D1FE7F2084F82C00FF2184F83B
:108E50002010E17484F82510207F054920F060007F
:108E60002030207700208860888002B010BD00008C
:108E70006001002010B582B0FBF7E6FD01AA69464B
:108E800004F09AFC009804F03EFC04461C220021E9
:108E9000123003F0A9FE7F2084F82C00FF2184F813
:108EA0002010E17484F82510207F064920F060002E
:108EB000203020770020886008708880487002B0D9
:108EC00010BD0000600100202DE9F04182B0FBF7E9
:108ED000BBFD01AA694604F06FFC009804F013FC86
:108EE000C07F0025002804BF02B0BDE8F0812D4EF0
:108EF000B468BCB1207F20F06000403020777778E4
:108F00002572022200212046FCF70CFC37B1657463
:108F10000222002104F10900FCF704FCFCF73AFFEF
:108F2000B5607570FBF790FD074601AA694604F02D
:108F300043FC009804F0E7FB0446C07F4FF00008B4
:108F400090B1384604F0E1FB38B3B8F1000F07D018
:108F50002046057202220021FCF7E4FBFCF71AFF11
:108F6000B58002B0BDE8F081384604F0CEFB0128A0
:108F700004BF02B0BDE8F081FBF760FD01460122AD
:108F8000384604F068FB002818BF4FF00108D8D11C
:108F900040F256213320FBF711F840F25A213320DA
:108FA000FBF70CF86001002070B516460C4605462C
:108FB00005F0BDF96074284605F0B6F9A074EB1C05
:108FC000DFF880C0981D0021072E34D2DFE806F0BC
:108FD00004131B33273304009CF800206270C4E99B
:108FE00001316A78921F12F0FF02227401D0E06012
:108FF00070BDE16070BD9CF801206270C4E9013071
:109000002174E16070BD9CF802206270C4E90131F6
:109010006A78921F12F0FF022274EAD0E7E79CF808
:1090200003206270C4E901316A78921F12F0FF02D6
:109030002274DED0DBE761706160A1602174E160C1
:1090400070BD00009A03010070B50646F9F708FBF1
:10905000294DA969441AFEF75DFC40780022072ECD
:1090600045D2DFE806F0044242272E42420008289B
:109070000DD004280FD0022813D00821012804BFE6
:109080002A20282310D0DF210520FAF797FF40215E
:1090900014200A4602E0102114202E224FF4A87357
:1090A00002E00421122018231A4411FB002080B290
:1090B000983008E010F00C0018BF282000F5577019
:1090C00001E04FF4FC70A96B0444F4398C4209D3DD
:1090D000002600F0C3FB30B1A86BF438844228BFEF
:1090E000002600D20126304670BD012070BD40F23E
:1090F00093513520FAF762FF8808002010B586B03A
:10910000FCF748FE144C207D98B1607888B90023A4
:109110001A461946684600F00BFC002804BF0120DF
:10912000A07006D0FEF7F6FB00786946F8F7BEFAA5
:1091300068B1207D002804BF06B010BD02F0C6F85B
:10914000F9F7E6F800202075607506B010BD40F60E
:1091500099213520FAF732FF8808002070B568227F
:109160000021134803F040FDFEF7D4FB20210170DD
:1091700010480021016041608160C1600E4841607B
:10918000406841F66A01884204D340F62A413520FE
:10919000FAF714FF00F012F8054D42F21074A01017
:1091A000686006F040F86B3080B2201AA86070BD8D
:1091B00088080020780800206C0100202DE9F04389
:1091C000354F83B03878002818BF00F0E1F801204F
:1091D000DFF8C88088F800006946002004F03DFCF4
:1091E000002804BF00254FF6FF762DD027E0029817
:1091F00000281CBF90F89012002925D00088B042AA
:1092000018BF4FF020093FD0002104F01CFC0400DF
:1092100020D094F89102F8F73BFF84F8905294F82C
:109220009102F8F713FFD0B184F8919204F51C7005
:1092300000F01EFF6946002004F00FFCF8B140F278
:1092400043213520FAF7BAFE6846FBF7F5F8002807
:10925000CDD019E040F244513520FAF7AFFE40F28C
:1092600033513520FAF7AAFE029800281CBF90F867
:109270009012002903D00088B042C5D104E06846AE
:10928000FBF7DAF80028EFD088F80050A7F8645010
:1092900003B00020BDE8F083880800207808002093
:1092A00001494870704700007808002070B50546F5
:1092B0000A484FF47A71B0FBF1F405F0B4FF6B305B
:1092C00080B2204400F1BC01284605F044F9B0F515
:1092D000296F28BF4FF4296080B270BDF9220100C8
:1092E00000291CBF11207047F0B5274C074687B0F6
:1092F000207800281EBF0C2007B0F0BDFEF70AFB47
:109300000646002060700421217084F82E00A4F825
:109310006400054605F087FF6B3081B294F82F207A
:10932000002000BF04EB8003401C9B6805EB010C90
:10933000C0B203EB0C058242F4D20021134825652C
:10934000F8F7BEFF3070202814D03B4600220121E0
:10935000684600F0EDFA90B130786946F8F7A6F962
:1093600000281EBF002007B0F0BD40F29A41352012
:10937000FAF724FE40F297413520FAF71FFE40F23B
:1093800099413520FAF71AFE8808002061950000FF
:109390002DE9F0410026FEF7BDFA3F4C0746207844
:1093A00004281FBF207805280C20BDE8F0814FF06D
:1093B00001006070207D4FF00005B0B1EFF3108820
:1093C00072B6207D00281CBF607D002809D0FEF702
:1093D00083FC207D28B101F079FFF8F799FF25750E
:1093E0006575B8F1000F0ED10CE03878F8F7F8FC8D
:1093F000B7F80300C004C00C05D000210320FEF71D
:1094000063FA00E062B63878F8F742FE94F82C0070
:10941000002820782FD0052804D040F29231352042
:10942000FAF7CCFD206E20B104F1480000F0D6FD23
:1094300003E004F1480000F01BFE657094F82C0076
:10944000002818BF0C26FEF739FBA57084F82C50B5
:10945000A5622078042808BFFFF736FD2570FEF7C7
:1094600059FA04460078F8F7F1FD78B12020207011
:109470003046BDE8F0810528DBD1206E0028D8D128
:10948000A06A00F51C7000F0F3FDD2E740F22B510A
:109490003520FAF793FD0000880800200148007885
:1094A0007047000088080020F0B52C4C83B021786C
:1094B00021B140F251413520FAF780FD002200929F
:1094C000019202920378154613F0010F11466B4684
:1094D00004D0D0E9012101250091294690F800C06F
:1094E0001CF0020F06D0D0E9032C43F821C045F050
:1094F0000205491C90F800C01CF0040F06D0D0E90A
:10950000052043F8210045F00805491C481E84F851
:109510002F001F460026626005F085FE6B3080B28A
:1095200015F0010F03D00099091A0126A16015F06A
:10953000020F06D057F8262004EB8601121A761C7B
:109540008A6015F0080F05D057F8261004EB860244
:10955000081A906003B00020F0BD000088080020C9
:109560002DE9F04F87B00D46FEF7D4F9DFF84092B1
:10957000012607464FF0000809F11004092D80F07C
:109580001281DFE805F00583AAAAA5FCD3FBFA0047
:109590002675607800281CBF07B0BDE8F08F3878CA
:1095A000F7F790FFC4E90601A16C0546401A61680F
:1095B000B0FBF1F0002814BF4FF0010A4FF0000A91
:1095C000CDF8088094F82F00002808BF414626D027
:1095D00005F029FE6B30A16C83B26268681AB0FB9B
:1095E000F2F002FB00F094F82FC008180CF1010C07
:1095F000281A4FF0000104F108020CF0FF0C00BF24
:10960000D2F800B09B44834503D8491CA0EB0B0063
:10961000C9B2121DACF1010C1CF0FF0CF0D184F8A2
:109620002E108DF80C10B7F80300C004C00C0FD03A
:10963000606C009003208DF804008DF80D80684662
:10964000FEF784FAC8B14FF441713520FAF7B6FC41
:10965000BAF1000F14BF8DF804808DF80460A06C7F
:109660006168281AB0FBF1F201FB120000280CBF60
:10967000012000208DF80D00E1E7A06BE338C9F868
:109680000C00F8F715FF07B0BDE8F08F607890B1D7
:10969000FEF722FB207D002804BF07B0BDE8F08F55
:1096A00001F014FEF8F734FE84F8148084F8158075
:1096B00007B0BDE8F08F6675FEF708FB002804BF11
:1096C00007B0BDE8F08F40F217313520FAF776FC8D
:1096D00007B0BDE8F04F02F059B93D78FEF71AF92E
:1096E000B0F80300C004C00C05D001210320FEF730
:1096F000EBF8FCF74FFB002301221946684600F007
:1097000017F968B128466946F7F7D0FF00281CBF53
:1097100007B0BDE8F08F40F6B5213520FAF74EFCD2
:10972000A67000F047F807B0BDE8F08FB7F8030067
:10973000C004C00C1DD0787810F00C0F24D094F821
:10974000400008BB84F84060012144F23650F7F72E
:109750008FFDC8B9A16B44F236500144A163D9F81A
:109760000C100844C9F80C0007B0BDE8F04FF8F73A
:109770009FBE00F073F8002802E00FE009E012E05D
:109780001CBF07B0BDE8F08F07B0BDE8F04F05F093
:1097900089BB07B0BDE8F04F00F00CB840F249318A
:1097A0003520FAF70BFC40F24D313520FAF706FC74
:1097B0007808002070B5284C207870B194F82C10EF
:1097C000204600250029006E21781BD0052909D0EC
:1097D00040F292313520FAF7F1FB40F2B721352003
:1097E000FAF7ECFB20B104F1480000F0F7FB03E0CE
:1097F00004F1480000F03CFCA07888B194F82C00FB
:1098000050B10DE0052908BF0028F1D1A06A00F58C
:109810001C7000F02DFCEBE7FEF788FAFCF7BAFAB3
:10982000FEF74CF9A57084F82C50A5622078042826
:1098300008BFFFF749FB2570FEF76CF80446007877
:10984000F8F704FC00281EBF2020207070BD40F2F5
:109850002B513520FAF7B2FB880800202DE9F041A2
:10986000F8F7FEFE304C05460F462178A069042922
:1098700009D16168A26C01EB81014900801A88421C
:1098800038BF022600D301263046F7F7CFFD652802
:109890003AD3B0F1FF3F08BFE06B21D0D4F838C015
:1098A000E26B0CEB00018A4298BFA2EB0C00B5F111
:1098B0003A0147F1FF330246D4E90C07411A67EB3E
:1098C00003000027B8463B467F1A78EB000705DA0D
:1098D000571A73EB0007A8BF0A4613460CEB0300A8
:1098E000A16B471A41F28830874288BF41F288371E
:1098F000F8F7B6FE401B00F19D00874204D33146C5
:109900003846F7F7B5FC10B10020BDE8F081A06B38
:1099100006493844A063C8683844C860F8F7C8FDF1
:109920000120BDE8F08100008808002078080020B0
:109930002DE9FF4F95B090468146FDF7EBFF0B9068
:10994000F8F78EFE4FF0000AFA4E05918DF824A02C
:1099500007465546B46805F066FC6B3081B296F850
:109960002F20002006EB8003401C9B6805EB010CB8
:10997000C0B203EB0C058242F4D2EE484068854247
:109980000CBF0121002118EA010F139108D0E94909
:109990000A78002A1ABFB1F864100029012101D009
:1099A0004FF000011291169900297DD0059917F505
:1099B000FA6041F10008029000F004FB00F08EFB19
:1099C0000646DC480078052840D1DA4DA86AD0F870
:1099D000780200F069FB0090B0421DD0A86A00999F
:1099E00000F51C7000F01EFB00212966D5F828B098
:1099F000009DBBF1000F1CD02DB300F0DDFAE8B1E3
:109A0000D5E901102A68121841EB0A00CBE99C2025
:109A1000A88BABF88C0219E0A96A01F51C712966C4
:109A2000A96A286DD1F87812884238BF084628659F
:109A3000DCE74FF4B9613520FAF7C0FA40F2CE51B5
:109A40003520FAF7BBFA0020CBE99C00B94D31462E
:109A500005F1480000F0E6FA002E1CBFB08BA5F817
:109A60006400AB466D68029A08BF002011D0D6E9A9
:109A700001103368CDE90028181841EB0A012A4685
:109A800005F0F2FBA84204D940F2E6513520FAF77E
:109A900095FA054600F09CFA029958464E1948EB93
:109AA0000A08DBF8041000E01DE0721A68EB0A01F6
:109AB000C0E91221189979B1084642F21071484361
:109AC0000BF13002301848EB0A01C2E9000100BF77
:109AD0004FF0010B00F09AB94FF0FF3251080263CA
:109AE000CBF83410F4E71299002971D0DFF84482E2
:109AF0000B98059E98F82E10801D095C082908D047
:109B000004290AD002290ED00822012911D000F020
:109B10008BB940221420134602E0102214202E2379
:109B20004FF4A87C09E00422122053464FF0180C91
:109B300003E02A2053464FF0280C634412FB003008
:109B400085B2084601F00EFD4AF2A13101444FF4FE
:109B50007A70B1FBF0F0284400F1F40508F1300010
:109B60006FF00042D0E90010504070EA010028D0A8
:109B70008DF830A00D9505F056FBADF838000120AA
:109B80008DF83B0005F04FFB00F5817080B2C019E5
:109B90004AEB0601CDE9100102208DF83A000CA82D
:109BA000F7F778FF0246DDE91001D8E90C3C4019CF
:109BB00041EB0A01181A6CEB01000AB1002800DA27
:109BC00000243E46D346DDF8148000F01FB9FFE7BD
:109BD000B8F1000F59D0574DD5E912137A1AB2FBDC
:109BE000F0F200FB02F2891843EB0A020E1842EB76
:109BF0000A000390B6EB070805F015FB00F581702D
:109C000080B2804511DAAA6C286A6968801AB0FBB4
:109C1000F1F001FB00F01018301AB0FBF1FB084620
:109C2000039980194AEB01012CE08DF830A0E86B14
:109C30000D9005F0F8FAADF8380001208DF83B00E2
:109C4000D5E91202296A0B1A6968B3FBF1F301FB2B
:109C500003F3C31842EB0A02CDE910322A78042A32
:109C600007D101EB81025200181A904238BF02203E
:109C700000D301208DF83A000CA804F0D3F98346F4
:109C8000DDE9100106468846C0E02A4A09A9039189
:109C9000D2E912127B1AB3FBF0F300FB03F00818B1
:109CA00042EB0A010C9106903C1AFDF733FE834605
:109CB00005F0B9FA00F5817080B2251800262C460F
:109CC00005F0B1FA6B301FFA80F81A484068A042DC
:109CD00098BF241A174B93F82F00002818BF03F1E0
:109CE00008010AD00A684244A24202D8A41A721C8F
:109CF000D6B2401E01F10401F4D10E4800EB8600FB
:109D00000F9080680D900BEB06008079082807D033
:109D1000042809D002280FD00822012812D083E09D
:109D200040221421134602E0102214212E234FF466
:109D3000A87C0BE0880800200422122153464FF033
:109D4000180C03E02A2153464FF0280C634412FB01
:109D500001311FFA81FB01F005FC4AF2A1310144F7
:109D60004FF47A70B1FBF0F00BEB000108190D997C
:109D7000F430884203D80F988068041B11E08C49A6
:109D800091F82F00B04218D9701CC6B24868A8429A
:109D90000ED901EB8600806800EB080501EB860018
:109DA0008468002C19DA40F20C713520FAF706F9B4
:109DB00040F2E6613520FAF701F948682A46854203
:109DC00038BF0546EAD3B2EB400F38BF4500E5D3B4
:109DD00040F203713520FAF7F1F80398744B0670DE
:109DE00006990C984E1940EB0A08D3E9120C9969B0
:109DF0005D68091AB1FBF5F101FB05F140184CEB68
:109E00000A01C3E91201301AB0FBF5FB9DF82410DA
:109E10000B980844807908280AD004280CD002281E
:109E200010D00823012813D0DF210520FAF7C6F847
:109E3000402314211A4602E0102314212E224FF44D
:109E4000A87C09E00423122152464FF0180C03E0CD
:109E50002A2152464FF0280C624413FB01218DB297
:109E600001F080FB4AF2A13101444FF47A70B1FB5A
:109E7000F0F028444E49F4300690D1E90C02801BE2
:109E800062EB080500221346121A73EB0502A8BF05
:109E9000504605DA221A7AEB0502A8BF044620468E
:109EA0009DF8242001EB82029268824298BF1046FE
:109EB0000C46C863129830BBBBF1000F23D04FF69D
:109EC000FF7000EA4B01B4F9640004F04FFBB4F8F2
:109ED0006410091A0AB2A4F86420A16A41B1A1F879
:109EE0008C22D1E99C23121843EBE073C1E99C2337
:109EF000D4E912234FEAE071361848EB0108101834
:109F00005941C4E912011698002818BFC4E906682F
:109F1000C4E908681398002814BF0698E06B01256F
:109F2000A06389F80B5005F07EF9A9F808002078A5
:109F3000042809D16068A26C00EB80004100B01ACF
:109F4000884238BF022000D3012089F80A00A06BA4
:109F5000C9F804001298002804BF89F800A0C9E9D4
:109F600004681BD089F80050D4E90C020599C01B85
:109F700062EB010B00210A46091A72EB0B0108DAA9
:109F80000C490022091A72EB0B01ACBF8246DFF8C4
:109F900024A00698AAEB0000C9F81000E16B06980F
:109FA00081422CBF0120002019B0BDE8F08F0000D5
:109FB000880800200040420F0148007970470000E7
:109FC00074010020014901200871704774010020CC
:109FD00001490020087170477401002010B58169A3
:109FE00019B182688B689A4203D2C7213720F9F7EA
:109FF000E5FF42694A6103690B61002A12BF1161E2
:10A00000074A11600A69002A08BF002005D0516183
:10A01000D0E9022010448A68801AC86010BD000090
:10A020007401002010B500234161C1B10A690861C3
:10A030000261002A18BF50614169C360002908BF4E
:10A0400010BDCA687AB1D0F808C0624524BFA2EB3F
:10A050000C02C26007D22A213720F9F7AFFF03496B
:10A0600003610860E8E7CB6010BD000074010020C8
:10A07000416949B1D0E902231A44CB681A44CA6045
:10A08000D0E90412116102E0064A01691160016918
:10A09000406900291CBF4861704700281CBF00218F
:10A0A000C1607047740100200B4984460020096894
:10A0B0000246431E69B1CA68624528BF934284BF05
:10A0C000134608460A4609690029F4D1002818BF3A
:10A0D0007047104670470000740100200548016871
:10A0E0000020002908BF7047084609690029FBD1F4
:10A0F00070470000740100200248002101604160A7
:10A100007047000074010020044900200A68002AFA
:10A1100012BF0C2000224A6070470000740100202A
:10A1200003494A8802800978817000207047000046
:10A13000BC0F00202DE9FC410E460546077805F0CE
:10A14000E0FD00280AD1284605F0A1FD002805D130
:10A150000220FAF709F9874202D30720BDE8FC8103
:10A160000221384603F06FFC040003D004F087FDA1
:10A1700070BB0CE000220221384603F05AFC0400B8
:10A1800011D0264890F90010204604F032FA2878C1
:10A19000032103F058FCE8B190F84800D0B168788A
:10A1A000C1070BD104E041F25A213920F9F706FF2B
:10A1B000810703D4C10601D4800601D51220CDE762
:10A1C000204604F060FB05F0F7FCA97D884201D031
:10A1D0000C20C3E7204604F042FB3070E8742946A7
:10A1E0002046FBF795FF0646687EA0B19EB9002287
:10A1F0006846616C03F0FBFC00220121606C03F0F7
:10A200006FFD04226846616C03F0F1FC00221146E8
:10A21000606C03F065FD3046A0E700007C01002083
:10A22000017871B1417861B141881B2909D38188D6
:10A230001B2906D3044902680A60808888800020B0
:10A240007047122070470000BC0F00200068B0F576
:10A250007A7F03D30249886000207047122070473C
:10A26000BC0F00207CB50546007898B16846F9F728
:10A2700013FD9DF8000008B1012400E0002401A8AE
:10A28000F9F7F2FC9DF8040000B10120044301D06D
:10A290000C207CBD02492878087200207CBD00009B
:10A2A0008E100020014890F9000070477C010020CA
:10A2B000034AD2E9001201604260002070470000AA
:10A2C000BCA7000070B5044600780025012804D022
:10A2D00018B1022801D0032868D1607828B101287C
:10A2E00003D0022801D0032860D1607E10B9A07885
:10A2F00001285BD1A078C10858D1810704D5022874
:10A3000054D12C49497AE9B340074FD000F0D4FA30
:10A310000146A07830EA010101D0112070BDC007CC
:10A3200006D0E07801232269A16805F0A7FD054663
:10A33000A078800706D5E07802232269A16805F09D
:10A340009DFD0543A078400706D5E07804232269E7
:10A35000A16805F093FD05430DB1284670BDA078B6
:10A3600005281FD1D4E9031520790423626905F07B
:10A3700085FD0028F2D1012004EB80010A69154413
:10A38000221800E012E0D378927893420ED18A68C6
:10A3900049688A420AD1401CC0B20228ECD3A068A6
:10A3A000A84203D3207E08B1072801D9122070BD2E
:10A3B000002070BD8E1000202DE9F0411D46DDE922
:10A3C0000647A1F1060C40F67A43089E9C4505D845
:10A3D000A2F1060C9C4501D8012300E0002320B126
:10A3E00090F8770068B16BB902E01548007AF9E798
:10A3F000A1F60150062821D8A2F60150062801D95D
:10A400001CE0DBB1914219D8B5F5FA7F16D2A4F160
:10A410000A0040F67641884210D8104603F0B5FD98
:10A420006D1C684340F2712140004C43B0EB041FA7
:10A4300004D2B74202D80120BDE8F0810020FBE73A
:10A440008E10002010B512484FF6FF71114A01839B
:10A450000021817681831B2313804FF4A4745480E0
:10A460009380D4808174C1745172032404700224D7
:10A4700044704380838040F6A66383605B00C360C2
:10A48000117280F82810817501740348017010BDA5
:10A49000BC0F00208E1000208401002030B587B052
:10A4A00005460888ADF8040013480C4603AB817CD0
:10A4B0008DF80610C17C8DF80710808AADF8080071
:10A4C00004A8009001AA2146284605F03BFD05009E
:10A4D00010D19DF80C008DF814009DF810008DF837
:10A4E0001500BDF80800ADF8160005A9204603F0D8
:10A4F00095FD284607B030BDBC0F00200449A0F6EA
:10A50000C410884201D3002070470120704700002A
:10A51000CCF370020449A0F6C410884201D3002095
:10A5200070470120704700003D369C000449A0F6AA
:10A53000C410884201D300207047012070470000FA
:10A540003D369C0010B50221002003F07CFA040087
:10A550000CD100220221104603F06BFA040007D050
:10A56000064890F90010204604F043F8204610BD3C
:10A5700040F235213920F9F721FD00007C0100204F
:10A5800030B50022074D09E050F822402B469C428E
:10A5900000D8234640F82230521CD2B28A42F3D36C
:10A5A00030BD00000024F4000449A0F57A70884210
:10A5B00001D300207047012070470000A8F9700205
:10A5C0000449A0F57A70884201D300207047012029
:10A5D00070470000A8F97002094A90420BD801297F
:10A5E00002D0042903D008E040F2537101E040F6A4
:10A5F000C411884201D2002070470120704700003A
:10A600008FFD70022DE9FC410C46064604F02AF944
:10A6100098B1304604F017F930B1B4F801101220A7
:10A6200000290BD0802909D8304604F0D1F838B180
:10A63000304603F0A6FF28B109E04220BDE8FC81C6
:10A640000C20FBE7304604F0F0F800285BD03046E1
:10A6500004F015FB0028F3D1304603F0AFFF0028CB
:10A66000EED13046FBF736FCB4F8010042F210712F
:10A6700000FB01F8E178304604F0A1F820780321CE
:10A6800003F0E1F938B14949096821B190F848204F
:10A690000AB138308847304604F0CBF848B130462C
:10A6A00004F0D1F8424F80B1304604F0D0F850B1F8
:10A6B0000BE0424600213046FCF76EFF0028BDD07B
:10A6C00041F27B4165E0387AE8B10022012101A81E
:10A6D000F9F7D8FE040046D00021FAF7D3FEBDF802
:10A6E000040020802146304604F0CFF800F0DEF868
:10A6F000400940EAC160C0072E4D04F1340004D087
:10A700006A88A98803E0122098E71B221146C284B8
:10A710000185387A00B1012005F1200184F8770025
:10A720000EC904F1800787E80E00A968616310B1C3
:10A730004FF47A7701E041F64C57304604F087F841
:10A7400010B9304604F09FF8214601206761FFF7F9
:10A75000A5FE50B10121BDF80400F9F7DFFE10B1EC
:10A7600041F2CB4115E0092068E7687800902B782A
:10A77000AA8869882088F9F7B7FF10B141F2D6415D
:10A7800007E0424621463046FCF706FF20B141F281
:10A79000D8413920F9F712FC0748436823B1002259
:10A7A00004F59D7120469847002047E78C01002062
:10A7B0008E100020BC0F00207C0100200CD8110C52
:10A7C0005900D81110B50C46FBF7B6FA054844609D
:10A7D000806805F02EFD05F02EF9BDE81040FBF76E
:10A7E0002BBB00009001002001480078704700005A
:10A7F000900100200149087070470000900100207E
:10A8000010B5054CE06805F014FD206905F011FD58
:10A81000BDE8104005F0A7B99001002010B505492A
:10A82000054805F0F9FC0448BDE810400349001D47
:10A8300005F0F2BCA401002098010020AC0100202A
:10A8400010B50549054805F0E7FC0448BDE810408F
:10A850000349001D05F0E0BCB40100209801002070
:10A86000BC010020014840787047000090010020A2
:10A8700010B5FCF773FF0348FBF798FDBDE81040E7
:10A88000FBF78EBAD312002010B5FFF735FCFEF7A8
:10A8900065FCFFF707FD01460348FDF72BF9BDE80E
:10A8A0001040FBF785BA0000D31200200149D1E91E
:10A8B0000001704720000020094908880979C20A70
:10A8C000000A42EA415240EA0160D20700F001006A
:10A8D000001840EA5272D0B240F001007047000008
:10A8E0002000002010B5F8F793FE0022084B114617
:10A8F00033F82140844203D303EB8100827803E0E4
:10A90000491CC9B20C29F3D30248027010BD0000E3
:10A91000960201001C0200200148007870470000E8
:10A920001C0200202DE9F84F0F46054615219046E0
:10A930000E46FF2002F0BDFF4FF6FC71C01C00EA7E
:10A9400001040DB3DFF84C9004FB0753C9E9015330
:10A95000A9F80040FA000021184602F045F9002548
:10A96000AA460FE0284600F017F82146FF2233469A
:10A97000CDF8008002F03BFFD9F8081001F835A0AF
:10A980006D1CADB2BD42EDD3083404FB07F0BDE849
:10A99000F88F0000C401002002494A68098800FBC2
:10A9A00001207047C401002070B5054616460C46CC
:10A9B000022000F0F1F80549012008700449F01E5A
:10A9C000086004480560001F046070BD1D0200207F
:10A9D00010F5004008F5004010480178A9B1104A70
:10A9E0004FF4000111600F49D1F800310022002B13
:10A9F0001CBFD1F80431002B02D0D1F8081141B1AD
:10AA000042704FF01001817002704FF0000000F0B2
:10AA1000C3B80121417004490968F4E71D02002010
:10AA200008F5014000F0004000F4004010B502209D
:10AA300000F0B2F806480122002102700548C0F873
:10AA40000011C0F80411C0F80811026010BD000028
:10AA50001D02002000F0004010B5022000F09CF81C
:10AA600007490120087007490020C1F80001C1F81A
:10AA70000401C1F8080104494FF40000086010BD4A
:10AA80001D02002000F0004004F5014003480021B1
:10AA90000170417010218170704700001D0200207C
:10AAA0000C480178002904BF807870470A48D0F824
:10AAB000001100291CBFD0F80411002902D0D0F8E1
:10AAC000080110B14FF01000704704480068C0B290
:10AAD000704700001D02002000F0004000F400401C
:10AAE000114810B50278114B4078C821491EC9B2EF
:10AAF0005AB1D3F800C1BCF1000F0CD0D3F8040157
:10AB000038B1D3F8080160B103E0022803D001286E
:10AB100007D0002010BD0029E8D19E213B20F9F785
:10AB20004DFA012010BD00001D02002000F0004081
:10AB3000054900200A781AB1054B044A1A600870CA
:10AB40004870887070470000200200200000020258
:10AB500008F5014002480021017041708170704782
:10AB60002002002010B54FF0E0224FF400410020F9
:10AB7000C2F88011BFF34F8FBFF36F8F0449086095
:10AB80000860FFF7D5FF03494FF40000086010BDCF
:10AB900000F5004008F5014070B5114C0546002055
:10ABA00020602060FFF7C4FF0E494FF400000860EA
:10ABB000002D08BF70BD0C480C49012D04BF0222B6
:10ABC00022600BD0022D03D081213D20F9F7F6F948
:10ABD00003222260086006494FF40000086070BD3F
:10ABE00000F5004008F50140D513002014F50040A1
:10ABF00004F501400548D0F8001221F04001C0F8EA
:10AC000000120021C0F860157047000000100040DD
:10AC10000449C1F86005D1F8000240F04000C1F8D5
:10AC20000002704700100040014890F82A00704769
:10AC3000181000200249085C00F5166070470000FB
:10AC400028C200002DE9F84FF8F758FFF8F7CCFFBD
:10AC50004A4C8046D4F8040310F0100F14BF4FF094
:10AC600001094FF000091020C4F808030220C4F8BD
:10AC70000002434DDFF80CA1002685F834604FF444
:10AC80006020CAF80000D4F850054FF0010710F01A
:10AC9000FF0F16D0FF208DF80000C4F81061276167
:10ACA00005E000BF9DF80000401E8DF800009DF8F3
:10ACB000001019B1D4F810010028F3D09DF800005D
:10ACC00040B1A88B962824D3687A012807D002289F
:10ACD00012D01EE040F683013E20F9F76FF9F8F735
:10ACE000C9FF002818BFB0F1FF3F12D040F6940111
:10ACF0004FF03E00F9F762F9F8F7AAFF002818BFF5
:10AD0000B0F1FF3F05D040F69A014FF03E00F9F751
:10AD100055F9C4F81061002001F04CF9EE712E7263
:10AD20006E7295F84400B0B1D4F8000220F480109F
:10AD300040F00200C4F800024FF48020CAF800007E
:10AD40006869114920F003006861086010490F48E4
:10AD5000086085F84460B9F1000F1CBF1020C4F8EA
:10AD60000403B8F1000F18BF276195F845000028CB
:10AD70001CBF276185F84560BDE8F88F00100040D2
:10AD80001810002008F50140001900408032020030
:10AD9000101900402DE9F0475C4C054686B094F848
:10ADA00034008A4610F0010F16D0DFF864814FF0AE
:10ADB0000209002DD8F80000059004BF04208DF88A
:10ADC00014000ED0012D08BF8DF8149009D040F664
:10ADD000B9213E20F9F7F2F84FF4ED613E20F9F782
:10ADE000EDF805A8F8F75AFE20B140F6BD213E2047
:10ADF000F9F7E4F8474FD7F8000240F00100C7F830
:10AE0000000294F83400012640F0020084F8340077
:10AE100015B1012D06D00BE0504601F08BF966729A
:10AE20003E6005E0504601F001F984F809907E602B
:10AE30003948C6643948D0F84005A18B96292ED3ED
:10AE4000374935B1012D17D040F24C713E20F9F74A
:10AE5000B5F800F12802C1E9020232493048F8F79A
:10AE60000FFF002818BFB0F1FF3F18D040F23B7130
:10AE70004FF03E00F9F7A2F800F12902C1E9020201
:10AE800028492748F8F7EAFE002818BFB0F1FF3F2D
:10AE900005D04FF4E9614FF03E00F9F78FF808F163
:10AEA0008C00012D0FC88DE80F00D8F89C0004908D
:10AEB00014BF012000208DF801006846F8F778FEE5
:10AEC00005A8F8F7D9FD20B140F6CF213E20F9F7CB
:10AED00075F8607A012807D0022804BF9DF8140095
:10AEE00010F0020F10D004E09DF8140010F0040FD1
:10AEF0000AD04FF0000000BF84F84500002818BFBA
:10AF00003E6106B0BDE8F0870120F5E7181000208B
:10AF100000C2000000100040008000400C80004093
:10AF2000D801002050C200002DE9F04F9B4C0500D5
:10AF3000DFF86C9294F8340089B040F0020084F895
:10AF40003400D9F800000F464FF0020A009004BF09
:10AF500004208DF8000009D0012D08BF8DF800A055
:10AF600004D040F6B9213E20F9F728F86846F8F7F2
:10AF700095FD20B140F6BD213E20F9F71FF8DFF81E
:10AF800024B2894E4FF0000815B1012D20D037E0D2
:10AF9000384601F0CFF801206072E079012805D130
:10AFA000D6F8000240F00800C6F80002206B40F41A
:10AFB000801020634FF48010CBF800007B4830F8FD
:10AFC000170000F5FA714FF47A70B1FBF0F817E052
:10AFD000384601F02BF884F809A0E079012805D162
:10AFE000D6F8000240F00400C6F80002206B40F4DE
:10AFF000001020634FF40010CBF800004FF0290838
:10B00000E079002804BF94F8340040F0020006D034
:10B01000012804BF94F8340040F0040001D184F802
:10B02000340094F83400DFF888A110F0010F29D023
:10B0300010F0020F16D0D6F8000240F00100C6F85A
:10B040000002D6F85005C0B20B2818BF0A2803D05A
:10B05000032818BF022815D140F217614FF03E00B7
:10B06000F8F7ACFF10F0040F0CD053495148C1F869
:10B070001405DAF8400128B140F21F614FF03E009C
:10B08000F8F79CFF01F0C6FB28B1FFF7DBFD09B024
:10B090000020BDE8F08F012D08BF49F6BA7104D039
:10B0A000424830F8170000F516714FF47A70B1FB82
:10B0B000F0F701F0C1FB0AEB8001D1F8401509F16E
:10B0C000A0020DF1080B92E80C148BE80C14D9F8CF
:10B0D000B0200692012D14BF012200228DF8092014
:10B0E000CDE90401069702A8F8F762FDA08B0021C4
:10B0F00096282CD3314835B1012D16D040F24C7131
:10B100003E20F8F75BFF2822C0E902122C492B48A9
:10B11000F8F7B6FD002818BFB0F1FF3F17D040F296
:10B120003B714FF03E00F8F749FF2922C0E90212B7
:10B1300023492248F8F792FD002818BFB0F1FF3FDD
:10B1400005D04FF4E9614FF03E00F8F737FF01A852
:10B15000F8F792FC20B140F6CF213E20F8F72EFF01
:10B16000607A012807D0022804BF9DF8040010F07F
:10B17000020F11D004E09DF8040010F0040F0BD072
:10B180004FF0000084F8450000281CBF012030610A
:10B19000404609B0BDE8F08F0120F3E71810002009
:10B1A00000C2000004F501400010004016C200007B
:10B1B000008000400810004098F00140D8010020B5
:10B1C00050C2000010B504460748F8F75BFC20B1F8
:10B1D00040F607113E20F8F7F1FE94E80E10034800
:10B1E00080E80E1010BD0000FDBF00000810002018
:10B1F00010B50F4C03460220207394F829C0A08B91
:10B2000094F82810227EBCF1010F0DD001F0B6F8A1
:10B21000206108480021C0F844112169606A08448F
:10B220000549C1F8400510BD01F0C6F8F0E700007F
:10B230001810002000800040048000402DE9F041FB
:10B24000482200211D4801F0CFFC1C480024FF21AA
:10B25000C4710472447280F837105F2180F838108E
:10B2600001F0DDFB164F174D174E28B901F0EEFB2C
:10B2700010B901F0F5FB40B12422FF21384601F05E
:10B28000B3FC2C603460BDE8F08101F029FC10B9FA
:10B2900001F01CFC40B14022FF21384601F0A4FC23
:10B2A0002C603460BDE8F0813822FF21384601F07F
:10B2B0009BFC2C603460BDE8F08100001810002079
:10B2C000000E0040080E0040100E00402DE9F04135
:10B2D000294E284C0020C6F84005271DC7F8400518
:10B2E000C4F8400506F10408C8F84005FFF7AAFCB9
:10B2F000224DA88B96280CD3F8F7A4FC002818BF81
:10B30000B0F1FF3F05D040F246514FF03E00F8F754
:10B3100055FEF8F7BDFB20B140F25A513E20F8F738
:10B320004DFE286B164940F04460086000202863F9
:10B33000287368622862C6F84005C7F84005C4F85B
:10B340004005C8F84005C4F84801C4F84401C4F8F1
:10B350004001C4F84C014FF0E0210220C1F8800107
:10B3600001F5C071BFF34F8FBFF36F8FC1F80001BC
:10B37000BDE8F081008000400880004018100020E7
:10B3800008F501402DE9F0474FF0E02801274FF084
:10B3900002090025C8F88091BFF34F8FBFF36F8F6C
:10B3A000394CC4F8FC5FC4F8FC7F01F06FFB374EEA
:10B3B00018B1306840F48060306001F05BFB38B158
:10B3C000306820F0690040F0960040F000403060A6
:10B3D00001F06CFB30B12E48016821F47F4141F44B
:10B3E000B05101602C492B480860F8F761FC40B16E
:10B3F0004FF08050D0F83003B0F1FF3F1CBF274919
:10B4000008604FF01020006EB0F1FF3F04D02449D7
:10B410000A6860F317420A6040F2031140F25B6071
:10B42000C4F83415C4F838051E4807601E481F4A82
:10B4300003210776116040F20121C4F85016022161
:10B44000C4F800121A4A4FF040611160A0F11001D7
:10B4500096220D871749456280F834500D7082831B
:10B46000154A1268426180F84450C8F88092102052
:10B47000C4F80403C8F800914868002808BFBDE874
:10B48000F087BDE8F0470047001000403C1700403F
:10B49000401700402C000089781700404C170040EE
:10B4A0008C15004030150040181000201015004089
:10B4B00004F50140D0010020001900400149487600
:10B4C0007047000018100020014951F82000704713
:10B4D000DCC200001E4910B5C1F804051D4A92F8EF
:10B4E000340040F0010082F8340010F0010F08BF72
:10B4F00010BD10F0020F16D0D1F8000240F001008C
:10B50000C1F80002D1F85005C0B20B2818BF0A28B4
:10B5100003D003281CBF022810BD40F217614FF072
:10B520003E00F8F74BFD10F0040F08BF10BD0A48AD
:10B530000A49C1F814050A48D0F84001002808BF9C
:10B5400010BD40F21F614FF03E00F8F737FD0000DC
:10B5500000100040181000200810004098F0014032
:10B5600000800040014951F82000704700C30000EE
:10B570002DE9F04F0600954889B0904600680D46C9
:10B58000009008BF042008D0012E08BF022004D07C
:10B5900040F6B9213E20F8F711FD8DF8000068460D
:10B5A000F8F77CFA20B140F6BD213E20F8F706FD01
:10B5B000DFF81C92874F884C4FF47A7B4FF0010ADA
:10B5C00036B1012E1AD040F614013E20F8F7F6FCF1
:10B5D000404600F0AFFD814884F809A030F818100B
:10B5E000E079012804D001F5FA71B1FBFBF16D1A85
:10B5F000002804BF3846C9F8147511E0404600F031
:10B6000015FD02206072E179012904D04AF2AE10E2
:10B61000B0FBFBF02D1A7248002908BFC9F81405C9
:10B620007049C1F840557048C9F810051020C7F896
:10B630000403206B6D4A40F4002020630801106071
:10B64000E079002804BF94F8340040F0020006D0EE
:10B65000012804BF94F8340040F0040001D184F8BC
:10B66000340094F8340010F0010F28D010F0020FCD
:10B6700016D0D7F8000240F00100C7F80002D7F852
:10B680005005C0B20B2818BF0A2803D0032818BFE2
:10B69000022814D140F217614FF03E00F8F78EFCFB
:10B6A00010F0040F0BD05248C9F81405D1F840012E
:10B6B00028B140F21F614FF03E00F8F77FFCC1F85F
:10B6C0004CA04C48D0F84005A84204D340F62A01CB
:10B6D0003E20F8F773FC012E0FBF49F6BA703F48C1
:10B6E00030F8180000F51670B0FBFBF037490DF18B
:10B6F000040901F1B40292E80C1189E80C11D1F8A7
:10B70000C410059114BF012100218DF80510CDE969
:10B71000045001A8F8F74CFAA08B96282ED336488F
:10B7200036B1012E17D040F24C713E20F8F746FC9E
:10B7300005F12801C0E9025130492F48F8F7A0FA75
:10B74000002818BFB0F1FF3F18D040F23B714FF016
:10B750003E00F8F733FC05F12901C0E90251274901
:10B760002548F8F77BFA002818BFB0F1FF3F05D055
:10B770004FF4E9614FF03E00F8F720FC6846F8F717
:10B780007BF920B140F6CF213E20F8F717FC607A14
:10B79000012807D0022804BF9DF8000010F0020F16
:10B7A00011D004E09DF8000010F0040F0BD04FF012
:10B7B000000000BF84F84500002818BFC7F810A09B
:10B7C00009B0BDE8F08F0120F4E7000000C20000DE
:10B7D00098F00140001000401810002016C2000030
:10B7E00004100040008000404081004004F501400A
:10B7F000081000400C800040D801002050C200001A
:10B8000030B5314C87B00D00E071A2720CBF012041
:10B8100002202072012806D0022826D040F63D21C1
:10B820003E20F8F7CBFB607A02281ED1104694F92F
:10B830001920A17E05AB00F01FFE9DF9140000F059
:10B84000DDFD0DF11500F8F721FA20B140F2EE51BF
:10B850003E20F8F7B3FBFF2084F837001B48D0F8F0
:10B86000001241F48871C0F80012627A207E022A28
:10B87000A28B4FF47A711DD0154B33F8100000F2F3
:10B88000E730B0FBF1F010441249012D01F1C8027C
:10B8900092E81C108DE81C10D1F8D810049114BF48
:10B8A000012100218DF8011001906846F8F780F918
:10B8B00007B030BD084B53F8200000F2E730B0FB72
:10B8C000F1F0101AE0E7000018100020001000400E
:10B8D00004C2000000C2000000C300000349096860
:10B8E00001F07F0149420170012070474815004076
:10B8F0000349020EC1F824250002C1F81C05704757
:10B90000001000400068034920F07F40C1F83C056A
:10B91000704700000010004010B50022012910D02F
:10B92000022908BF4FF080720BD0042914BF0829E8
:10B930004FF0C74205D04FF42F714FF03E00F8F79B
:10B940003DFB42F484710C4A41F48011116040F4D3
:10B950004030111D40F0007008600848D0F85005D4
:10B96000C0B203281CBF0B2810BD4FF435714FF037
:10B970003E00F8F723FB00001415004000100040C3
:10B980000149887670470000181000202DE9F84F13
:10B99000DFF8F4830127C8F84C70FC48D0F840B5B4
:10B9A00000F036FFFA4CDFF8ECA3FB4DC4E90F0BB7
:10B9B00094F835000026D8B1D5F8040110F100093B
:10B9C00018BF4FF00109D5F81001002818BF012059
:10B9D00050EA090115D08021C5F808130903CAF8F7
:10B9E000001084F8356090F0010F18BFBDE8F88FA3
:10B9F000A08B96287ED3607A01287CD002287BD049
:10BA0000BAE0D5F80001E549DFF894B338B3C5F8DA
:10BA100000616F61FF20009002E0401E009019D08D
:10BA2000D5F81C0100280098F7D098B1086800F0FC
:10BA30007F0B94F8380058453CBF002000F0BAFA5C
:10BA400084F837B0C5F81C610120C5F808032F64DD
:10BA5000AF6307E040F667313E20F8F7AFFAB9F17F
:10BA6000000F03D0B9F1000F2AD063E0086800F09E
:10BA70007F0084F83700C5F81C6194F8361049B18E
:10BA800094F83810814218D2002000F093FA2F6405
:10BA9000AF6312E0C3490A6894F8383091B2120CCF
:10BAA000984203D30F2906D9022A04D2012000F0BC
:10BAB00081FA2F6401E02F64AF63DBF8000000908F
:10BAC0008020C5F80403C8F84070D8F84015B6487F
:10BAD000D0F8400543F698220A44B44982421CD269
:10BAE000D8F8400542F210721044C8F84005C8F872
:10BAF000406102E040E025E031E0AD4AC2F81015B7
:10BB0000AC48C2F81405AC484FF400210160206B2A
:10BB100040F400202063BDE8F88F0020C8F84005FD
:10BB2000C8F840618020C5F808030003CAF8000087
:10BB3000C8F840618020C5F808030003CAF8000077
:10BB4000BDE8F88FF8F796F8002818BFB0F1FF3F6E
:10BB500012D040F694014FF03E00F8F72FFAF8F7B4
:10BB600077F8002818BFB0F1FF3F05D040F69A01E2
:10BB70004FF03E00F8F722FA8648216B01602663F9
:10BB8000D5F8000220F01D0020F48070C5F80002F6
:10BB900084F83460207B4FF0000900281BBFD8F8E0
:10BBA0004401002800210121607A012802D00228E6
:10BBB0000AD005E0D5F80C01002818BF4FF008099D
:10BBC00019F00B0F18D111E0D5F80C01002818BF9F
:10BBD0004FF002097948006810F0010F08BF49F0E2
:10BBE0000409002918BF49F00109E9E7D5F8100157
:10BBF000002818BF49F0100971480078C0B1714899
:10BC0000006810F0FF001BBFD5F8141100290021B7
:10BC1000012184F82A1000281BBFD5F8180100283C
:10BC20000020012084F82B00D5F8100484F82C00A3
:10BC3000D5F80401002818BF01208DF80000C5F8D0
:10BC40000061C5F80C61C5F81061C5F80461C5F85C
:10BC50001461C5F81861C5F80861C5F86C616846DB
:10BC6000F7F798FF002818BF49F01009C8F8446199
:10BC700019F0100F06D019F0080F02BF607A0128E2
:10BC800049F020095048D0F8400560624648D0F895
:10BC90004005206294F8290002281CBF607A02281F
:10BCA000217E0ED084F82810627A84F82920207A28
:10BCB0004FF0000A88B119F0110F13D0FEF7C2FF40
:10BCC0003DE0042918BF0829ECD14048006810F075
:10BCD000060F0CBF08210421E4E7E67126726672A4
:10BCE00026732CE0012814BF4FF001084FF0000824
:10BCF000E079012818BF00200090E6712672667274
:10BD0000A08B0023F2B3B8F1000F6ED0B8F1000F92
:10BD100005D0012A76D004F0ECFA616A4318009845
:10BD2000194640B10BF13B00884292BFE7712F6189
:10BD30004FF0010A03D8A27A4046FFF719FC94F8A5
:10BD40004400B0B1D5F8000220F4801040F00200A9
:10BD5000C5F800020F484FF48021016060691C495A
:10BD600020F00300606108601B491A48086084F8ED
:10BD70004460DFF8688019F0010F48D0D8F800005F
:10BD800080477AE02CE030E0008000400C800040EA
:10BD90001810002008F50140001000404815004030
:10BDA0001C11004074150040048000404081004098
:10BDB00098F001401410004004F5014000140040C8
:10BDC000D0010020401600400880004014140040BC
:10BDD00000190040803202001019004008100020B5
:10BDE00040F647013E20F8F7E9F8012A05D004F0B3
:10BDF0008EFA616A431892E704E000F013FB616A6F
:10BE000043188CE700F000FB616A431887E719F0DC
:10BE1000020F29D019F0040F20D100F047FEE8B935
:10BE200000F034FED0B940480068C0F34253C0F37C
:10BE3000006200F00F01C0F3031CC0F303206AB1DD
:10BE400000291CBFBCF1000F002807D1374800684B
:10BE5000002818BF032B38BF49F0040927EA9900CE
:10BE60005146D8F8042007E019F0280F05D0D8F87B
:10BE7000082027EA59115046904719F0100F1CBFAF
:10BE8000D8F80C008047607A022818D1207BB0B126
:10BE9000022806D0012835D040F634413E20F8F77C
:10BEA0008DF82169606A08442149C1F84005206B7A
:10BEB000204940F4800020634FF48000086094F82B
:10BEC0004500002818BFBDE8F88F19F0100F14BF07
:10BED0000096BDE8F88F0098401C0090B0F1FF3F3D
:10BEE0001DD0D5F85005C0B2042818BF0C28F2D0D8
:10BEF000C5F810614FF0E0214FF00200C1F8800258
:10BF0000BDE8F88F616A2069884284BF0849C1F89A
:10BF10004005CCD840F635413E20F8F74FF840F6C2
:10BF20005D413E20F8F74AF8501400405414004098
:10BF30000480004004F5014010B5194BB1F804C06D
:10BF400003EB8004C4F820C691F800C0D1F80110BA
:10BF50004CEA0121C4F800161249D1F800C00121B1
:10BF600001FA00F04CEA0001C9B232B1012A0BD04B
:10BF700040F2AD513E20F8F721F8D3F84026C2F345
:10BF8000072222EA000005E0D3F84026C0B2C2F33F
:10BF90000722104341EA0020C3F8400610BD00000C
:10BFA0000010004040160040014901200870704711
:10BFB000D00100200E4A0F49136870B123F08203AC
:10BFC00043F07D0343F0004313600A6822F010023F
:10BFD00042F0600242F0004205E023F000431360AB
:10BFE0000A6822F000420A60034981F8360070476F
:10BFF0003C1700407C170040181000200949497A7E
:10C0000001290AD002290CBF10F0020F704700BFAF
:10C0100005494FF001000861704710F0040FF7D098
:10C02000704700001810002000100040F8B53B4C8D
:10C030000546012D20763A4808BF032110D0022D75
:10C0400008BF04210CD0042D08BF062108D0082DFC
:10C0500008BF052104D040F655513E20F7F7AEFF4A
:10C060000160A17E2F48405C00F51660B0F5166FA8
:10C070003ABFA0F6381040F48070A0F516602A4E42
:10C08000C6F80805294A01F07F001060207A0128CF
:10C0900013D1A07A94F919206B4600F0EDF99DF9BF
:10C0A000000000F0ABF90DF10100F7F7EFFD20B152
:10C0B00040F2EE513E20F7F781FFFF2084F8370071
:10C0C000D6F8000240F48870C6F8000200F008FDBF
:10C0D00080B115F00C0F0AD00120C6F80403FFF759
:10C0E00069FF0120F063306484F8350002E000202D
:10C0F000FFF760FF284600F027F900F0D7FC002882
:10C1000018BFF8BD00F0C2FC002818BFF8BD0848F1
:10C11000016841F4C0210160F8BD00001810002042
:10C120001015004028C200000010004054150040C7
:10C130006815004038B52C4A0446012C10762B486F
:10C1400008BF032110D0022C08BF04210CD0042CFE
:10C1500008BF062108D0082C08BF052104D040F6EE
:10C1600055513E20F7F72AFF0160917E2048405C40
:10C1700000F51660B0F5166F3ABFA0F6381040F41F
:10C180008070A0F516601B4BC3F808051A4B01F030
:10C190007F001860204692F919206B4600F06CF978
:10C1A0009DF9000000F02AF90DF10100F7F76EFD8E
:10C1B00020B140F2EE513E20F7F700FF00F076FC90
:10C1C000002808BF38BD0D4A11685006022CD0F86F
:10C1D00020030CBFC0F30660C0F3062021F4FE412B
:10C1E00041EA0020106038BD1810002010150040F2
:10C1F00028C200000010004054150040881500407F
:10C20000040000000000DC05E8030000000000005E
:10C2100000000000D41700002CA6E0A1000020A818
:10C2200000000000000020A80406080A0C0E1012EE
:10C230001416181C1E20222426282A2C2E303234B4
:10C2400036383A3C3E40424446484A4C4E021A5028
:10C25000010000001011004000000000000000007C
:10C26000000000000000000000000000141E00009C
:10C27000301100000000000060EA00000000000033
:10C28000000000000000000060EA00000200000062
:10C29000000000000000000000000000000000009E
:10C2A00000000000008000400000000000000000CE
:10C2B00000000000000000000080004000000000BE
:10C2C000000000000000000001000000000000006D
:10C2D000000000000000000000000000000000005E
:10C2E00028000000180000000000000050010000BD
:10C2F00000000000000000000000000050010000ED
:10C3000000000000141E00003011000000000000BA
:10C31000B45F00000000000000000000000000000A
:10C320003C7300000000000070170000A00F000028
:10C33000000000003C280000000000000000000099
:10C34000000000003C28000010B5044600F0C8FBC7
:10C35000002808BF10BD0849082C18BF042C086825
:10C3600003BF20F46C5040F4444040F0004020F003
:10C370000040086010BD00004017004070B5054641
:10C3800014460846FFF7EEF805EB4501C1EBC51171
:10C39000C0EBC101074850F8240008444FF47A71FB
:10C3A00000F6B730B0FBF1F52046FFF78DF82844D2
:10C3B000401D70BD54C4000070B5DFF83CC01C4681
:10C3C0000C4B3CF8111000EB400C53F82230CCEB36
:10C3D000C01001EBC00003F6B73318444FF47A7174
:10C3E000B0FBF1F51046FFF76FF828442044401DDC
:10C3F00070BD000054C4000040C400000149C0B238
:10C40000086070470C150040054A32F811104FF4CF
:10C410007A7201F2E731B1FBF2F10844801E7047F5
:10C4200040C40000054A32F811104FF47A7201F549
:10C430007A71B1FBF2F108447047000040C400007B
:10C440000000DC05E8030000000000000000000020
:10C45000D417000000000000141E0000301100007E
:10C460000000000060EA0000000000000000000082
:10C470000000000060EA00002DE9F8431E469046E7
:10C480000F460546F3F756FE254C81462078A84214
:10C4900004BF6078B8420BD194F90200404504BF54
:10C4A000E078484504D1A0883080A079B07032E0AF
:10C4B0004246012D08BF002010D0022D08BF0120E8
:10C4C0000CD0042D08BF032008D0082D08BF02207F
:10C4D00004D040F233410620F7F770FD6B46394631
:10C4E000F3F76EFE18B13D217520F7F767FD38466A
:10C4F000FEF7A0FB024631469DF90000F7F7D2FB9C
:10C50000E0713088A080B078A0712570677084F8E1
:10C51000028084F8039094F90700BDE8F8830000D6
:10C52000250200202DE9F04F07468C460846099E5B
:10C5300015463C461946002B40F0C6808242B2FAAE
:10C5400082F746D94FB1C7F1200E24FA0EFE00FA49
:10C5500007F3BD404EEA030CBC404FEA15481FFAF2
:10C5600085FEBCFBF8F9220C08FB19C309FB0EFA87
:10C5700042EA03439A4528D9EB1809F1FF3004D267
:10C580009A4502D9A9F102002B44A3EB0A03A4B2F5
:10C59000B3FBF8F208FB123302FB0EFE44EA03443D
:10C5A000A64514D92C1902F1FF3303D2A64501D9AF
:10C5B000931E2C44A4EB0E0443EA00401EB1FC4041
:10C5C000002334607360BDE8F08F4846DDE7134612
:10C5D000F0E702B9FFDE87BB831A01214FEA154E4F
:10C5E000AAB2B3FBFEFC200C0EFB1C330CFB02F8C2
:10C5F00040EA0343984563D9EB180CF1FF3004D2AD
:10C60000984502D9ACF102002B44A3EB0803A4B275
:10C61000B3FBFEFC0EFB1C330CFB02F244EA0344AA
:10C62000A2424FD92C190CF1FF3304D2A24202D9F5
:10C63000ACF102032C44A41ABEE7C7F1200C20FA87
:10C640000CF800FA07F324FA0CFCBD404CEA030294
:10C650004FEA154EABB2B8FBFEFC110C0EFB1C8072
:10C660000CFB03F941EA0040814504FA07F423D9A1
:10C6700028180CF1FF3104D2814502D9ACF1020136
:10C680002844A0EB090092B2B0FBFEFC0EFB1C009C
:10C690000CFB03F842EA004398450FD9EB180CF164
:10C6A000FF3204D2984502D9ACF102022B44A3EB2D
:10C6B000080342EA014191E76146E2E76246F6E794
:10C6C0006046A2E76346B6E7834205D90EB1C6E9E4
:10C6D00000700021084676E7B3FA83F181B98342FE
:10C6E00001D3BA420AD8BC1A60EB030301209C466E
:10C6F000002E68D0C6E9004C002164E70846F7E741
:10C70000C1F1200C8B4022FA0CF41C4302FA01F513
:10C7100000FA01F327FA0CF220FA0CFB4FEA144955
:10C720001343BBFBF9F81FFA84FE09FB18BB1A0C74
:10C7300008FB0EFA42EA0B42924507FA01F73ED98E
:10C74000A21808F1FF3004D2924502D9A8F10200E4
:10C750002244A2EB0A029BB2B2FBF9F809FB1822B1
:10C7600008FB0EFE43EA024296452AD9A21808F1B8
:10C77000FF3304D2964502D9A8F10203224443EACA
:10C780000040A0FB0593A2EB0E029A42CE469846CB
:10C7900002D306D14F4504D2B9EB050E63EB040872
:10C7A000013886B1B7EB0E0362EB080707FA0CFC01
:10C7B000CB404CEA0303CF40C6E900379CE7404634
:10C7C000C7E74346DBE73146FDE6042802D24FF0D7
:10C7D0002800704702D14FF0100070474FF0000062
:10C7E0007047002180F8261000F8241F4170704720
:10C7F00070B5F3F705FD0546002406E02046F3F783
:10C8000005FDFFF7EEFF641CE4B2AC42F6D370BD49
:10C81000F6F7BEB810B50020F6F7E0FB0068002878
:10C8200018BF012010BD10B5F6F772FCF5F72AFF0E
:10C8300000F004F880B210BD00F00DB8410A43F6D4
:10C8400009525143C0F3080010FB02F000F580705C
:10C8500001EB5020704700207047002809DB00F0F2
:10C860001F02012191404009800000F1E020C0F842
:10C870008012704700280DDB00F01F02012191405B
:10C880004009800000F1E020C0F88011BFF34F8F15
:10C89000BFF36F8F704770B50246002000291DD08E
:10C8A000A2FB0101400A40EAC150490A401C41F183
:10C8B000000140F2A172831841F100015B1C41F1BB
:10C8C00000040021D3F1FF33A14103D272216D2076
:10C8D000F6F778FF00F5F460B0FBF2F070BD405859
:10C8E000002800D001207047D0F80C24D0F80C04A8
:10C8F00002F00102C00303D58A4201D10120704732
:10C900000020704710B501218807F6F705FF0028C1
:10C9100000D0012010BD4FF0804001210160704720
:10C920004FF08041D1F81824D1F8181402F0030216
:10C93000C90303D5824201D101207047002070470E
:10C9400010B500214FF08040F6F7E6FE002800D039
:10C95000012010BD002809DB00F01F0201219140D9
:10C960004009800000F1E020C0F8801270470028E4
:10C970000DDB00F01F02012191404009800000F111
:10C98000E020C0F88011BFF34F8FBFF36F8F704767
:10C9900000100200FA000000140FA763CFF977C45B
:10C9A000EFF931E961F5BC039A74062B002809DB25
:10C9B00000F01F02012191404009800000F1E020B9
:10C9C000C0F880127047EFF3108172B60278012A26
:10C9D00001D0012200E000220123037001B962B6F8
:10C9E0000AB1002070476FF02200704700210170EB
:10C9F00008467047EFF3108172B60022027001B949
:10CA000062B600207047F6F7CDBF4FF08050D0F8E7
:10CA100030010F2801D000207047012070474FF0EF
:10CA20008050D0F830010A2801D000207047012042
:10CA3000704700B5FFF7F3FF20B14FF08050D0F8FA
:10CA4000340108B1002000BD012000BD4FF080502E
:10CA5000D0F830010E2801D0002070470120704727
:10CA60004FF08050D0F83001102801D000207047DE
:10CA7000012070474FF08050D0F83001062803D0D5
:10CA8000401C01D0002070470120704700B5FFF71F
:10CA9000F1FF48B14FF08050D0F83401062803D39D
:10CAA000401C01D0012000BD002000BD00B5FFF7F3
:10CAB000E1FF38B14FF08050D0F83401062803D39D
:10CAC000401C01D0002000BD012000BD4FF080506F
:10CAD000D0F830010D2801D00020704701207047A8
:10CAE0004FF08050D0F83001082801D00020704766
:10CAF00001207047F0B480EA010C03461CF0030FDC
:10CB00003CD113F0030F0BD0002A04BFF0BC7047D8
:10CB100011F801CB03F801CB521E13F0030FF3D130
:10CB2000032A4FD9B2F1004F4CD2C2F1000C4FEAA8
:10CB3000EC740CEB947C4FEAAC0CCCF1000CBCF127
:10CB4000000F1BDD0D1F1C1F1CF0010F03D055F83B
:10CB5000046F44F8046F5FEA6C0607D06F68676083
:10CB600055F8087F44F8087F761EF7D101EB8C0159
:10CB700003EB8C03CCF1000C02EB8C02002A04BF07
:10CB8000F0BC7047B2F1004F26D2002ADCBFF0BCE7
:10CB90007047491E5B1E12F0010F03D011F801CF40
:10CBA00003F801CF521004BFF0BC704791F801C0E8
:10CBB00083F801C011F802CF03F802CF521EF5D15D
:10CBC000F0BC7047042AD9D351F804CB121F43F8A4
:10CBD00004CB042AF8D2D1E711F801CB03F801CB3A
:10CBE000521EF9D1F0BC704770B4034601F0FF0C3F
:10CBF00010F0030F09D0002A04BF70BC704703F87F
:10CC000001CB521E13F0030FF5D1C9B241EA012145
:10CC100041EA0145032A39D9B2F1004F36D25142D7
:10CC2000CC1701EB947189104E42002E11DD191FB3
:10CC300016F0010F18BF41F8045F741004D04D6066
:10CC400041F8085F641EFAD1714203EB860302EBE0
:10CC50008102002A04BF70BC7047B2F1004F1DD2A0
:10CC6000002ADCBF70BC7047591E12F0010F18BFBC
:10CC700001F801CF521004BF70BC704781F801C0A9
:10CC800001F802CF521EF9D170BC7047042AE0D3DC
:10CC9000121F43F8045B042AFAD2DAE703F801CB47
:10CCA000521EFBD170BC70470721017000207047F5
:10CCB00000207047002070470020704708B1002016
:10CCC00070476FF0150070474FF0FF30704700203D
:10CCD0007047002070474FF0FF3070477047704733
:10CCE000002070470021017070474FF0FF307047FF
:10CCF0004FF0FF3070470021017070474FF0FF3058
:10CD000070474FF0FF3070470078002801D06FF077
:10CD10001500704700207047002200F000B870B581
:10CD200014460D46001B6FF07F01884201DA084669
:10CD300002E07F2800DD7F2040B2F3F72FFA287051
:10CD40006C7000212044A97040B270BD2DE9F843F9
:10CD50008146009015460C466846F6F7DDFF2078C0
:10CD60006178A84600260844C7B2354608E0237A11
:10CD7000E279A179607900F08CFE6D1C0644EDB279
:10CD8000BD42F4D30098C01C20F003000090B8F11D
:10CD9000000F00D0002032463946F7F725FD0099F4
:10CDA0000844C01D20F007000090A0EB0900BDE87A
:10CDB000F88310B504462046F7F7D6F9002806D0C8
:10CDC000A1782078F7F714FA0028F4D0012010BDDC
:10CDD0002DE9F84F044691F800C00D4600201323BA
:10CDE00010273E2212264FF00C0A4FF0050E4FF08E
:10CDF000010904F10D014FF0110BBCF1260F73D2A4
:10CE0000DFE80CF072132B2D33FD73CBD5FCFBFA4E
:10CE1000F9F8F7F6F572725599F4F3F2F1F0EFEED6
:10CE200072EDECEBEAE9E8E772E684F800A0287915
:10CE3000A0706879E070B5F80500000A2071E87903
:10CE40006071287AA0712889000AE071A87A20729E
:10CE50006889000A60720820A7E1277001E01A20A3
:10CE600020702879A07001209FE122700220A0701C
:10CE700015F8040FE070A87A207168786071D5F811
:10CE80000200C4F80600E8886081287A20732E7AB0
:10CE90001F2E00D31F260846324605F10B01FFF76F
:10CEA00029FE0D36697AA155761EF0B27BE122701B
:10CEB0000B20A0702879E07068792071A8796071E2
:10CEC000D5F80700C4F80600B5F80B006081687B50
:10CED0002073D5F80E00C4F80D00688AA4F811007C
:10CEE000287DE074304660E161E1227084F80290B0
:10CEF0002879E070A8792071E888000A6071287AA2
:10CF0000A071687AE071D5F80A00A060E889A08174
:10CF1000287CA073288A000AE073A87C2074688AA1
:10CF2000000A6074287DA074A88A000AE074A87DB5
:10CF30002075184639E122700A20A07015F8040FF8
:10CF4000E070A87820716888000A60712879A07163
:10CF50006879E071D5F80600A0606889A081E8686A
:10CF6000C4F80E00288A6082D5F812006061E88A51
:10CF70002083287EA076288B000AE076A87E207782
:10CF8000688B000A6077287FA077A88B000AE0777B
:10CF9000A87F84F820001F2007E122701420A070D1
:10CFA0002879E070A888000A2071A87951E12270E0
:10CFB0000420A0702879E070A8792071E888000A20
:10CFC0006071A868C4F80600E868C4F80A0017E0B1
:10CFD0008EE160E140E16DE17BE131E107E1EFE00D
:10CFE000E7E0D5E0CAE0B5E0B9E060E05CE071E020
:10CFF0006BE04FE043E036E032E01DE002E072E03B
:10D000000C20D2E022700320A0702879E070A8796B
:10D010002071E888000A6071287AA0712889000AC6
:10D02000E071A87A20726889000A6072287BA07279
:10D03000A889000AE0724AE1227084F802E02879A7
:10D04000E070A888000A2071D5F80600C4F8050031
:10D05000D5F80A00C4F80900E889A4F80D005DE1DC
:10D0600084F800B038E084F800E02879A07068798E
:10D07000E070B5F80500000A2071E879E9E00820C1
:10D0800020702879A070A879E070E888000A2071E3
:10D09000287ADEE0302020702879A070A879E0702E
:10D0A000E888000A207189E022700720D7E022700A
:10D0B00084F802A02879E070A8792071E888000A35
:10D0C0006071287AA071687A55E0291D2046F7F72B
:10D0D000B1F868E0572020702879A070A888000A6D
:10D0E000E070022061E022700D22A2702A79E270C5
:10D0F000EA89A2806A79A271D5F80620C4F80720CF
:10D100006A89A4F80B202A7C20466273291D6A7C58
:10D1100082738A7BC2738A7E02744A7A4274B1F83F
:10D120001120ADF800204282CA7C02754A69C0F81D
:10D1300015200A8BA0F819200A7AC2760D7AE52DFF
:10D1400000D3E5252A461C301C31FFF7D3FC1A35E5
:10D15000E8B228E0227084F802B0484625E0227048
:10D16000A6702879E07068792071A8796071E888E4
:10D17000000AA071287AE071062016E022700E20C5
:10D18000A0700F22291DE01CFFF7B4FC10200CE05A
:10D1900022700F20A070AA7A291DE01CD21DFFF773
:10D1A000A9FCA87A0830002801D06070801CBDE876
:10D1B000F88F2270A770A888A4F803000320F4E772
:10D1C00022702120A0702879E07068792071B5F86C
:10D1D0000500000A6071E879A071287AE071687A28
:10D1E0002072A87A6072E87AA0720920DDE72270C6
:10D1F0001820A0702879E07015F8050F2071288894
:10D20000000A6071A878A0716888000AE071287926
:10D210002072A888000A6072A879A072E879E0728A
:10D22000A868E060A8892082A87BA074E87BE074ED
:10D23000B5F80F00000A2075687C60751420B4E70B
:10D24000FF202070A120A0702879E07068792071FB
:10D25000002060710420A8E7FF202070A220A070A9
:10D260002879E070A888000A2071A8796071E888A0
:10D27000000AA071287AE0712889000A2072A87A31
:10D2800060726889000AA072287BE072A889000A8F
:10D2900020730B2089E7FF202070A320A07028793D
:10D2A000E070A888000A2071A8796071E879A071FF
:10D2B00005207AE72270A3702879E07068792071E0
:10D2C000D5F80600C4F805006889A4F809000A200A
:10D2D0006BE7FF202070A420A0702879E070A88858
:10D2E000000A2071A8796071E879A07107205CE7D5
:10D2F000FF2020708020A070A988A4F80310E9887E
:10D30000A4F80510297AE17169892181A9896181CF
:10D31000E989A181297C01F00101A1730D2044E775
:10D320003E2202700122827011F8042FC2708A78A6
:10D3300002714A88120A42710A7982714A79C2716D
:10D34000D1F8062082604A8982810A7E82730A8B24
:10D35000120AC2738A7E02744A8B120A42740A7FCE
:10D3600082748A8B120AC274897F017513214170FD
:10D37000084670474A0901F01F0150F82200C840D2
:10D3800000F00100704710B520B1FFF712FD20B189
:10D39000002010BD6FF0150010BD6FF0220010BD11
:10D3A00018B111B16FF0220070476FF0150070478F
:10D3B00010B5F6F78FFF002010BD08B500788DF886
:10D3C0000000684602F0C8F908BD1FB500210091B1
:10D3D000019102910391D0F8021041F64C52914212
:10D3E00004D340F2E242B1FBF2F105E04FF47A726D
:10D3F000B1FBF2F101F55061028889B2ADF800206D
:10D40000ADF80210ADF80410C188ADF8061000891F
:10D41000ADF80800684601F08BFF04B010BDFCF7C2
:10D4200015BF08B500788DF800006846FCF71AFFB4
:10D4300008BD007800B1012002F068B970B505465A
:10D4400010220021FFF7D0FB1022002105F110006F
:10D45000FFF7CAFB4FF08054D4F88000401C0BD17A
:10D46000D4F88400401C07D1D4F88800401C03D1B4
:10D47000D4F88C00401C0BD0D4F88020D4F8840061
:10D48000D4F88810D4F88C302A616861A961EB6106
:10D490000020F7F775FC18B9D4F8A000C00718D120
:10D4A000D4F89000401C0BD1D4F89400401C07D154
:10D4B000D4F89800401C03D1D4F89C00401C08D03C
:10D4C00054F8900F6168A268E36828606960AA60F8
:10D4D000EB60002070BD38B54FF080550446D5F89C
:10D4E000A400401C05D1D5F8A800C0430004000CDE
:10D4F0003ED0D5F8A000C0073AD0D5F8A400D5F8A2
:10D50000A810ADF80010C4F80100BDF80000A4F8A0
:10D510000500A07940F0C000A071D5F89000401C33
:10D520000FD0D5F89400401C0BD0D5F89800401CC3
:10D5300007D0D5F89C00401C03D00020F7F720FC52
:10D5400040B110220021E01DFFF74EFB01202070AA
:10D55000002038BD55F8902F6968A868EB68C4F8BA
:10D560000720C4F80B10C4F80F00C4F81330EDE71F
:10D570000020ECE702F0E2B802F04CBAFCF798BEEB
:10D5800001F0AFBE01F0CABE01F023BF02880A80DD
:10D5900001F028BF01F03FBF01F043BFFCF7C0BD61
:10D5A00001F051BF01F046BF01F051BF01F06BBF68
:10D5B00001F07EBF01F0AFBF10B5F6F783FE00208B
:10D5C00010BD02F03DB802F049B802F05DB802F0BB
:10D5D00088B8891D0844504380B2704770B50B88E5
:10D5E000047F00F12406C3F30E0502882E44A41D17
:10D5F0003688224492B22644541E344494FBF2F4FA
:10D6000002FB0452408892B2904203D903F40040D6
:10D61000104302E04FF400409843088070BD8842F8
:10D6200001D101207047002070474204B2EB414F06
:10D6300007D100F4004001F40041884201D00120EC
:10D64000704700207047C1888088FFF7E8BF818855
:10D650000089FFF7E4BFF8B5044600F12403C08851
:10D660000F46C0F30E06608A991908B1B84201D27C
:10D670000020F8BDE089002540B1B1F800C0604548
:10D6800008D040F251211420F6F798FC607F887092
:10D690000D800EE094F81CC018440CF1060CB44444
:10D6A0006044B4F81EC020F803CC94F820C000F801
:10D6B00001CCE0893844E0810888384408809AB178
:10D6C000A11D2046FFF78AFFE581607F401C60773F
:10D6D000A07D8DF80000009800909DF8000078B1C2
:10D6E000E088A082A5750BE0207FE189801D304491
:10D6F0001944084430F8031DE183807884F8200041
:10D7000065820120F8BDC01C704710B5C2884389EE
:10D71000C2F30E04C3F30E01091B02F4004203F42A
:10D7200000439A4201D1428811440288007F801D43
:10D73000104480B291FBF0F080B210BD10B50446E9
:10D74000C1888088FFF76BFF38B9A08928B9208A83
:10D7500018B9A088A18A884201D1002010BD211DDE
:10D760002046FFF73BFF00202082012010BD70B54E
:10D77000044600F12402C1888088C0F30E03D51846
:10D78000A288A38A9A4213D0FFF749FF80B9A089E3
:10D7900070B9A46974B12046FFF759FF50B92089C8
:10D7A0002434C0F30E002044A9788078884201D147
:10D7B000002070BD284670BD0388452B00D245234C
:10D7C0001380C288C2F30E0300F124021A440A60D7
:10D7D000C0897047007F801D0844C01E1060088803
:10D7E00070474FF6FF7181820021817570472DE9E6
:10D7F000F0411646DDF818800F4604461D464246A5
:10D800001946304600F055F8874201D2A82119E0A8
:10D81000E01C20F003012046A14201D0A92111E023
:10D8200024220021FFF7E0F94FF6FF70A082257750
:10D83000424629463046FFF7CCFE6080B0F5004FE7
:10D8400003D9AF211420F6F7B9FB268000206077BA
:10D85000BDE8F0818161886170472DE9F047894614
:10D86000044600F124010689B0F80A808088174632
:10D87000C6F30E028D1801463046FFF7D0FE10B1F8
:10D880000020BDE8F0870FB1E81C3860B9F1000056
:10D8900003D0227FE91CFFF72DF92D8804F1080140
:10D8A0002046FFF79BFE464501D12089608128462E
:10D8B000E7E710B50446FFF78CFE0021452C02D2A5
:10D8C000C4F1450189B22430084480B210BD2DE96D
:10D8D000F0478846C18804460089C1F30E0504F16B
:10D8E0002406C0F30E0706EB0509FFF79EFE002293
:10D8F00098B92088452800D24520AF4206D9217F1B
:10D900007B1B891D591A814200DA0846E18911B151
:10D91000B9F80030C01A404503DA62820020BDE841
:10D92000F087207F3144801D28440844A4F81280E9
:10D93000C01EF4E770B50023A1F108024FF6F7749A
:10D94000A24204D340F2CD111520F6F737FB02684E
:10D950000AB91EE01046026893888B4202D0136811
:10D96000002BF7D1948813468C4201D111680DE049
:10D9700001F10805ADB2AC420AD3641A1144002289
:10D980000A608C800268126802600A60016000E030
:10D990000023184670BD10B50C0004D0082C07D227
:10D9A00040F295110AE008B100210160002010BD8D
:10D9B00058B1B4F5803F04D340F2A7111520F6F713
:10D9C000FDFAA1B2006800F014F8201D10BD00217E
:10D9D000026803E093881268194489B2002AF9D1D9
:10D9E00000F007B800230B608A8002680A600160BB
:10D9F000704700234360021D0181026070473EB5FD
:10DA00000446694600F029F868B140F25A2107E05F
:10DA1000BDF804002146F6F781FD20B140F25F21F8
:10DA20001720F6F7CBFA6846F6F706FD0028EFD088
:10DA30003EBDA0F57F43FF3B01D0052901D3002067
:10DA40007047F6F79DBDA0F57F42FF3A01D005294A
:10DA500001D300207047F6F7CDBD70B505460C46E2
:10DA6000084600F0BDF908B1102070BD052D01D3A6
:10DA7000072070BD25700020608070BD10B5044681
:10DA8000F6F704FEA04201D9012010BD002010BD10
:10DA9000704770B50E461D46114600F013F8044657
:10DAA0002946304600F004F82044001D80B270BDC5
:10DAB00010B50A460121FFF7FCFE4FF6FC71C01CB1
:10DAC000084010BD10B50A460A21FFF7F2FE4FF6D6
:10DAD000FC71C01C084010BD10B50446084600F09B
:10DAE00015F821180A7D022A08D0497D022909D09B
:10DAF000032A03D0032905D0002010BD04EB400009
:10DB0000008B10BD04EB4000408B10BD08B100201D
:10DB100070470220704710B504460846FFF7F6FF2D
:10DB200004EB4000018B11B9408B002800D001208C
:10DB300010BD38B5044680780D468DF80000009879
:10DB400000909DF8000048B91046FFF7DFFF21184C
:10DB50000A7D022A04D0497D022905D0002038BD63
:10DB60000246401CC0B201E0411CCAB285B1231874
:10DB7000002104EB4000197501830320A1180875EA
:10DB800004EB82004068286004EB4200008BA88010
:10DB9000012038BD70B5044615460846FFF7B6FFAC
:10DBA00021180A7DAA4203D104EB4000008B70BD0E
:10DBB000497DA94203D104EB4000408B70BD002099
:10DBC00070BDB0F5FF7F01D240087047FF2070475D
:10DBD00010B50446FFF7F5FF201A40F27261884243
:10DBE00000DB084680B210BD0121FFF775BF2DE9AB
:10DBF000F041064642F3800748780C4622F00405BF
:10DC00007F1C00B195B9284310D0002020B17DB110
:10DC100000212046F6F74AFEFF20A0703846FFF7A5
:10DC200075FF2118097D032904D007E00120EDE7E5
:10DC30000121EEE7022D01D0401CC0B222180121C3
:10DC4000117504EB4002002104EB8000118342684F
:10DC5000A170334661F30F030CC6BDE8F0812DE9D6
:10DC6000F04104461E4690460846FFF74FFFFF214D
:10DC7000A17021180A7D012A04D0497D01290CD107
:10DC8000401CC0B204EB40050027298B2B8C8A195D
:10DC90009A4205D920442F8307750020BDE8F08102
:10DCA00004EB80003246406808444146FEF722FFFC
:10DCB000288B30442883A7700120EFE7022200213F
:10DCC000FFF768BF10B50121FFF725FF002800D03E
:10DCD000012010BD0122FFF72CBF0022FFF729BF52
:10DCE00070B5044615460846FFF710FFFF21A170E6
:10DCF000211802220B7D012B07D04B7D012B09D06F
:10DD00004FF48B710920F6F759F904EB40000583B5
:10DD10000A7503E004EB400045834A750020A070BB
:10DD200070BD01210170704701221146FFF732BF1B
:10DD300001220021FFF72EBF0021FFF7CDBE0028F2
:10DD400009DB00F01F02012191404009800000F131
:10DD5000E020C0F88012704700280DDB00F01F02A1
:10DD6000012191404009800000F1E020C0F88011BD
:10DD7000BFF34F8FBFF36F8F704710B50E20FFF7C3
:10DD8000EBFF0E20FFF7DBFF0F20FFF7E5FFBDE8FD
:10DD900010400F20FFF7D3BF002809DB00F01F025F
:10DDA000012191404009800000F1E020C0F880127C
:10DDB00070474058002800D00120704710B5044635
:10DDC0002046F6F7CFFE1128FAD010BD10B5FFF7A8
:10DDD000F5FF002803D0A0211D20F6F7EFF810BDB5
:10DDE00008B1002070470120704750400A7893F82E
:10DDF00000C082EA0C0210444A7893F801C082EA1B
:10DE00000C0210448A7893F802C082EA0C02104493
:10DE1000CA7893F803C082EA0C0210440A7993F896
:10DE200004C0497982EA0C0210445A795140C14237
:10DE30000CBF01200020704710B5002904464FF0A8
:10DE4000060102D0F6F728F901E0F6F741F960790A
:10DE500000F03F00607110BD704730B50C460546BC
:10DE60008DB04FF0030104F1030012B1F6F714F97D
:10DE700001E0F6F72DF960790D2200F03F0040F047
:10DE800040006071002104A8FEF7AEFEE0788DF836
:10DE90001F0020798DF81E0060798DF81D0028681C
:10DEA000009068680190A8680290E868039068464E
:10DEB000FFF78CFF9DF82F0020709DF82E006070FA
:10DEC0009DF82D00A0700DB030BD30B58DB00C4662
:10DED00005460D22002104A8FEF786FEE0788DF8A5
:10DEE0001F0020798DF81E0060798DF81D002868CC
:10DEF000009068680190A8680290E86803906846FE
:10DF0000FFF764FF20789DF82F1088420CD16078CD
:10DF10009DF82E10884207D1A0789DF82D108842D8
:10DF200002BF01200DB030BD00200DB030BD10B5D6
:10DF3000FCF7D6FD002804BFFF2010BDBDE810404F
:10DF4000FCF7AEBD10B5F7F7C7F9102804BF0020E5
:10DF500010BDF7F707FA012010BD70B50C46054655
:10DF60000021FFF770FD606010B10020207070BDCF
:10DF700001212846FFF767FD6060002804BF0220EA
:10DF800070BD01202070002070BDA0F6015106294F
:10DF90009ABF4FF47A71A0F5506040F2E2414843D5
:10DFA0007047A0F57A7141F27072914294BF4FF4BC
:10DFB0007A7140F2E241B0FBF1F098BF00F5506099
:10DFC00080B2704711F00C0F14D001F00401002949
:10DFD0000DBF4022102296214FF4167101F5BC713D
:10DFE000A0EB0103884282BF93FBF2F080B270473E
:10DFF00000207047022908D07028F9D97038C1175D
:10E0000000EB5170C0F3CF0070473C28F0D93C388A
:10E01000C11700EB9170C0F38F0070470968C0F81A
:10E020006E1070472DE9F04107460E46D7E90445CA
:10E03000F3F730FDA0B136B3D7E90401021B61EB61
:10E04000050300200146801A71EB03001BDA501C07
:10E0500073F1000009DB40F236212920F5F7AEFF0D
:10E060004FF40B712920F5F7A9FF9019401EB0FB62
:10E07000F6F101FB06F0201845F10002C7E90402A1
:10E080000846BDE8F0810020BDE8F08141F64C5221
:10E0900091423EBF642110FB01F0704740F27121B4
:10E0A00010FB01F04FF6FF7101EA40007047C378A2
:10E0B000024613F03F0008BF70470520127903F0B5
:10E0C0003F0C12F0010318BF012323B1002914BF34
:10E0D0000B20704701E000294FD012F0020318BF57
:10E0E000012323B1012914BF801D704701E00129DC
:10E0F00043D012F0040318BF012323B1022914BF37
:10E10000401C704701E0022937D012F0080318BF05
:10E11000012323B1032914BF801C704701E00329A8
:10E120002BD012F0100318BF012323B1042914BF10
:10E13000C01C704701E004291FD012F0200318BF53
:10E1400001232BB105291ABF1230C0B2704701E07C
:10E15000052912D012F0400218BF01222AB1062967
:10E160001ABF401CC0B2704701E0062905D007293C
:10E1700003D1411F8C45C8BF70470020704770B560
:10E180000278417802F00F02082A4AD2DFE802F052
:10E1900004080B4949490F14881F1F280AD940E079
:10E1A0000C2907D03DE0881F1F2803D939E0881FBC
:10E1B0001F2836D8012070BD0A0032D00446C0782E
:10E1C00000268209032A09D000F03F05681C884216
:10E1D00004D8204600F04EF8A84201D9304670BD60
:10E1E000E0784FF0010510F03F0F1EBF14F104005E
:10E1F000007810F0100F12D004212046FFF757FFCF
:10E20000002818BF14EB0000E8D0017801F03F01AE
:10E210002529E3D280780221B1EB501FDED32846B6
:10E2200070BD002070BDC178407801F03F01401AF8
:10E23000401EC0B2704770B5C4788C4604F03F01F0
:10E24000457804F03F042C1B641EE41AE4B29442A7
:10E2500088BF1446BCF1000F06D019440844011DC4
:10E2600022466046FEF746FC204670BDC07800F0AE
:10E270003F007047C17811F03F0218BF01220079BA
:10E2800010F0010318BF012303EA020C11F03F0F45
:10E2900014BF0123002310F0020218BF01221A400C
:10E2A000624402EB42024FEA420C11F03F0F14BFEE
:10E2B0000123002310F0080218BF01221A400CEBC2
:10E2C000420C11F03F0218BF012210F0040318BFE6
:10E2D00001231A40944411F03F0218BF012210F0AC
:10E2E000200318BF01231A4002EBC2020CEB420CC0
:10E2F00011F03F0218BF012210F0100318BF0123D4
:10E300001A4002EB4202624411F03F0118BF0121A2
:10E3100010F0400018BF01200840104410F0FF002A
:10E320001CBF401CC0B270470078C009704700781D
:10E33000C0F38010704730B5027883B002F00F024E
:10E34000032A57D0052A52D10D46044600F11F0179
:10E35000684601F0E7FF9DF804009DF8001000F00A
:10E36000E0008DF80400002904BF9DF80110002989
:10E370000AD19DF80210002901BF9DF80310002961
:10E38000002803B008BF30BDB4F81900B4F81B3042
:10E39000B4F81710A27D002D18BFB0F5506F09D941
:10E3A00040F6075C604505D894F801C0BCF1220F27
:10E3B0001DD111E094F801C0BCF1220F17D1A0F1DA
:10E3C000060C40F67A45AC4511D882B1082A98BFB0
:10E3D00082420CD288420AD3B3F5FA7F07D2B4F84E
:10E3E0001D00B0F5486F02D803B0012030BD03B066
:10E3F000002030BD40780C28F9D1F5E72DE9F04137
:10E400000178012601F00F01002504290CD007290D
:10E410000FD008291CBF0020BDE8F08140780E28ED
:10E4200034D02846BDE8F0814078801F1F282DD9C0
:10E43000F7E704464078E1788A09032AF1D001F031
:10E440003F07791C8142ECD82046FFF713FFB84202
:10E45000E7D8E07810F03F0F1EBF14F104000078F9
:10E4600010F0100F12D004212046FFF720FE0028E4
:10E4700018BF14EB0000D4D0017801F03F0125292A
:10E48000CFD280780221B1EB501FCAD33046BDE80D
:10E49000F08170B5144605461F2A03D9B5212A20FC
:10E4A000F5F78CFD05F10900FEF724FBA01D68704F
:10E4B00070BD10B5027801F00F0302F0F0021A43AC
:10E4C0000270092913D2DFE801F0050705070509E5
:10E4D000050B0F00062108E00C2106E0222104E0D4
:10E4E00001210022C27000E00E21417010BD6F2199
:10E4F0002A20F5F763FD0A68C0F809208988A0F88A
:10E500000D1070470278802302F07F0203EAC111E8
:10E510001143017070470A68C0F803208988A0F889
:10E52000071070470278402302F0BF0203EA81110E
:10E5300011430170704770B5144605461F2A03D970
:10E54000D7212A20F5F73AFD05F10900FEF7D2FAA6
:10E55000A01D687070BD006801F19C0290429CBFD4
:10E5600000207047401A9C3840087047002803DBA1
:10E57000884204DB084602E049428842FADB00B2E6
:10E58000704710B50446807C022818BF032809D1C3
:10E5900094F8670004F16801F6F724FD08281CBF11
:10E5A000012010BDA07C00281EBF0228607E10BD87
:10E5B0004FF00000BDE81040F6F7E2BB08B590F858
:10E5C00086108DF800109DF8001059B990F8B00031
:10E5D0008DF800009DF8000010B1FCF705F908B1B6
:10E5E000002008BD012008BDFF200870486CFFF71F
:10E5F00098BB30B50D4685B004464FF4AC7200218F
:10E60000FEF7F2FAFF2020707F2084F83F001320ED
:10E610006080F6F7E1F901466064002202A8FFF786
:10E62000E6FA00220121606CFFF75AFB042202A8DF
:10E63000616CFFF7DCFA00221146606CFFF750FBBB
:10E64000257404F1280000F019FA6846F6F7FEFF79
:10E6500030B1694604F12E00F7F70CF805B030BD73
:10E6600040F226312D20F5F7A9FC4088C0F30011B7
:10E6700031B1C0F38000002804BF1F20704702E0C2
:10E68000C0F3400109B10020704710F0010F1CBF1A
:10E69000EE207047F6F7C6B9FF2180F87C1070476E
:10E6A000F8F79ABD10B504460020122A3CD004DCCD
:10E6B000032A18D00E2A1DD003E0192A06D01E2ADC
:10E6C0004CD040F2D2212D20F5F778FC4870212063
:10E6D0000870D4F8CF004860D4F8D300886094F86C
:10E6E000D700087310BD487007200870D4F8C20026
:10E6F000486010BD48701420883401F8040BB4E859
:10E700000D10A1E80D1094E80D10A1E80D100120E6
:10E7100001F81C0C11F8200C983C002818BF10BD03
:10E72000FCF762F890B910BD487017200870D4F853
:10E73000B2004860B4F8B60008810879002818BF14
:10E7400010BDFCF751F8002818BF10BD206A0088E2
:10E75000F6F77EF8BDE81040FFF743B84870262072
:10E760000B46087004F1E1012222BDE81040181D9B
:10E77000FEF7C0B98068704700B5428885B0C2F323
:10E7800000138C46002B07BFC2F3C002002A0120F1
:10E7900005B018BF00BD00F1280100914188ADF817
:10E7A00004108168029101798DF80C1040798DF880
:10E7B0000D0069466046F8F77BFD05B000BD0022FC
:10E7C000A0F8402043881D2B0CBF42734173704753
:10E7D00010B54188C1F300122AB9C1F340010029E4
:10E7E00018BF012400D10024406CFFF767FA00280D
:10E7F00018BF012024EA000080F0010010BD10B510
:10E800004088C0F3001119B1C0F3800048B10AE09C
:10E81000C0F3400139B910F0010F02D1F6F702F947
:10E8200008B1012010BD002010BD8078C0F3401059
:10E830007047807800F001007047408809280CBFBD
:10E840000120002070478078C0F3C00070478078B6
:10E85000C0F3001070478078C0F34000704790F913
:10E86000100070470078FF2814BF01200020704777
:10E870000A68C0F813208988A0F817100121417692
:10E880007047007B704740797047016290F86020C4
:10E890004A72D0F86120C1F80A20B0F86500C8813A
:10E8A000704780F8781070472DE9F0410446807871
:10E8B000C0F3C00058B13C23FF222046216AF8F77C
:10E8C00061FD0E22214604F17E00F6F72BFFA078B1
:10E8D0004FF0000510F0010F22D0206A3C26078877
:10E8E000F7F758FAFBF780FFA8B9217884F8B3103E
:10E8F000A4F8B47084F8B260607B10B984F8B650A4
:10E9000003E094F8400084F8B6001222214604F196
:10E91000A800F6F707FF012084F87900BDE8F08130
:10E920004FF6FF773C26F7F735FAFBF75DFF002837
:10E93000F1D1217884F8B310A4F8B47084F8B260EF
:10E94000607B0028DDD1D9E7407C002818BF01207A
:10E9500070470121F7F788BD0121F7F785BD10B594
:10E96000017042708078C0F38003C0F3400C6344B0
:10E9700000F00100184410FB01F010FB02F0FF282A
:10E9800038BF10BD5C212E20F5F718FB8178C1F34C
:10E990008002C1F340031A4401F00101114442789E
:10E9A000007812FB00F04843C0B270478278002123
:10E9B00012F0010F05D0C37813F0010F08BF012139
:10E9C00010D012F0020F05D0C37813F0020F08BF69
:10E9D000022107D012F0040F04D0C37813F0040F03
:10E9E00008BF042143795B1CDBB2437190F801C07E
:10E9F00063450DD10023437190F803C04CEA010C2C
:10EA000080F803C0944503D1C3700279521C02718F
:10EA1000012904BF25207047022904BF2620704722
:10EA2000042904BF2720704710B539212E20F5F79F
:10EA3000C5FA8170704710B48178C1F38002C1F3C8
:10EA400040031A4401F001014378114413FB01F221
:10EA5000C178C1F3800CC1F34004A44401F001016A
:10EA6000614490F805C011FB03C103780079181ABE
:10EA700010FB02F0401A10BCC0B2704710B504463B
:10EA800001F055FC01206070207010BD0021C170A4
:10EA900041710171704740F25A314843704740F26A
:10EAA000EF2070470E021C043006600C5A03B406B7
:10EAB000C505F50B2512A301B103BF05EF024906F9
:10EAC000A30910B590F8501100291CBF002010BDFB
:10EAD00090F8101100291CBFD0E945128A429CBF52
:10EAE000012010BDFFF7E0FE002010BDF0B583B09F
:10EAF000002531B1012976D040F295713020F5F72B
:10EB00005DFA044690F80901002638B1F7F7B2F92A
:10EB100042F21071B0FBF1F201FB12062046FFF742
:10EB200029FED4E94E123044401845EB0201C4E9F5
:10EB30004E0184F82851012084F83301022084F822
:10EB400032012046FFF783FE002808BF6B2624D041
:10EB50002046FFF76EFE30B92046FFF77CFE002806
:10EB600008BF422600D049266846F5F795F89DF87B
:10EB70000000002814BF0127002701A8F5F774F84A
:10EB80009DF80400002818BF0120384318BF09363B
:10EB9000F4F7C8FF002818BF1836A4F8306194F8BD
:10EBA0005001F8B9D4F84C016FF00042D4F8481184
:10EBB000504070EA010017D02046F7F753FAD4F816
:10EBC000382100F59670D4F83C118018D4F84831FB
:10EBD0006941D4F84C21181A72EB010004D5204683
:10EBE000FFF762FE07E014E094F8080104F5947161
:10EBF000F2F75CFD40B1A4F84051FCF767FB03B0AD
:10EC0000BDE8F040F3F784BB40F2EF613020F5F748
:10EC1000D5F980F81051FCF759FB03B0BDE8F0407E
:10EC2000F3F776BB10B5044690F82001002808BF22
:10EC300010BD012084F8500101462046FFF731FE47
:10EC400094F8200188B194F80801F3F7C9F894F812
:10EC50000801F3F71DFA94F80801F3F7F7F9002813
:10EC60001CBF002084F8200101D0002010BD40F21C
:10EC700009213020F5F7A2F9D0F80C01704790F87F
:10EC8000200170472DE9F04182B004000AD0002530
:10EC9000092980F00181DFE801F0091B494944FF9F
:10ECA000F3DAF900CA213020F5F788F92046F7F7A2
:10ECB000ABFB20B140F279213020F5F77FF9D4F891
:10ECC0002C0102B0A0F21B10BDE8F041F3F7F0BB3D
:10ECD0002046FFF7B8FDB8B92046F7F7C3F900F5AD
:10ECE0009675D4F82C01A8420CD2281A0321F2F709
:10ECF000BFFA38B1C4F82C5102B02046BDE8F0414B
:10ED0000FFF7CEBCC4F82C512046F7F79FFB002834
:10ED100004BF02B0BDE8F0814FF42B713020F5F74D
:10ED20004DF902B0BDE8F041FCF730BE01272046A6
:10ED3000FFF78DFD002808BF6B2627D02046FFF780
:10ED400078FD30B92046FFF786FD002808BF42262F
:10ED500000D049266846F4F79FFF9DF80000002880
:10ED600014BF4FF001084FF0000801A8F4F77CFF32
:10ED70009DF80400002818BF012058EA000018BFC1
:10ED80000936F4F7CFFE002818BF1836A4F8306112
:10ED900084F82851012684F8336194F8100168B191
:10EDA000D4E94E0210F57A7142F10000C4E94E1028
:10EDB000002104F59470FFF735F90EE02046FFF7C7
:10EDC000D9FCD4E94E1209186A41C4E94E12014631
:10EDD00004F59470FFF726F9471CB4F84001411C74
:10EDE0000A293CBF3844A4F84001D4F80C0138B1DA
:10EDF000B4F84001401C0A2828BF84F8326102D2CE
:10EE0000022084F8320194F8500100BBD4F84C0180
:10EE10006FF00042D4F84811504070EA01001FD052
:10EE20002046F7F71FF9D4F8381100F59670D4F89A
:10EE30003C21401845EB0201D4F84831D4F84C216C
:10EE4000181A72EB01000BD52046FFF72DFD94F840
:10EE50000801F3F7FBF884F8205102B0BDE8F08117
:10EE600094F8080104F59471F2F720FC00281CBF07
:10EE700002B0BDE8F0814FF4D5613020F5F79EF87F
:10EE800002B02046BDE8F041FFF70ABCEA2130207D
:10EE900000E001E0F5F792F8EE213020F5F78EF86A
:10EEA000F5F776BCF9F7B2BD40F291313220F5F7B3
:10EEB00085F8F9F7ABBD00B583B0F5F7C5FD01AA3C
:10EEC0006946FEF779FC0098FEF71DFCC07CFF2820
:10EED00014BF0120002003B000BD2DE9FF4F83B017
:10EEE0001D46DDE910890E460746DDF848B0F5F706
:10EEF000ABFD0446FEF709FC012804BF07B0BDE8DE
:10EF0000F08F204601AA6946FEF756FC0098FEF7EE
:10EF1000FAFB04461C2200211230FDF765FE4FF07B
:10EF2000010A84F812A056B1012E0DD0022E10D085
:10EF3000062E13D04FF42C713320F5F73FF8207FC5
:10EF400040F0130020770DE0207F40F0150020777F
:10EF500008E0207F40F01000207703E0207F40F0A1
:10EF60001200207704F11402561E4046B8F1FF0F3C
:10EF70000CD03146F6F70AF820B1307840F00200A4
:10EF800030700AE089213320F5F718F8787C30706A
:10EF90007868016811608088908084F81BB084F8DC
:10EFA0001EA00026E677FF2084F82000217F11F0C4
:10EFB000040F08BF84F8250012D004F12600411E7A
:10EFC000022D18BF032D05D0BA681368036092881C
:10EFD000828004E0059A13680360928882800D7035
:10EFE0004FF07F0084F82C0084F82D90F5F72CFD6D
:10EFF0000546F5F723FD014601222846FEF72BFBC7
:10F0000050B12046067202220021F6F78BFB07B0B2
:10F01000BDE8F04FF6F7BEBE4FF434713320F4F77D
:10F02000CDFF2DE9F04F83B01F4690460D460646B2
:10F03000DDF830A0F5F708FD0446FEF766FB012871
:10F0400004BF03B0BDE8F08F204601AA6946FEF771
:10F05000B3FB0098FEF757FB04461C220021123038
:10F06000FDF7C2FD4FF0010984F8129004F114027B
:10F0700004F1130BFF2D0FD059462846F5F786FFF4
:10F0800030B19BF8000040F002008BF800000BE06C
:10F0900089213320F4F792FF707C8BF800007068B0
:10F0A000016811608088908084F81BA0207F002573
:10F0B00068F3000040F01A00207784F81E90E5778E
:10F0C000FF2084F8200084F825007F2084F82C009D
:10F0D00084F82D70F5F7B8FC0646F5F7AFFC01464D
:10F0E00001223046FEF7B7FA50B1204605720222DF
:10F0F0000021F6F717FB03B0BDE8F04FF6F74ABE64
:10F1000040F2FD213320F4F759FF2DE9F041064686
:10F11000C07805240D4610F03F0F4FF000081CBFCB
:10F12000304616F1040761D0FFF701F968743046E4
:10F13000FFF7FAF8A87438786870F07880092870BA
:10F14000387810F0010F08BFC5F8048002D0701D98
:10F150000B246860387810F0020F08BFC5F80880EB
:10F1600002D03019A41DA860387810F0040F18BF21
:10F17000641C10F0080F08BFC5F8148002D03019C5
:10F18000A41C6861387810F0100F08BFC5F818800B
:10F1900002D03019E41CA861387810F0200F08BFA5
:10F1A000C5F81C8004D03019E86104F11200C4B223
:10F1B000387810F0400F08BFC5F8208003D0301910
:10F1C0002862601CC4B23046FFF750F8001B001DD7
:10F1D0002044C4B23046FFF726F8287400281ABF2E
:10F1E0003019E860C5F80C80BDE8F081C5F80080F2
:10F1F000C5F80480C5F80880C5F80C80C5F81080F3
:10F20000C5F81480C5F81880C5F81C80C1F82080A6
:10F21000BDE8F081027802F00F02072A01D0F9F769
:10F22000C3BEFFF772BF30B583B05B24F4F77AFC3E
:10F23000002818BF73246846F4F72EFD9DF80000DF
:10F24000002814BF0125002501A8F4F70DFD9DF845
:10F250000400002818BF0120284318BF09342046A5
:10F2600003B030BDF5F794BA10B5DDE9023CC01A21
:10F2700071EB0C0116D54FF0FF3CD0F100437CEB55
:10F28000010103DBB2213720F4F798FE404200EB86
:10F290000201A1F10101B1FBF2F101FB02F1A1EBCD
:10F2A000000010BD6FF00043C31A71F10001BEBF32
:10F2B00090FBF2F101FB120010BDBB213720F4F7E7
:10F2C0007DFE00EBD10001F007010078C84000F09E
:10F2D0000100704718B1022801D0012070470020BA
:10F2E000704710B5044600F05BFF08B10C2010BD5C
:10F2F000207828B1012803D0FF280BD0122010BDA0
:10F30000FFF7E8FF611CF5F7F1FE08B1002010BD22
:10F31000072010BD0120F5F72BFFF7E710B500F02F
:10F320003FFF08B10C2010BDF5F728FF002010BDED
:10F330002DE9F843064600F0F5FB002812D130888D
:10F340000021FEF780FB04000ED000F01EFE58B135
:10F3500094F8A4028DF80000009800909DF8000039
:10F3600020B13A20BDE8F8830220FBE74FF0000807
:10F37000B088FEF70AFE054601460520FEF786FE28
:10F38000074629460820FEF781FEB84201D3AF4266
:10F3900001D31220E6E741F64C50854209D294F899
:10F3A0007200022803D194F87300022801D00C20C7
:10F3B000D8E7A4F8A872C4E9AB85F088A4F8B40231
:10F3C0003089A4F8B60204F52974FF2020700020CB
:10F3D000C8E710B50B46012200F11001F6F710F84E
:10F3E000002010BD10B500880121FEF72CFB18B1DC
:10F3F00090F8001311B107E0022010BD90F89E10A4
:10F40000152903D0162901D00C2010BD022180F847
:10F410000013002010BD10B50821F4F759FE00209C
:10F4200010BD10B50446FBF78DF8FFF718FA2070F1
:10F43000002010BD10B50446D820207000F0A2FDB9
:10F440006070002010BD082101700020704710B5C9
:10F45000044600F0A5FE08B10C2010BD207820B1B4
:10F46000012802D0FF2808D109E0FFF733FF611C13
:10F47000FEF768FD08B1002010BD122010BD00206D
:10F48000F5F776FEF7E71CB50446FBF75BF80020BE
:10F490008DF8020003218DF8011014F8011B8DF87E
:10F4A00003108DF800006846019400F065F91CBD5A
:10F4B0007FB50546FBF746F806462878002460B17C
:10F4C0008DF8004001200DF10101F5F72BFC20B172
:10F4D000684600F097F8002812D18DF80C403046AD
:10F4E000FFF7B1F918B18020ADF80D0001E0ADF8DB
:10F4F0000D408DF80F402878012803D038B1122034
:10F5000004B070BD03A93046FBF77CF8F8E730463D
:10F5100000F05CFDF4E730B58BB00446FBF712F861
:10F5200002462079042803D86088B0F5804F02D9BC
:10F5300012200BB030BD00258DF8045021790095C4
:10F540009DF80000052940F010008DF8000054D20D
:10F55000DFE801F0030805110B0040F0010040F066
:10F56000020006E040F0090001E040F0010040F038
:10F5700004008DF80000BDF800000090BDF8000008
:10F58000ADF805002188DDF8060061F31F20CDF8F5
:10F5900006006188DDF8090061F31F20CDF809003D
:10F5A000607B8DF80D0060798DF80E00A0798DF8E4
:10F5B0000F00D4F807000490B4F80B00ADF8140065
:10F5C000A07B8DF816007F208DF8170001208DF8A4
:10F5D00018008DF819508DF81A008DF81B50104640
:10F5E000FFF74FF98DF81C008DF81D508DF81E5057
:10F5F00009A901A8FAF79EFD9BE741F2CF01392046
:10F60000F4F7DCFC70B5044600780221FEF71BFA23
:10F61000050007D0FFF733FB60B12846FFF71BF961
:10F6200010B105E0422070BD2846FFF702F908B18D
:10F630000C2070BD611C2846FFF71AF9002070BD30
:10F6400010B50446012000F0DFFA28B12146012060
:10F65000F5F780FB002010BD0C2010BD1CB5017813
:10F660008DF8001040788DF801000020ADF8020000
:10F67000ADF804000146684600F0E0FB002802D126
:10F68000684600F0BBFB1CBD00B587B041798DF822
:10F69000001081798DF8011001218DF80210017898
:10F6A0008DF80310B0F8011040F27122514302911D
:10F6B000B0F803005043049007208DF81800002094
:10F6C0008DF819000498FAF731FF40B10298FAF763
:10F6D00021FF20B1684600F0DDF807B000BD302002
:10F6E000FBE71CB50446FAF72DFF00208DF800005B
:10F6F0008DF8020003208DF8010014F8010B8DF83D
:10F7000003006846019400F023F91CBD10B5F5F71D
:10F7100047FB002010BD1CB50C466946FEF71DFCDA
:10F72000002808D19DF8000030B100212246019840
:10F7300000F0CEFB00201CBD0121F7E710B5044608
:10F74000002000F061FA28B121460020F5F702FB05
:10F75000002010BD0C2010BD10B50446007800B18B
:10F760000120F9F79DFD207800B10120F8F792F80B
:10F77000002010BD00F050BC2DE9FC47064647783C
:10F7800000780221FEF75FF905000BD0FBF72CF89B
:10F7900058B12846FEF769FF0446F078A04205D824
:10F7A000044603E04220BDE8FC87F478042F31D002
:10F7B000686CFEF7B9FA20441FFA80F8FBF714F8DA
:10F7C000A0B9F0784FF0120918B12846FFF717F8E2
:10F7D00040B12846FEF749FF404507D22846FFF7CB
:10F7E00036F808B14846DEE70720DCE7FAF7FCFF09
:10F7F00002464146284600F026FA0028D3D1032FBE
:10F8000000D0C4B12846FFF722F8717803290DD043
:10F8100088B901E07CB9F5E7042907D12846FFF74C
:10F820002EFA40B1686CFEF74DFA20B1012F04D0DA
:10F83000032F02D00EE01220B5E72846FFF707F8A5
:10F8400008B1002202E0012F14D001226846696C41
:10F85000FEF7CDF9042F18D0726823460121686C99
:10F86000FEF7FDF90028BFD07078022804D00328E5
:10F8700002D00DE00222E9E7686CFEF755FA024675
:10F880000121686CFEF72CFA02E02846FEF704FF1F
:10F89000002088E710B58AB00446FAF713FD002867
:10F8A00003D100F088FB10B10C200AB010BD02217A
:10F8B00004F11000FAF764FEA0788DF80000A0783B
:10F8C0008DF81C0060788DF8210020788DF82000DC
:10F8D000207E8DF82200607E00B101208DF823008B
:10F8E000A078C10714D0E07800F0E9FA8DF81D0087
:10F8F000A068019020690290A078400715D5207972
:10F9000000F0DDFA8DF81F00E068059060690BE0FB
:10F91000022813D0400708D5E07800F0D0FA8DF81F
:10F920001F00A0680590206906906846F9F7BCFDA5
:10F930000028BAD107A8F8F77BF9B6E7E07800F01D
:10F94000BEFA8DF81E00A068039020690490ECE7D1
:10F950002DE9FC4106464578C77800780221FEF77C
:10F9600072F8040007D0FAF73FFF40B12046FEF7D7
:10F9700072FF18B103E04220BDE8FC810027606CF3
:10F98000FEF7D6F938441FFA80F8FAF72DFF28B9A8
:10F99000F07818B12046FEF75EFF98B1FAF724FF21
:10F9A00002464146204600F04EF90028E4D1042DDD
:10F9B00008D0032D0AD02FB12046FFF760F918B107
:10F9C0000C20D9E71220D7E7012D0CD12046FEF7F5
:10F9D0003EFF08B1042202E0012D10D00522684646
:10F9E000616CFEF704F972683B460021606CFEF71B
:10F9F00036F930B1022D06D0032D04D008E00622DE
:10FA0000EDE70720B8E742460021606CFEF768F991
:10FA10000020B1E710B5044601460020F5F782F951
:10FA200010B900202060A080002010BD10B5FAF7AA
:10FA3000E7FE002010BD00F096B82DE9F0478AB02F
:10FA400089460546008804A9FEF787FA002847D1B1
:10FA500005980146884690F8BC1100F59C748DF815
:10FA60001810069906919DF81810903009B10127D9
:10FA700000E00027817B222900D13FB100266230BF
:10FA800008218246FFF71DFC10B107E00126F6E7CA
:10FA90000B215046FFF715FC00B906B302A80090F1
:10FAA0009DF8100001AB2A46414600F04BFA0600D3
:10FAB00016D198F877000C3468B19DF8040010F066
:10FAC00002019DF808008DF8041000F002008DF886
:10FAD000080008D038B1FF20607047B905E01A204F
:10FAE0000AB0BDE8F0870920FAE7207808B13A2685
:10FAF00014E084F800909DF80410A1709DF80800AF
:10FB0000E070AA88A2808DF818108DF81900A888D6
:10FB1000ADF81A0006A94046FEF780FA0020607092
:10FB20003046DDE710B504460020228886B0A2F5F5
:10FB30007F41FF3908D003A91046FEF70EFA10B135
:10FB4000022006B010BD04982189A38962898DE83E
:10FB50000E00E388A2886188FAF72EFC08B1002025
:10FB6000EFE73020EDE710B5FEF776F9F5F7D4F9B9
:10FB7000FAF7B8FEF6F7F8F80120FAF73BFEBDE811
:10FB80001040FAF75FBC4FF4A471884203D34FF4DE
:10FB90002961884200D3084680B27047410701D5E9
:10FBA00008207047C10701D001207047800701D5A8
:10FBB000022070470020704710B501280BD00228A2
:10FBC00009D0042806D0082804D040F2A921062034
:10FBD000F4F7F4F9032010BD0EB569460220FDF7D5
:10FBE0003CFF50B14FF4A3713920F4F7E7F90298C4
:10FBF000FFF745F808B101200EBD6846F4F71CFC7C
:10FC00000028F4D000200EBD10B50446FFF7E4FF35
:10FC100070B1FAF7E9FD50B1FAF794FC0446FEF72B
:10FC20001AFE60B92046FEF704FE08B107E034B1C1
:10FC300000F0C1F928B1F8F78FF8012801D00020B1
:10FC400010BD012010BD70B50C46054612B11F292C
:10FC50000CD816E0F4F7E6FEA04201D2072070BDF2
:10FC60002846FEF7F4FD18B11F2C01D9122070BDF3
:10FC70002846FEF7F7FD30B121462846FEF77CFD09
:10FC800018B1002070BD422070BD452070BD10B578
:10FC900004464078C00613D4FAF70EFE800705D458
:10FCA000207D022829D0A07D022826D0FAF704FE64
:10FCB000400705D4207D03281FD0A07D03281CD039
:10FCC0006078C00702D0FAF7CDFDB0B16078C10608
:10FCD00005D4010703D5207D02280ED10FE0217D38
:10FCE000022901D0A17E41B9000708D4D4F805004B
:10FCF0004FF48041B1EB102F01D2112010BD002034
:10FD000010BD38B504460078EF285CD8B4F801007F
:10FD1000ADF80000009800F014FAA0B36078010775
:10FD20000BD4D4F80210D4F805300A0AB2EB132F22
:10FD300049D82022B2EB112F45D8617A19B307298F
:10FD400041D8A17A29B1012903D0022901D0032980
:10FD500039D1420703D4022901D0032905D1E17A20
:10FD600009B101292FD1410707D4A17C29B101296B
:10FD700003D0022901D0032925D1C10604D5207D55
:10FD8000012820D11BE01EE0217D02290BD1C107F3
:10FD900019D0410717D4010715D5410613D48106A0
:10FDA00011D481070FD4C00609D4A07D012803D047
:10FDB000022801D0032806D1E07D0F2803D8207E39
:10FDC00018B1012801D0122038BD002038BDFB2811
:10FDD00002D8B1F5296F01D9112070470020704772
:10FDE0001B38E12806D2B1F5A47F03D344F290205A
:10FDF000814201D9122070470020704710B5044697
:10FE00000078012809D0F9F749FB052803D0F9F754
:10FE1000BFFA002800D00C2010BDF7F7FBFE58B148
:10FE2000F7F77EFDF7F7F4FD0028F5D1A18860888B
:10FE3000BDE81040F9F754BA122010BD0278012A2B
:10FE400001D0BAB118E042783AB1012A05D0022AAD
:10FE500012D189B1818879B100E059B1418849B1A5
:10FE6000808838B101EB8101490000EB8000B1EBE3
:10FE7000002F01D2002070471220704770B5144641
:10FE80000D4608B101280CD1022B0CD019461046A2
:10FE9000FAF7A2FB78B12846FAF730FB58B1AC422A
:10FEA0000BD9122070BD1046FAF78AFB18B128460C
:10FEB000FAF77AFBF2E7302070BD002070BD012810
:10FEC00002D018B10020704702207047012070470F
:10FED0002DE9F0410546B0F85A70B0F85C4016467E
:10FEE000343011B1F9F7E2F901E0F7F7D9FC8046B7
:10FEF0000221FEF767F8874200D238460746022102
:10FF00004046FEF75FF8844200D2204629883180BF
:10FF10001B2F13D9FB2F00D3FB2777801B280FD96A
:10FF2000FB2800D3FB20F0804046FFF72CFEB0807A
:10FF30004046FFF728FE3081BDE8F0811B27ECE743
:10FF40001B20F0E72DE9F0419078069E1D461446EF
:10FF500008B9FAF7B1FCE478074614B9FAF7ACFC33
:10FF600004466FB164B13846FFF718FE2046FFF72C
:10FF700015FE2FB124B12F7034700020BDE8F08140
:10FF80000920FBE77F2000F0D5B808B590F8901263
:10FF900090F8BD008DF80000009800909DF80000DA
:10FFA00000B10120401E084203D0042901D00120E5
:10FFB00008BD002008BD10B5F9F770FA042803D079
:10FFC000052801D0002010BD012010BD70B50546E8
:10FFD000FEF748FC70B12846FEF751FE002808D015
:10FFE0002846FEF749FE04462846FEF71BFE18B1D8
:10FFF0000C2070BD422070BD64B12088F4F784FEEF
:020000021000EC
:1000000020880121F4F78AFA20B141F2FD4139201C
:10001000F3F7D4FF002070BDF0B585B0044600882A
:100020006946FDF79AFF00284ED1019890F8A81173
:100030008DF81010049904919DF81010903001B1C2
:1000400001218DF808109DF8001019B1C17B8906B7
:100050000FD405E0817B1E290BD001E0012100E0D7
:1000600000218DF80C1005216230FFF72AF928B124
:1000700007E09DF808100029F2D1EFE79DF80C0089
:1000800008B32189E088FFF7ABFE00281CD1A188C6
:100090006088FFF7A5FE002816D12189E088FFF7C8
:1000A00096FE002810D1A1886088FFF790FE060018
:1000B0000AD1019800F59D75FF276F709DF8081013
:1000C00021B13A2630E01A2005B0F0BD9DF80010AD
:1000D00071B3002102AAFFF7FBFE6188BDF80E0094
:1000E000814200D20846E880A188BDF81000814214
:1000F00000D208462881E288BDF80A108A4200D260
:10010000114669802289BDF80C108A4200D211463E
:1001100040F64802A980914200D31146A98090423E
:1001200000D202462A812F70002068703046CBE74B
:100130000121CFE708B540F688126946F3F7B2FD12
:1001400008BDC0B2C10615D481064FEAC07103D5FF
:1001500021BB810722D401E00029FAD101071BD578
:10016000C1071BD0810719D4410617D4410715D404
:1001700080060FE0410611D481060FD4C1074FEA73
:10018000807104D0002902DB400705D406E0010796
:1001900004D44007002801DB01207047002070478D
:1001A0003EB5FFF708FF10B1F7F7DEFD90B96946DD
:1001B0000220FDF752FC78B14FF4B2713920F3F709
:1001C000FDFE029C2046FEF75AFD28B12046FEF7B0
:1001D000BBFB08B101203EBD6846F4F72DF90028AD
:1001E000EFD000203EBD10B5F6F706F9BDE810408F
:1001F000FAF73EBB10B5F7F7BBFA08B1E72103E009
:10020000F6F70AF918B1EC210120F3F7D7FEBDE8A3
:1002100010400220FDF7F3BB026812B9016070477D
:100220000246506808B18A42FAD18A42F7D051603A
:10023000704710B5044602E0206880476468002CCF
:10024000FAD110BD10B5F7F779FCBDE81040FAF708
:100250001BBB10B5F8F7B2FF20B140F22D11012001
:10026000F3F7ACFEFAF71EF8F7F78CFCBDE8104088
:10027000F9F74ABF10B50121C1718171818004462F
:100280000421F3F717FF002802D12068401C2060EA
:1002900010BDF3F7BDB901000B0002000A00050014
:1002A00009000A000800140007001E0006003200C2
:1002B00005004B0004006400030096000200FA00F1
:1002C0000100F4010000C868FDF72BBD704790F8ED
:1002D0008C0008B1002070470120704710B5FAF774
:1002E000ADFFFAF73FFCFAF7D1FBBDE81040FAF793
:1002F00031BC10B504460846FBF734F94FF47A7167
:1003000000F2E730B0FBF1F0201A801E10BD10B5EE
:1003100004460846FBF726F94FF47A71B0FBF1F07A
:10032000201A10BD0A6802600B7903717047002122
:10033000016081807047D8D8D8D8D8D8D8D8D8D834
:10034000D8D8D8D8D8D8D8D8D8D8ECECECECF0F0AD
:10035000F0F0F4F4F4F4F8F8F8F8FCFCFCFC00001D
:1003600002030405060708D8D8D8D8D8D8D8D8D8D2
:10037000D8D8D8D8D8D8D8D8D8D8D8ECECECECF095
:10038000F0F0F0F4F4F4F4F8F8F8F8FCFCFCFC00FD
:1003900000000304555555252627010301010000DF
:1003A00010B5A2B01C4607480DF02EFA812301AA11
:1003B000A18820680DF0A5F901A903480DF024FAE1
:1003C00022B010BD880F0200980F020008B508493E
:1003D000084805F07FFE28B943F23430002109F0C7
:1003E000A7FE08BD014604480DF00EFAF9E700BF6C
:1003F000A103010050030020AC0F020008B500204B
:1004000005F06AF898B90E480DF0FEF9FFF7DEFF27
:1004100046F26760002109F08BFE05F0F3FE01460D
:1004200050B943F23430002109F082FEFEE7014664
:1004300004480DF0E9F908BD03480DF0E5F9FAE7C5
:10044000F00F0200D00F0200081002002DE9F04F5B
:1004500091B00646934601931A9F029159B196F8BE
:100460000280CDF80080B8F1000F08D017F0010F1E
:1004700010D1002304E00DF0DAF80290EFE700233A
:1004800096F803A0BAF1000F06D017F0020F1DD1A5
:10049000002202E00123F3E7002202B9C3B135785C
:1004A000AA00039206EB8505BBF1000F1CD0002BC0
:1004B00040F08680009B002B00F08E8017F0040F28
:1004C00040F08E800020814680467CE00122E4E7F7
:1004D000BBF1000F03D0019A02993046D847029C25
:1004E000204611B0BDE8F08F029C03BB009BA3B374
:1004F00017F0040928D01D444FF0000924E00444FB
:10050000013508F10108D0451BD22A78002356F89E
:100510002220194658460DF09FF8002FEFD01C9B63
:100520009945ECD227F8190009F10109E7E74FF0E6
:100530000008C146CDF804A0DDF800A01A971B9F63
:10054000E1E7DDF804A01A9F07F0050300934FF0E0
:100550000008CDF804B0B34623E0DDF80090F3E7DF
:1005600000231E4613B117F0010F03D196B917F0FF
:10057000020F0FD00023194601980DF06DF81B9B58
:100580003BB11C9B994504D21B9B23F8190009F130
:100590000109044416B1009B03B9013C013508F17F
:1005A0000108D0459CD22B785BF823206B4B9A42F4
:1005B000D6D36B4B9A4201D30023D2E70123D0E775
:1005C0000BA84FF0000918B1009A29460EF07BF9EC
:1005D000009B1D44002317E0002081468046F2E77F
:1005E000C14607A84FF00008EDE7002139B317F026
:1005F000010F18D008F1010110A8804408F8142C4C
:100600005FFA81F80135013353452DD22A7856F827
:10061000221052488142E8D35148814201D300213F
:10062000E4E70121E2E717F0040FEBD009F1010143
:1006300010A8814409F8242C5FFA81F9E2E717F049
:10064000020F08D008F1010110A8804408F8142C0A
:100650005FFA81F8D6E709F1010110A8814409F891
:10066000242C5FFA81F9CDE733788DF83C3073782C
:1006700043448DF83D3017F0020F0AD000238DF867
:100680003F3017F0010F06D117F0040F32D10023CD
:1006900002E04B46F3E700238DF83E3030680690C9
:1006A0000F983060019F3A4603993046D847041EA0
:1006B000FFF616AF0698306001973A46494607A8FC
:1006C000D847002843DB27180098039B18440146AD
:1006D0005144DDF804904A46029B591A2846D847EF
:1006E000041EFFF6FDAE3D19002700965E46DDF8BC
:1006F0006CB015E04B46CFE74FF0000A4A460121A7
:100700000DF11700B047002823DB0544534622466D
:10071000494630460CF0A0FF00281CDB0544013799
:10072000B8450EDD10AB3B4413F8143C8DF8173080
:10073000009A52F82340BBF1000FDDD03BF817A020
:10074000DCE7019A00210846B0472C46C8E604467B
:10075000C6E60446C4E60446C2E600BF180B020023
:100760005025020008B5024B1B68984708BD00BF22
:1007700064030020014B1860704700BF6403002031
:1007800000B583B002460B4600210091024800F0FC
:1007900053FA03B05DF804FB6507010010B586B09D
:1007A00004460390049100210591009103A9064895
:1007B00000F042FA059B049A934201DA0022E254C7
:1007C000059806B010BD00BFD9D701002DE9F04350
:1007D00083B0044608461546238B13F0080F05D155
:1007E00003F0070600230093019369E0012909D073
:1007F00043F02003238385F31188BFF36F8F03B089
:10080000BDE8F08343F010032383F4E720460DF0A6
:100810003EF857E0D4F814904A46694620460DF059
:100820004FF800275AE023691F68062120460DF083
:1008300007F84FF0000951E023695F680421204662
:100840000CF0FEFF4FF0000948E023699F68052186
:1008500020460CF0F5FF4FF000093FE0002246E093
:10086000002244E043F00803238385F31188BFF39B
:100870006F8F002944D1009B2BB14B4642466946FD
:1008800020460DF094F817B125492046B8474FF09F
:100890004003EFF3118583F31288BFF36F8F238B2F
:1008A00023F008032383238B13F0100F2ED023F0A3
:1008B000100323830120268B06F0070600289AD018
:1008C0000228A3D0002896D00128A3D00328AAD0BC
:1008D0000428B1D00528B8D00027B946238B03F0EF
:1008E0000708B045BAD0A268002AB9D00122114643
:1008F000002AB7D1009A002AB4D1002FB2D1D2E792
:100900004A46414620460CF0A3FFB4E713F0200FFF
:1009100004D023F0200323830220CCE70020CAE781
:10092000DDD9010070B582B0044600230360436046
:1009300083604B78252B02D04E1C01251FE0881CBC
:10094000E37045E1237843F004032370B5B1013629
:1009500014E0237843F008032370F7E7237843F08B
:1009600010032370F2E7237843F020032370EDE7B0
:10097000237843F040032370E8E7002545B333783C
:10098000203B102BF9D801A252F823F05D09010099
:100990007B0901007B090100670901007B09010057
:1009A0007B0901007B0901007B0901007B09010033
:1009B0007B0901007B090100530901007B0901004B
:1009C000450901007B0901007B0901007109010053
:1009D000237803F04403442B5FD00196237843F03F
:1009E0008003237033782A2B5CD001A80DF089FA9C
:1009F000019B9E420FD0237843F0800323706060F8
:100A0000DBB2C3F34003002854DB002213432278F7
:100A100063F341022270019B01931B782E2B14BFBC
:100A200000230123627863F341026270002B43D0FC
:100A3000019B5A1C01925B782A2B3FD001A80DF034
:100A400060FAA0602378C3F3400300283EDB002255
:100A50001343227863F341022270019803784C3BE0
:100A60002E2B00F29D80DFE803F0909B9B9B9B9BCD
:100A70009B9B9B9B9B9B9B9B9B9B9B9B9B9B9B9BC6
:100A80009B9B9B9B9B9B339B579B459B9B9B9B9BB8
:100A90009B9B899B9B9B9B9B820023786FF3861378
:100AA00023709AE7637843F00103637033460133A0
:100AB0000193B1E70122A9E70198CFE7637843F0FA
:100AC00004036370104601300190C7E70122BFE7BD
:100AD000421C4378682B06D06378022161F3C60379
:100AE000637010461EE06378012262F3C6036370F0
:100AF000023017E0421C43786C2B06D06378032148
:100B000061F3C603637010460CE06378042262F35D
:100B1000C6036370023005E06378052262F3C60302
:100B20006370013010F8013BE370A3F14102372AF2
:100B30007DD8DFE802F05E7C7C7C5E5E5E7C7C7C47
:100B40007C7C7C7C7C7C7C7C7C7C7C7C7C4F7C7C12
:100B50007C7C7C7C7C7C5E7C4F3A5E5E5E7C3A7CFE
:100B60007C7C7C654F717C7C717C4F7C7C4F637896
:100B7000062262F3C60363700130D3E7637807226D
:100B800062F3C60363700130CCE76378082262F336
:100B9000C60363700130237843F002032370C1E77A
:100BA00063786FF3C6036370BCE7A278012161F339
:100BB0000202A270627802F07802402A10D0632B01
:100BC00013D02378C3F34002154365F34103237028
:100BD00002B070BDA278022161F30202A270E9E7BF
:100BE000217841F001012170E9E7151E18BF0125A8
:100BF000E7E7A378042262F30203A3700125E0E78C
:100C0000A378032262F30203A370637803F07803EE
:100C1000402BD6D10125D4E7A378032262F3020347
:100C2000A370637813F0780FCBD00125C9E7237840
:100C300043F001032370C4E72DE9F04F91B006465D
:100C40000D4691460393002499F80000002800F017
:100C5000D582252808D009F101092946B047002886
:100C6000C0F2CD820134EFE700230493059306938D
:100C7000079308930993494606A8FFF753FE02908D
:100C80009DF8193013F0010F00F09780039B1A1D97
:100C900003921F68002FC0F288809DF8193013F06E
:100CA000040F00F09C80039B1A1D0392D3F800A050
:100CB000BAF1000FC0F28A800023079308939DF8D1
:100CC0001A3003F007039DF81910C1F3C301012B7B
:100CD00000F08E80022B00F0D380042B00F02481E2
:100CE000032B00F03B819DF8188018F0030B40F0B7
:100CF0003B819DF81B30253B532B00F2E681DFE85A
:100D000013F04001E401E401E401E401E401E40141
:100D1000E401E401E401E401E401E401E401E401AB
:100D2000E401E401E401E401E401E401E401E4019B
:100D3000E401E401E401E401E401E401E401E4018B
:100D4000E401E401E401E401E401E401E401E4017B
:100D5000E401E401E401E401E401E401E401E4016B
:100D6000E401E401E401E4018101E401E401E401BE
:100D7000E401E401E401E401E401E401E4015E01D1
:100D80006701E401E401E401E4016701E401E40135
:100D9000E401E401BE018101A201E401E4014D018D
:100DA000E4018101E401E40181019DF8183043F080
:100DB00004038DF818307F426FE79DF91830002B3F
:100DC00002DB4FF0FF3768E7079F66E79DF81930B1
:100DD0006FF341038DF819304FF0FF3A6CE713F0D1
:100DE000020F02D0DDF820A066E74FF0FF3A63E77C
:100DF000CB1E042B04D8DFE803F00B1D293535008A
:100E0000039B1A1D03921B68DA170493059206E0F0
:100E1000039B1A1D03921B68DA170493059201299C
:100E200028D002297FF45FAFBDF91030DA170493A0
:100E3000059258E7039B073323F0070303F10802E9
:100E40000392D3E90023CDE90423E8E7039B0733AA
:100E500023F0070303F108020392D3E90023CDE94D
:100E60000423DCE7039B1A1D03921B68DA17049323
:100E70000592D4E79DF91030DA170493059232E712
:100E8000CB1E042B04D8DFE803F00B1F35414100D3
:100E9000039B1A1D03921B680493002305931EE015
:100EA0009DF81B30632B07D0039B1A1D03921B6810
:100EB00004930023059312E0039B1A1D03921B6801
:100EC0000493002305930AE0039B073323F00703F1
:100ED00003F108020392D3E90023CDE90423012999
:100EE0001CD002297FF4FFAEBDF81030049300231C
:100EF0000593F8E6039B073323F0070303F1080289
:100F00000392D3E90023CDE90423E8E7039B1A1DEC
:100F100003921B68049300230593E0E79DF81030CB
:100F2000049300230593DEE608290BD0039B0733C7
:100F300023F0070303F108020392D3E90023CDE96C
:100F40000423D0E6039B073323F0070303F10802D1
:100F50000392D3E90023CDE90423C4E6039B1A1DC1
:100F600003921B680493BEE6029F3B464A4629460D
:100F700030460DF042F80028C0F241810444B946E1
:100F800062E629462520B0470028C0F238810134A6
:100F9000D8460DF13E0A4FF000099BE0DDF81090B5
:100FA000BAF1000F07DB514648460DF05DFC09EB36
:100FB000000AD8468EE048460DF04DFCF7E7049B4A
:100FC0008DF82830D8460DF1290A0DF1280981E065
:100FD00018F0080F05D118F0100804D04FF02008C1
:100FE00001E04FF02B08049A059B002B02DB0492D2
:100FF000059308E0524263EB4303049205934FF0DC
:101000002D0800E0D8460DF13E0300930AAB06AA76
:10101000DDE904010CF087FF8146BAF1000FC0F250
:1010200088800DF13E03A3EB09039DF818206FF3B0
:1010300086128DF818209A457ED9AAEB03030793F0
:101040000DF13E0A46E0049828B9D846DFF8B4A16D
:10105000AAF105093EE00DF13E0300930AAB06AA92
:1010600000210CF060FF81469DF81A3043F0100318
:101070008DF81A3078238DF81B30D846CDE7049AC6
:101080009DF81930C3F3C303072B06D8DFE803F03C
:10109000040B0D0F1115191B1460D8460DF13E0AF3
:1010A0004FF0000916E01470F7E71480F5E71460BC
:1010B000F3E7E31714605360EFE7E317146053603E
:1010C000EBE71460E9E71460E7E7D8460DF13E0A64
:1010D0004FF00009B9F1000F00F08D80AAEB090371
:1010E000B8F1000F00D001339DF81A2012F0100F54
:1010F00025D0023307990B4412F0400F01D0089A13
:101100001344002F31DDFF1A9DF8183013F0040F3F
:101110002BD113F0400F17D0B8F1000F17D029468C
:101120004046B04700286ADB0134D8464FF0300B08
:101130000FE00DF13E0ACDE70DF13E0ACAE712F0CD
:10114000080FD7D00133D5E74FF0200B01E04FF067
:10115000300B3B465F1E002B07DD29465846B04743
:1011600000284CDB01343B46F4E7B8F1000F05D012
:1011700029464046B047002841DB01349DF81A302B
:10118000C3F30012C3F3C003134305D02946302034
:10119000B047002833DB01349DF81A3013F0100FEC
:1011A00006D029469DF81B00B047002827DB0134F4
:1011B000079B03F1FF38002B07DD29463020B0479D
:1011C00000281CDB01344346F3E753464A462946D0
:1011D00030460CF012FF002811DB0444002F07DD1D
:1011E00029462020B047002809DB0134013FF5E7FC
:1011F000DDF8089028E5DDF8089025E5204611B0D7
:10120000BDE8F08F2D10020008B54FF04002EFF35B
:10121000118382F31288BFF36F8F02F0C9FB03487A
:101220000CF0F2FA01F06AF8FCE700BF301002009F
:1012300006F080BEF8B50646002400E001340E4BEF
:101240000E4A9B1AB4EB231F14DA0C4D05EB041560
:101250006B685B79002BF1D0314628460DF099F987
:101260000028EBD02701054BDB591B683146284687
:101270009847E3E7F8BD00BFF00E0200D00E020071
:1012800070B506460D46002403E02A4631469847CD
:101290000134084B084A9B1AB4EB231F08DA2301D8
:1012A000054A02EB04109B589B69002BEDD1EFE738
:1012B00070BD00BFF00E0200D00E02002DE9F0411B
:1012C000074605460AE007EA0807144B03EB061633
:1012D000736804221968204600F07CFAD5B195FAAB
:1012E000A5F6B6FA86F60D4C04EB06140123B340BE
:1012F0006FEA030825EA0305237B002BEED03301B8
:10130000064AD3581B69002BDDD020469847002899
:10131000E4D1D8E73846BDE8F08100BFD00E020026
:101320002DE9F04780460F46284BBFF35B8F53E80B
:10133000006F721C43E800210029F8D1BFF35B8FD6
:10134000002E3ED100240AE0214B03EB0919D9F805
:10135000043004221968284600F03CFA01341D4B81
:101360001B4A9B1AB4EB231F1BDAA146184D05EB51
:1013700004152B7B002BF1D02301154A52F803A052
:10138000DAF80C300BB128469847DAF81030002B09
:10139000DAD0284698470028D6D00123A3401E4320
:1013A000DCE7B8F1000F0DD066B13046FFF786FFDD
:1013B0000646002FF8D04FF4A470002108F0B8FEC4
:1013C000F2E700263046BDE8F08700BFB01E0020DF
:1013D000D00E0200F00E020008B5064B186018B1DE
:1013E000054B1B68092B00DC08BD044808F03AF9DE
:1013F000FAE700BFF41E0020A81E00208C05002084
:1014000008B5024808F02EF908BD00BF8C05002081
:1014100030B589B000220F490F480FF0AFFA0F4DD9
:1014200000220023CDE90623002404940E23039315
:101430000294019400940A4B4FF4407209492846E3
:101440000EF0D7FE0849284607F01EFF204609B0D7
:1014500030BD00BF01140100E01800201819002061
:1014600045170100803A00205C100200014B53F840
:10147000200070476810020038B108B5044A1060B7
:10148000084600F003FC002008BD6FF0150070470F
:101490006803002008B5054B1B781BB1034B0122E4
:1014A0001A7008BD024808F0DDF8F7E7503A00204E
:1014B0008C0500200D4BBFF35B8F53E8002F0132EA
:1014C00043E800210029F8D1BFF35B8F00B97047D2
:1014D000074BBFF35B8F53E8002F013A43E800212D
:1014E0000029F8D1BFF35B8FF1E700BFAC1E0020ED
:1014F000A81E0020064B00200246BFF35B8F53E876
:10150000000F43E800210029F9D1BFF35B8F70473A
:10151000AC1E002038B5FFF7EDFF0546002400E0C3
:1015200001340B4B0B4A9B1AB4EB231F0FDA09480B
:1015300000EB041043685B79002BF1D02301054ACE
:10154000D3585B68002BEBD029469847E8E738BDB5
:10155000F00E0200D00E0200034B18680028D4BF22
:1015600000200120704700BFAC1E002008B50249D2
:1015700002480CF01CFE08BD74100200B41E0020CE
:1015800008B50023054A1370054A13604FF4004163
:101590000448FFF771FFFFF7E9FF08BD513A00204B
:1015A000AC1E002097E5010008B50146002200238B
:1015B00001480CF023FE08BDB41E002008B5024807
:1015C0000CF019FF08BD00BFB41E002008B501468D
:1015D00001480CF081FF08BDB41E002008B5024888
:1015E0000CF0B7FF08BD00BFB41E0020114B1878E7
:1015F00000B9704710B5FFF7E1FF044688B10E4B04
:10160000BFF35B8F53E8002F013A43E80021002924
:10161000F8D1BFF35B8F2046FFF70CFE2046FFF7A3
:10162000D5FFFFF799FF10B9FFF7D8FF10BDFFF7FF
:1016300071FFF9E7503A0020A81E0020134B1B78D9
:1016400003B1704710B500210120FFF769FE0024A7
:1016500000E001340E4B0F4A9B1AB4EB231F0CDA47
:101660000C4800EB041043685B79002BF1D0230198
:10167000084AD3589B689847EBE7FFF7B7FF002865
:10168000FBD1024B01221A7010BD00BF513A00205D
:10169000F00E0200D00E020010B582B01B4BBFF35B
:1016A0005B8F53E8002F511C43E800100028F8D14D
:1016B000BFF35B8F164B1B7863B9164B1B68BBB12E
:1016C000C2B10A2A14D114480FF064F9134807F084
:1016D000C9FF0DE04FF04003EFF3118483F312884C
:1016E000BFF36F8FFFF782FF84F31188BFF36F8F13
:1016F00002B010BD00220023CDE900234FF40042C8
:101700000023054808F072FFF2E700BFA81E002082
:10171000513A0020F41E0020E01800208C05002023
:1017200010B50446054B1B689847A0602146044845
:101730000CF000FEFFF7B0FF10BD00BF68030020F3
:10174000B41E00202DE9F04100210846FFF7E8FD16
:10175000804640B140F26766002708F015FDFFF7AC
:101760003BFE002515E04FF0FF364FF0FF37F4E762
:101770004046FFF7A3FD804670B94FF0FF364FF0AB
:10178000FF3709E02C4632463B46094807F092FFF6
:101790002546B8F1000FEBD1FFF728FF04460028DB
:1017A000F6D1002DEED000210846FFF769FDEAE7EB
:1017B0008C050020054B064A9B1AB1EBD30F02D2D1
:1017C00052F8310070470020704700BFD00E020071
:1017D000380E020008B5074BC31A1B1101334268CB
:1017E000137143681960436801225A71FFF752FE72
:1017F00008BD00BFD00E02002DE9F0478AB00546B3
:101800001E460F46C1F34924002C35D090460022D5
:101810000792089209920423029305AB01930223D5
:10182000009307AB21464046FEF710FEC0F30909BE
:1018300069F35227C7F3CB404844173020F0070024
:101840008008FFF7B1FE824600B300F11003079352
:10185000CDF820900022099263B1114A042302932B
:1018600005AB01930223009307AB21464046FEF7E8
:10187000EDFD0BE00022F1E7C1F3CB410C4417343E
:1018800024F00704A008FFF78FFE824633463A464D
:10189000294650460CF0A0FE0AB0BDE8F08700BF14
:1018A000ADE501000EB400B584B0014605AB53F8B8
:1018B000042B0393002000900348FFF7BDF904B008
:1018C0005DF804EB03B07047B5E6010030B585B0B4
:1018D00011F0440F05D01A4B1C6834B9002005B034
:1018E00030BD1849FFF7DEFFF9E7174B1968B2FB67
:1018F000F1F1B1FBF4FC154AA2FB0C32D20A4FF411
:10190000616E0EFB12CE124BA3FB0E535B0904FB60
:101910001C114FF47A7C0CFB01F1B1FBF4F505FBD3
:1019200014110CFB01F1B1FBF4F102910195C3EB31
:101930000311AEEB810100910649FFF7B3FFCEE73B
:10194000F81E002088100200FC1E0020C5B3A291E2
:10195000898888889410020061B108B52AB1064AC6
:1019600052F8232012B9054A00E0044A0449FFF75F
:1019700099FF08BD704700BF0C110200B0100200B3
:10198000601A02002DE9F041054617461E46DDF8B3
:10199000188099B900242EB1324612492846FFF723
:1019A00081FF0444B8F1000F17D087B10123079AD3
:1019B000934013F0100F13D10B4909E00B4B079A1A
:1019C00053F822200A49FFF76DFF0446E3E7064972
:1019D00042462846FFF766FF04442046BDE8F081F2
:1019E0000449F5E7CC100200B810020048110200CB
:1019F000C4100200C01002002DE9F04F85B005466A
:101A00000C46164603939DF8408001F0020B01F04E
:101A1000010AC1F3C0090CF0C7FDD8B10246124952
:101A20002846FFF73FFF0746BBF1000F14D142469F
:101A3000514628460CF0FEFDCDF804800F9B009324
:101A40000E9B324649462846FFF79CFF384405B0B6
:101A5000BDE8F08F0027E7E7039A21462846FFF705
:101A600035FF0744E3E700BFD010020011F0100F6C
:101A70000BD108B511F0200F03D00449FFF712FF76
:101A800008BD0349FFF70EFFFAE77047F82402008C
:101A90002C2402002DE9F04105460F4616469846D3
:101AA0000699FFF7E3FF0024444505DA2349284659
:101AB000FFF7F8FE0134F7E7002409E01F49284644
:101AC000FFF7F0FE0BE01E492846FFF7EBFE01345E
:101AD0000F2C0CDC002C02DD14F0070FEED0B4420A
:101AE000F1D23A5D17492846FFF7DCFEEFE71649C9
:101AF0002846FFF7D7FE002409E010492846FFF7E3
:101B0000D1FE0BE011492846FFF7CCFE01340F2C23
:101B100012DC002C02DD14F0070FEED0B44206D226
:101B20003A5DA2F120035E2BECD92E22EAE70349AD
:101B30002846FFF7B7FEE9E7BDE8F081C8100200CC
:101B4000DC100200D4100200E0100200E4100200D9
:101B50002DE9F04184B004469DF828500B9F0D9E5E
:101B60008DB94FF0000837B1BDB914483B46224645
:101B700013490BF088FD96B9D5B920460CF08DFDC0
:101B800004B0BDE8F0810295019300920B4600225B
:101B90000E99FFF731FF8046E5E70A48E6E70E9B1E
:101BA0000093434632460C9920460CF05BFDE3E778
:101BB0002A460E9920460CF049FDDEE7EDE60100CD
:101BC00025E60100B5E601002DE9F04387B00646A1
:101BD0000C469046D1F808900F88C7F382174B68DF
:101BE0000878C0F3C20033B11149591A41F3CF014B
:101BF000002919DA0023214651F8105BC5F3492565
:101C00006288C2F3CB02481905B90021CDF81080D3
